Archive member included because of file (symbol)

/opt/toolchains/n64/mips64-elf/mips64-elf/lib/libm.a(lib_a-s_sin.o)
                              ../y3d/y3d_yeti.o (sin)
/opt/toolchains/n64/mips64-elf/mips64-elf/lib/libm.a(lib_a-w_pow.o)
                              ../y3d/y3d_yeti.o (pow)
/opt/toolchains/n64/mips64-elf/mips64-elf/lib/libm.a(lib_a-e_pow.o)
                              /opt/toolchains/n64/mips64-elf/mips64-elf/lib/libm.a(lib_a-w_pow.o) (__ieee754_pow)
/opt/toolchains/n64/mips64-elf/mips64-elf/lib/libm.a(lib_a-e_rem_pio2.o)
                              /opt/toolchains/n64/mips64-elf/mips64-elf/lib/libm.a(lib_a-s_sin.o) (__ieee754_rem_pio2)
/opt/toolchains/n64/mips64-elf/mips64-elf/lib/libm.a(lib_a-e_sqrt.o)
                              /opt/toolchains/n64/mips64-elf/mips64-elf/lib/libm.a(lib_a-e_pow.o) (__ieee754_sqrt)
/opt/toolchains/n64/mips64-elf/mips64-elf/lib/libm.a(lib_a-k_cos.o)
                              /opt/toolchains/n64/mips64-elf/mips64-elf/lib/libm.a(lib_a-s_sin.o) (__kernel_cos)
/opt/toolchains/n64/mips64-elf/mips64-elf/lib/libm.a(lib_a-k_rem_pio2.o)
                              /opt/toolchains/n64/mips64-elf/mips64-elf/lib/libm.a(lib_a-e_rem_pio2.o) (__kernel_rem_pio2)
/opt/toolchains/n64/mips64-elf/mips64-elf/lib/libm.a(lib_a-k_sin.o)
                              /opt/toolchains/n64/mips64-elf/mips64-elf/lib/libm.a(lib_a-s_sin.o) (__kernel_sin)
/opt/toolchains/n64/mips64-elf/mips64-elf/lib/libm.a(lib_a-s_fabs.o)
                              /opt/toolchains/n64/mips64-elf/mips64-elf/lib/libm.a(lib_a-e_pow.o) (fabs)
/opt/toolchains/n64/mips64-elf/mips64-elf/lib/libm.a(lib_a-s_finite.o)
                              /opt/toolchains/n64/mips64-elf/mips64-elf/lib/libm.a(lib_a-w_pow.o) (finite)
/opt/toolchains/n64/mips64-elf/mips64-elf/lib/libm.a(lib_a-s_floor.o)
                              /opt/toolchains/n64/mips64-elf/mips64-elf/lib/libm.a(lib_a-k_rem_pio2.o) (floor)
/opt/toolchains/n64/mips64-elf/mips64-elf/lib/libm.a(lib_a-s_fpclassify.o)
                              /opt/toolchains/n64/mips64-elf/mips64-elf/lib/libm.a(lib_a-w_pow.o) (__fpclassifyd)
/opt/toolchains/n64/mips64-elf/mips64-elf/lib/libm.a(lib_a-s_lib_ver.o)
                              /opt/toolchains/n64/mips64-elf/mips64-elf/lib/libm.a(lib_a-w_pow.o) (__fdlib_version)
/opt/toolchains/n64/mips64-elf/mips64-elf/lib/libm.a(lib_a-s_matherr.o)
                              /opt/toolchains/n64/mips64-elf/mips64-elf/lib/libm.a(lib_a-w_pow.o) (matherr)
/opt/toolchains/n64/mips64-elf/mips64-elf/lib/libm.a(lib_a-s_nan.o)
                              /opt/toolchains/n64/mips64-elf/mips64-elf/lib/libm.a(lib_a-e_pow.o) (nan)
/opt/toolchains/n64/mips64-elf/mips64-elf/lib/libm.a(lib_a-s_rint.o)
                              /opt/toolchains/n64/mips64-elf/mips64-elf/lib/libm.a(lib_a-w_pow.o) (rint)
/opt/toolchains/n64/mips64-elf/mips64-elf/lib/libm.a(lib_a-s_scalbn.o)
                              /opt/toolchains/n64/mips64-elf/mips64-elf/lib/libm.a(lib_a-e_pow.o) (scalbn)
/opt/toolchains/n64/mips64-elf/mips64-elf/lib/libm.a(lib_a-s_copysign.o)
                              /opt/toolchains/n64/mips64-elf/mips64-elf/lib/libm.a(lib_a-s_scalbn.o) (copysign)
/opt/toolchains/n64/mips64-elf/lib/libdragon.a(n64sys.o)
                              main.o (data_cache_hit_writeback_invalidate)
/opt/toolchains/n64/mips64-elf/lib/libdragon.a(interrupt.o)
                              main.o (register_VI_handler)
/opt/toolchains/n64/mips64-elf/lib/libdragon.a(entrypoint.o)
                              (_start)
/opt/toolchains/n64/mips64-elf/lib/libdragon.a(dragonfs.o)
                              main.o (dfs_init)
/opt/toolchains/n64/mips64-elf/lib/libdragon.a(audio.o)
                              main.o (audio_init)
/opt/toolchains/n64/mips64-elf/lib/libdragon.a(display.o)
                              main.o (__safe_buffer)
/opt/toolchains/n64/mips64-elf/lib/libdragon.a(controller.o)
                              main.o (controller_init)
/opt/toolchains/n64/mips64-elf/lib/libdragon.a(graphics.o)
                              main.o (graphics_make_color)
/opt/toolchains/n64/mips64-elf/lib/libdragon.a(rdp.o)
                              main.o (rdp_init)
/opt/toolchains/n64/mips64-elf/lib/libdragon.a(dma.o)
                              /opt/toolchains/n64/mips64-elf/lib/libdragon.a(dragonfs.o) (dma_read)
/opt/toolchains/n64/mips64-elf/lib/libdragon.a(timer.o)
                              main.o (timer_init)
/opt/toolchains/n64/mips64-elf/lib/libdragon.a(inthandler.o)
                              /opt/toolchains/n64/mips64-elf/lib/libdragon.a(entrypoint.o) (inthandler)
/opt/toolchains/n64/mips64-elf/lib/libdragon.a(exception.o)
                              /opt/toolchains/n64/mips64-elf/lib/libdragon.a(inthandler.o) (__onCriticalException)
/opt/toolchains/n64/mips64-elf/mips64-elf/lib/libc.a(lib_a-assert.o)
                              stb_image.o (__assert_func)
/opt/toolchains/n64/mips64-elf/mips64-elf/lib/libc.a(lib_a-errno.o)
                              /opt/toolchains/n64/mips64-elf/mips64-elf/lib/libm.a(lib_a-w_pow.o) (__errno)
/opt/toolchains/n64/mips64-elf/mips64-elf/lib/libc.a(lib_a-fclose.o)
                              stb_image.o (fclose)
/opt/toolchains/n64/mips64-elf/mips64-elf/lib/libc.a(lib_a-fflush.o)
                              /opt/toolchains/n64/mips64-elf/mips64-elf/lib/libc.a(lib_a-fclose.o) (_fflush_r)
/opt/toolchains/n64/mips64-elf/mips64-elf/lib/libc.a(lib_a-findfp.o)
                              /opt/toolchains/n64/mips64-elf/mips64-elf/lib/libc.a(lib_a-fclose.o) (__sinit)
/opt/toolchains/n64/mips64-elf/mips64-elf/lib/libc.a(lib_a-fiprintf.o)
                              /opt/toolchains/n64/mips64-elf/mips64-elf/lib/libc.a(lib_a-assert.o) (fiprintf)
/opt/toolchains/n64/mips64-elf/mips64-elf/lib/libc.a(lib_a-fopen.o)
                              stb_image.o (fopen)
/opt/toolchains/n64/mips64-elf/mips64-elf/lib/libc.a(lib_a-fread.o)
                              stb_image.o (fread)
/opt/toolchains/n64/mips64-elf/mips64-elf/lib/libc.a(lib_a-freer.o)
                              /opt/toolchains/n64/mips64-elf/mips64-elf/lib/libc.a(lib_a-fclose.o) (_free_r)
/opt/toolchains/n64/mips64-elf/mips64-elf/lib/libc.a(lib_a-fseek.o)
                              /opt/toolchains/n64/mips64-elf/mips64-elf/lib/libc.a(lib_a-fopen.o) (_fseek_r)
/opt/toolchains/n64/mips64-elf/mips64-elf/lib/libc.a(lib_a-fstatr.o)
                              /opt/toolchains/n64/mips64-elf/mips64-elf/lib/libc.a(lib_a-fseek.o) (_fstat_r)
/opt/toolchains/n64/mips64-elf/mips64-elf/lib/libc.a(lib_a-ftell.o)
                              stb_image.o (ftell)
/opt/toolchains/n64/mips64-elf/mips64-elf/lib/libc.a(lib_a-fwalk.o)
                              /opt/toolchains/n64/mips64-elf/mips64-elf/lib/libc.a(lib_a-findfp.o) (_fwalk)
/opt/toolchains/n64/mips64-elf/mips64-elf/lib/libc.a(lib_a-fwrite.o)
                              ../y3d/y3d_record.o (fwrite)
/opt/toolchains/n64/mips64-elf/mips64-elf/lib/libc.a(lib_a-impure.o)
                              /opt/toolchains/n64/mips64-elf/mips64-elf/lib/libc.a(lib_a-fflush.o) (_global_impure_ptr)
/opt/toolchains/n64/mips64-elf/mips64-elf/lib/libc.a(lib_a-makebuf.o)
                              /opt/toolchains/n64/mips64-elf/mips64-elf/lib/libc.a(lib_a-fseek.o) (__smakebuf_r)
/opt/toolchains/n64/mips64-elf/mips64-elf/lib/libc.a(lib_a-malloc.o)
                              main.o (malloc)
/opt/toolchains/n64/mips64-elf/mips64-elf/lib/libc.a(lib_a-mallocr.o)
                              /opt/toolchains/n64/mips64-elf/mips64-elf/lib/libc.a(lib_a-findfp.o) (_malloc_r)
/opt/toolchains/n64/mips64-elf/mips64-elf/lib/libc.a(lib_a-memcpy.o)
                              stb_image.o (memcpy)
/opt/toolchains/n64/mips64-elf/mips64-elf/lib/libc.a(lib_a-memset.o)
                              main.o (memset)
/opt/toolchains/n64/mips64-elf/mips64-elf/lib/libc.a(lib_a-mlock.o)
                              /opt/toolchains/n64/mips64-elf/mips64-elf/lib/libc.a(lib_a-freer.o) (__malloc_lock)
/opt/toolchains/n64/mips64-elf/mips64-elf/lib/libc.a(lib_a-openr.o)
                              /opt/toolchains/n64/mips64-elf/mips64-elf/lib/libc.a(lib_a-fopen.o) (_open_r)
/opt/toolchains/n64/mips64-elf/mips64-elf/lib/libc.a(lib_a-realloc.o)
                              stb_image.o (realloc)
/opt/toolchains/n64/mips64-elf/mips64-elf/lib/libc.a(lib_a-reallocr.o)
                              /opt/toolchains/n64/mips64-elf/mips64-elf/lib/libc.a(lib_a-realloc.o) (_realloc_r)
/opt/toolchains/n64/mips64-elf/mips64-elf/lib/libc.a(lib_a-reent.o)
                              /opt/toolchains/n64/mips64-elf/mips64-elf/lib/libc.a(lib_a-fstatr.o) (errno)
/opt/toolchains/n64/mips64-elf/mips64-elf/lib/libc.a(lib_a-refill.o)
                              /opt/toolchains/n64/mips64-elf/mips64-elf/lib/libc.a(lib_a-fread.o) (__srefill_r)
/opt/toolchains/n64/mips64-elf/mips64-elf/lib/libc.a(lib_a-sbrkr.o)
                              /opt/toolchains/n64/mips64-elf/mips64-elf/lib/libc.a(lib_a-freer.o) (_sbrk_r)
/opt/toolchains/n64/mips64-elf/mips64-elf/lib/libc.a(lib_a-sprintf.o)
                              ../game/game.o (sprintf)
/opt/toolchains/n64/mips64-elf/mips64-elf/lib/libc.a(lib_a-stdio.o)
                              /opt/toolchains/n64/mips64-elf/mips64-elf/lib/libc.a(lib_a-findfp.o) (__sread)
/opt/toolchains/n64/mips64-elf/mips64-elf/lib/libc.a(lib_a-strcmp.o)
                              /opt/toolchains/n64/mips64-elf/lib/libdragon.a(dragonfs.o) (strcmp)
/opt/toolchains/n64/mips64-elf/mips64-elf/lib/libc.a(lib_a-strcpy.o)
                              /opt/toolchains/n64/mips64-elf/lib/libdragon.a(dragonfs.o) (strcpy)
/opt/toolchains/n64/mips64-elf/mips64-elf/lib/libc.a(lib_a-strlen.o)
                              ../y3d/y3d_engine.o (strlen)
/opt/toolchains/n64/mips64-elf/mips64-elf/lib/libc.a(lib_a-svfprintf.o)
                              /opt/toolchains/n64/mips64-elf/mips64-elf/lib/libc.a(lib_a-sprintf.o) (_svfprintf_r)
/opt/toolchains/n64/mips64-elf/mips64-elf/lib/libc.a(lib_a-vfiprintf.o)
                              /opt/toolchains/n64/mips64-elf/mips64-elf/lib/libc.a(lib_a-fiprintf.o) (_vfiprintf_r)
/opt/toolchains/n64/mips64-elf/mips64-elf/lib/libc.a(lib_a-writer.o)
                              /opt/toolchains/n64/mips64-elf/mips64-elf/lib/libc.a(lib_a-stdio.o) (_write_r)
/opt/toolchains/n64/mips64-elf/mips64-elf/lib/libc.a(lib_a-wsetup.o)
                              /opt/toolchains/n64/mips64-elf/mips64-elf/lib/libc.a(lib_a-vfiprintf.o) (__swsetup_r)
/opt/toolchains/n64/mips64-elf/mips64-elf/lib/libc.a(lib_a-abort.o)
                              /opt/toolchains/n64/mips64-elf/mips64-elf/lib/libc.a(lib_a-assert.o) (abort)
/opt/toolchains/n64/mips64-elf/mips64-elf/lib/libc.a(lib_a-closer.o)
                              /opt/toolchains/n64/mips64-elf/mips64-elf/lib/libc.a(lib_a-stdio.o) (_close_r)
/opt/toolchains/n64/mips64-elf/mips64-elf/lib/libc.a(lib_a-dtoa.o)
                              /opt/toolchains/n64/mips64-elf/mips64-elf/lib/libc.a(lib_a-svfprintf.o) (_dtoa_r)
/opt/toolchains/n64/mips64-elf/mips64-elf/lib/libc.a(lib_a-flags.o)
                              /opt/toolchains/n64/mips64-elf/mips64-elf/lib/libc.a(lib_a-fopen.o) (__sflags)
/opt/toolchains/n64/mips64-elf/mips64-elf/lib/libc.a(lib_a-fputwc.o)
                              /opt/toolchains/n64/mips64-elf/mips64-elf/lib/libc.a(lib_a-vfiprintf.o) (_fputwc_r)
/opt/toolchains/n64/mips64-elf/mips64-elf/lib/libc.a(lib_a-fvwrite.o)
                              /opt/toolchains/n64/mips64-elf/mips64-elf/lib/libc.a(lib_a-fwrite.o) (__sfvwrite_r)
/opt/toolchains/n64/mips64-elf/mips64-elf/lib/libc.a(lib_a-isattyr.o)
                              /opt/toolchains/n64/mips64-elf/mips64-elf/lib/libc.a(lib_a-makebuf.o) (_isatty_r)
/opt/toolchains/n64/mips64-elf/mips64-elf/lib/libc.a(lib_a-locale.o)
                              /opt/toolchains/n64/mips64-elf/mips64-elf/lib/libc.a(lib_a-fputwc.o) (__locale_mb_cur_max)
/opt/toolchains/n64/mips64-elf/mips64-elf/lib/libc.a(lib_a-lseekr.o)
                              /opt/toolchains/n64/mips64-elf/mips64-elf/lib/libc.a(lib_a-stdio.o) (_lseek_r)
/opt/toolchains/n64/mips64-elf/mips64-elf/lib/libc.a(lib_a-memchr.o)
                              /opt/toolchains/n64/mips64-elf/mips64-elf/lib/libc.a(lib_a-svfprintf.o) (memchr)
/opt/toolchains/n64/mips64-elf/mips64-elf/lib/libc.a(lib_a-memmove.o)
                              /opt/toolchains/n64/mips64-elf/mips64-elf/lib/libc.a(lib_a-reallocr.o) (memmove)
/opt/toolchains/n64/mips64-elf/mips64-elf/lib/libc.a(lib_a-mprec.o)
                              /opt/toolchains/n64/mips64-elf/mips64-elf/lib/libc.a(lib_a-dtoa.o) (_Balloc)
/opt/toolchains/n64/mips64-elf/mips64-elf/lib/libc.a(lib_a-readr.o)
                              /opt/toolchains/n64/mips64-elf/mips64-elf/lib/libc.a(lib_a-stdio.o) (_read_r)
/opt/toolchains/n64/mips64-elf/mips64-elf/lib/libc.a(lib_a-signal.o)
                              /opt/toolchains/n64/mips64-elf/mips64-elf/lib/libc.a(lib_a-abort.o) (raise)
/opt/toolchains/n64/mips64-elf/mips64-elf/lib/libc.a(lib_a-signalr.o)
                              /opt/toolchains/n64/mips64-elf/mips64-elf/lib/libc.a(lib_a-signal.o) (_kill_r)
/opt/toolchains/n64/mips64-elf/mips64-elf/lib/libc.a(lib_a-svfiprintf.o)
                              /opt/toolchains/n64/mips64-elf/mips64-elf/lib/libc.a(lib_a-svfprintf.o) (__ssprint_r)
/opt/toolchains/n64/mips64-elf/mips64-elf/lib/libc.a(lib_a-wbuf.o)
                              /opt/toolchains/n64/mips64-elf/mips64-elf/lib/libc.a(lib_a-fputwc.o) (__swbuf_r)
/opt/toolchains/n64/mips64-elf/mips64-elf/lib/libc.a(lib_a-wcrtomb.o)
                              /opt/toolchains/n64/mips64-elf/mips64-elf/lib/libc.a(lib_a-fputwc.o) (_wcrtomb_r)
/opt/toolchains/n64/mips64-elf/mips64-elf/lib/libc.a(lib_a-wctomb_r.o)
                              /opt/toolchains/n64/mips64-elf/mips64-elf/lib/libc.a(lib_a-wcrtomb.o) (__wctomb)
/opt/toolchains/n64/mips64-elf/mips64-elf/lib/libc.a(lib_a-callocr.o)
                              /opt/toolchains/n64/mips64-elf/mips64-elf/lib/libc.a(lib_a-mprec.o) (_calloc_r)
/opt/toolchains/n64/mips64-elf/lib/libdragonsys.a(system.o)
                              /opt/toolchains/n64/mips64-elf/lib/libdragon.a(dragonfs.o) (attach_filesystem)
/opt/toolchains/n64/mips64-elf/mips64-elf/lib/libnosys.a(_exit.o)
                              /opt/toolchains/n64/mips64-elf/mips64-elf/lib/libc.a(lib_a-abort.o) (_exit)

Allocating common symbols
Common symbol       size              file

__width             0x4               /opt/toolchains/n64/mips64-elf/lib/libdragon.a(display.o)
__bitdepth          0x4               /opt/toolchains/n64/mips64-elf/lib/libdragon.a(display.o)
gTicks              0x4               main.o
errno               0x4               /opt/toolchains/n64/mips64-elf/mips64-elf/lib/libc.a(lib_a-reent.o)
yeti                0x749fc           main.o
stbi_png_partial    0x4               stb_image.o
tv_fps              0x4               main.o
gCursorY            0x2               main.o
__height            0x4               /opt/toolchains/n64/mips64-elf/lib/libdragon.a(display.o)
buf_size            0x4               main.o
lastticks           0x8               main.o
gKeys               0xa0              main.o
gCursorX            0x2               main.o
buf_ptr             0x4               main.o
frameticks          0x4               main.o
sintable            0x2000            ../y3d/y3d_fixed.o
reciprocal          0x10000           ../y3d/y3d_fixed.o
__safe_buffer       0xc               /opt/toolchains/n64/mips64-elf/lib/libdragon.a(display.o)
yetiMap             0x10080           main.o

Discarded input sections

 .reginfo       0x0000000000000000       0x18 stb_image.o
 .reginfo       0x0000000000000000       0x18 ../game/ai/boost.o
 .reginfo       0x0000000000000000       0x18 ../game/ai/bullet.o
 .reginfo       0x0000000000000000       0x18 ../game/ai/death.o
 .reginfo       0x0000000000000000       0x18 ../game/ai/explode.o
 .reginfo       0x0000000000000000       0x18 ../game/ai/pickup.o
 .reginfo       0x0000000000000000       0x18 ../game/ai/quad.o
 .reginfo       0x0000000000000000       0x18 ../game/ai/sheba.o
 .reginfo       0x0000000000000000       0x18 ../game/ai/static_model.o
 .reginfo       0x0000000000000000       0x18 ../game/ai/static_sprite.o
 .reginfo       0x0000000000000000       0x18 ../game/ai/teleporter.o
 .reginfo       0x0000000000000000       0x18 ../game/ai/torch.o
 .reginfo       0x0000000000000000       0x18 ../game/data.o
 .reginfo       0x0000000000000000       0x18 ../game/entities.o
 .reginfo       0x0000000000000000       0x18 ../game/game.o
 .reginfo       0x0000000000000000       0x18 ../game/maps.o
 .reginfo       0x0000000000000000       0x18 ../game/models.o
 .reginfo       0x0000000000000000       0x18 ../game/screens.o
 .reginfo       0x0000000000000000       0x18 ../game/sprites.o
 .reginfo       0x0000000000000000       0x18 ../y3d/y3d_animation.o
 .reginfo       0x0000000000000000       0x18 ../y3d/y3d_ansic.o
 .reginfo       0x0000000000000000       0x18 ../y3d/y3d_cell.o
 .reginfo       0x0000000000000000       0x18 ../y3d/y3d_draw.o
 .reginfo       0x0000000000000000       0x18 ../y3d/y3d_engine.o
 .reginfo       0x0000000000000000       0x18 ../y3d/y3d_entity.o
 .reginfo       0x0000000000000000       0x18 ../y3d/y3d_file.o
 .reginfo       0x0000000000000000       0x18 ../y3d/y3d_fixed.o
 .reginfo       0x0000000000000000       0x18 ../y3d/y3d_fruity.o
 .reginfo       0x0000000000000000       0x18 ../y3d/y3d_image.o
 .reginfo       0x0000000000000000       0x18 ../y3d/y3d_keyboard.o
 .reginfo       0x0000000000000000       0x18 ../y3d/y3d_map.o
 .reginfo       0x0000000000000000       0x18 ../y3d/y3d_matrix.o
 .reginfo       0x0000000000000000       0x18 ../y3d/y3d_pixel.o
 .reginfo       0x0000000000000000       0x18 ../y3d/y3d_record.o
 .reginfo       0x0000000000000000       0x18 ../y3d/y3d_sound.o
 .reginfo       0x0000000000000000       0x18 ../y3d/y3d_spanner.o
 .reginfo       0x0000000000000000       0x18 ../y3d/y3d_surface.o
 .reginfo       0x0000000000000000       0x18 ../y3d/y3d_vertex.o
 .reginfo       0x0000000000000000       0x18 ../y3d/y3d_yeti.o
 .reginfo       0x0000000000000000       0x18 /opt/toolchains/n64/mips64-elf/mips64-elf/lib/libm.a(lib_a-s_sin.o)
 .reginfo       0x0000000000000000       0x18 /opt/toolchains/n64/mips64-elf/mips64-elf/lib/libm.a(lib_a-w_pow.o)
 .reginfo       0x0000000000000000       0x18 /opt/toolchains/n64/mips64-elf/mips64-elf/lib/libm.a(lib_a-e_pow.o)
 .reginfo       0x0000000000000000       0x18 /opt/toolchains/n64/mips64-elf/mips64-elf/lib/libm.a(lib_a-e_rem_pio2.o)
 .reginfo       0x0000000000000000       0x18 /opt/toolchains/n64/mips64-elf/mips64-elf/lib/libm.a(lib_a-e_sqrt.o)
 .reginfo       0x0000000000000000       0x18 /opt/toolchains/n64/mips64-elf/mips64-elf/lib/libm.a(lib_a-k_cos.o)
 .reginfo       0x0000000000000000       0x18 /opt/toolchains/n64/mips64-elf/mips64-elf/lib/libm.a(lib_a-k_rem_pio2.o)
 .reginfo       0x0000000000000000       0x18 /opt/toolchains/n64/mips64-elf/mips64-elf/lib/libm.a(lib_a-k_sin.o)
 .reginfo       0x0000000000000000       0x18 /opt/toolchains/n64/mips64-elf/mips64-elf/lib/libm.a(lib_a-s_fabs.o)
 .reginfo       0x0000000000000000       0x18 /opt/toolchains/n64/mips64-elf/mips64-elf/lib/libm.a(lib_a-s_finite.o)
 .reginfo       0x0000000000000000       0x18 /opt/toolchains/n64/mips64-elf/mips64-elf/lib/libm.a(lib_a-s_floor.o)
 .reginfo       0x0000000000000000       0x18 /opt/toolchains/n64/mips64-elf/mips64-elf/lib/libm.a(lib_a-s_fpclassify.o)
 .reginfo       0x0000000000000000       0x18 /opt/toolchains/n64/mips64-elf/mips64-elf/lib/libm.a(lib_a-s_lib_ver.o)
 .reginfo       0x0000000000000000       0x18 /opt/toolchains/n64/mips64-elf/mips64-elf/lib/libm.a(lib_a-s_matherr.o)
 .reginfo       0x0000000000000000       0x18 /opt/toolchains/n64/mips64-elf/mips64-elf/lib/libm.a(lib_a-s_nan.o)
 .reginfo       0x0000000000000000       0x18 /opt/toolchains/n64/mips64-elf/mips64-elf/lib/libm.a(lib_a-s_rint.o)
 .reginfo       0x0000000000000000       0x18 /opt/toolchains/n64/mips64-elf/mips64-elf/lib/libm.a(lib_a-s_scalbn.o)
 .reginfo       0x0000000000000000       0x18 /opt/toolchains/n64/mips64-elf/mips64-elf/lib/libm.a(lib_a-s_copysign.o)
 .reginfo       0x0000000000000000       0x18 /opt/toolchains/n64/mips64-elf/lib/libdragon.a(n64sys.o)
 .reginfo       0x0000000000000000       0x18 /opt/toolchains/n64/mips64-elf/lib/libdragon.a(interrupt.o)
 .reginfo       0x0000000000000000       0x18 /opt/toolchains/n64/mips64-elf/lib/libdragon.a(entrypoint.o)
 .reginfo       0x0000000000000000       0x18 /opt/toolchains/n64/mips64-elf/lib/libdragon.a(dragonfs.o)
 .reginfo       0x0000000000000000       0x18 /opt/toolchains/n64/mips64-elf/lib/libdragon.a(audio.o)
 .reginfo       0x0000000000000000       0x18 /opt/toolchains/n64/mips64-elf/lib/libdragon.a(display.o)
 .reginfo       0x0000000000000000       0x18 /opt/toolchains/n64/mips64-elf/lib/libdragon.a(controller.o)
 .reginfo       0x0000000000000000       0x18 /opt/toolchains/n64/mips64-elf/lib/libdragon.a(graphics.o)
 .reginfo       0x0000000000000000       0x18 /opt/toolchains/n64/mips64-elf/lib/libdragon.a(rdp.o)
 .reginfo       0x0000000000000000       0x18 /opt/toolchains/n64/mips64-elf/lib/libdragon.a(dma.o)
 .reginfo       0x0000000000000000       0x18 /opt/toolchains/n64/mips64-elf/lib/libdragon.a(timer.o)
 .reginfo       0x0000000000000000       0x18 /opt/toolchains/n64/mips64-elf/lib/libdragon.a(inthandler.o)
 .reginfo       0x0000000000000000       0x18 /opt/toolchains/n64/mips64-elf/lib/libdragon.a(exception.o)
 .reginfo       0x0000000000000000       0x18 /opt/toolchains/n64/mips64-elf/mips64-elf/lib/libc.a(lib_a-assert.o)
 .reginfo       0x0000000000000000       0x18 /opt/toolchains/n64/mips64-elf/mips64-elf/lib/libc.a(lib_a-errno.o)
 .reginfo       0x0000000000000000       0x18 /opt/toolchains/n64/mips64-elf/mips64-elf/lib/libc.a(lib_a-fclose.o)
 .reginfo       0x0000000000000000       0x18 /opt/toolchains/n64/mips64-elf/mips64-elf/lib/libc.a(lib_a-fflush.o)
 .reginfo       0x0000000000000000       0x18 /opt/toolchains/n64/mips64-elf/mips64-elf/lib/libc.a(lib_a-findfp.o)
 .reginfo       0x0000000000000000       0x18 /opt/toolchains/n64/mips64-elf/mips64-elf/lib/libc.a(lib_a-fiprintf.o)
 .reginfo       0x0000000000000000       0x18 /opt/toolchains/n64/mips64-elf/mips64-elf/lib/libc.a(lib_a-fopen.o)
 .reginfo       0x0000000000000000       0x18 /opt/toolchains/n64/mips64-elf/mips64-elf/lib/libc.a(lib_a-fread.o)
 .reginfo       0x0000000000000000       0x18 /opt/toolchains/n64/mips64-elf/mips64-elf/lib/libc.a(lib_a-freer.o)
 .reginfo       0x0000000000000000       0x18 /opt/toolchains/n64/mips64-elf/mips64-elf/lib/libc.a(lib_a-fseek.o)
 .reginfo       0x0000000000000000       0x18 /opt/toolchains/n64/mips64-elf/mips64-elf/lib/libc.a(lib_a-fstatr.o)
 .reginfo       0x0000000000000000       0x18 /opt/toolchains/n64/mips64-elf/mips64-elf/lib/libc.a(lib_a-ftell.o)
 .reginfo       0x0000000000000000       0x18 /opt/toolchains/n64/mips64-elf/mips64-elf/lib/libc.a(lib_a-fwalk.o)
 .reginfo       0x0000000000000000       0x18 /opt/toolchains/n64/mips64-elf/mips64-elf/lib/libc.a(lib_a-fwrite.o)
 .reginfo       0x0000000000000000       0x18 /opt/toolchains/n64/mips64-elf/mips64-elf/lib/libc.a(lib_a-impure.o)
 .reginfo       0x0000000000000000       0x18 /opt/toolchains/n64/mips64-elf/mips64-elf/lib/libc.a(lib_a-makebuf.o)
 .reginfo       0x0000000000000000       0x18 /opt/toolchains/n64/mips64-elf/mips64-elf/lib/libc.a(lib_a-malloc.o)
 .reginfo       0x0000000000000000       0x18 /opt/toolchains/n64/mips64-elf/mips64-elf/lib/libc.a(lib_a-mallocr.o)
 .reginfo       0x0000000000000000       0x18 /opt/toolchains/n64/mips64-elf/mips64-elf/lib/libc.a(lib_a-memcpy.o)
 .reginfo       0x0000000000000000       0x18 /opt/toolchains/n64/mips64-elf/mips64-elf/lib/libc.a(lib_a-memset.o)
 .reginfo       0x0000000000000000       0x18 /opt/toolchains/n64/mips64-elf/mips64-elf/lib/libc.a(lib_a-mlock.o)
 .reginfo       0x0000000000000000       0x18 /opt/toolchains/n64/mips64-elf/mips64-elf/lib/libc.a(lib_a-openr.o)
 .reginfo       0x0000000000000000       0x18 /opt/toolchains/n64/mips64-elf/mips64-elf/lib/libc.a(lib_a-realloc.o)
 .reginfo       0x0000000000000000       0x18 /opt/toolchains/n64/mips64-elf/mips64-elf/lib/libc.a(lib_a-reallocr.o)
 .reginfo       0x0000000000000000       0x18 /opt/toolchains/n64/mips64-elf/mips64-elf/lib/libc.a(lib_a-reent.o)
 .reginfo       0x0000000000000000       0x18 /opt/toolchains/n64/mips64-elf/mips64-elf/lib/libc.a(lib_a-refill.o)
 .reginfo       0x0000000000000000       0x18 /opt/toolchains/n64/mips64-elf/mips64-elf/lib/libc.a(lib_a-sbrkr.o)
 .reginfo       0x0000000000000000       0x18 /opt/toolchains/n64/mips64-elf/mips64-elf/lib/libc.a(lib_a-sprintf.o)
 .reginfo       0x0000000000000000       0x18 /opt/toolchains/n64/mips64-elf/mips64-elf/lib/libc.a(lib_a-stdio.o)
 .reginfo       0x0000000000000000       0x18 /opt/toolchains/n64/mips64-elf/mips64-elf/lib/libc.a(lib_a-strcmp.o)
 .reginfo       0x0000000000000000       0x18 /opt/toolchains/n64/mips64-elf/mips64-elf/lib/libc.a(lib_a-strcpy.o)
 .reginfo       0x0000000000000000       0x18 /opt/toolchains/n64/mips64-elf/mips64-elf/lib/libc.a(lib_a-strlen.o)
 .reginfo       0x0000000000000000       0x18 /opt/toolchains/n64/mips64-elf/mips64-elf/lib/libc.a(lib_a-svfprintf.o)
 .reginfo       0x0000000000000000       0x18 /opt/toolchains/n64/mips64-elf/mips64-elf/lib/libc.a(lib_a-vfiprintf.o)
 .reginfo       0x0000000000000000       0x18 /opt/toolchains/n64/mips64-elf/mips64-elf/lib/libc.a(lib_a-writer.o)
 .reginfo       0x0000000000000000       0x18 /opt/toolchains/n64/mips64-elf/mips64-elf/lib/libc.a(lib_a-wsetup.o)
 .reginfo       0x0000000000000000       0x18 /opt/toolchains/n64/mips64-elf/mips64-elf/lib/libc.a(lib_a-abort.o)
 .reginfo       0x0000000000000000       0x18 /opt/toolchains/n64/mips64-elf/mips64-elf/lib/libc.a(lib_a-closer.o)
 .reginfo       0x0000000000000000       0x18 /opt/toolchains/n64/mips64-elf/mips64-elf/lib/libc.a(lib_a-dtoa.o)
 .reginfo       0x0000000000000000       0x18 /opt/toolchains/n64/mips64-elf/mips64-elf/lib/libc.a(lib_a-flags.o)
 .reginfo       0x0000000000000000       0x18 /opt/toolchains/n64/mips64-elf/mips64-elf/lib/libc.a(lib_a-fputwc.o)
 .reginfo       0x0000000000000000       0x18 /opt/toolchains/n64/mips64-elf/mips64-elf/lib/libc.a(lib_a-fvwrite.o)
 .reginfo       0x0000000000000000       0x18 /opt/toolchains/n64/mips64-elf/mips64-elf/lib/libc.a(lib_a-isattyr.o)
 .reginfo       0x0000000000000000       0x18 /opt/toolchains/n64/mips64-elf/mips64-elf/lib/libc.a(lib_a-locale.o)
 .reginfo       0x0000000000000000       0x18 /opt/toolchains/n64/mips64-elf/mips64-elf/lib/libc.a(lib_a-lseekr.o)
 .reginfo       0x0000000000000000       0x18 /opt/toolchains/n64/mips64-elf/mips64-elf/lib/libc.a(lib_a-memchr.o)
 .reginfo       0x0000000000000000       0x18 /opt/toolchains/n64/mips64-elf/mips64-elf/lib/libc.a(lib_a-memmove.o)
 .reginfo       0x0000000000000000       0x18 /opt/toolchains/n64/mips64-elf/mips64-elf/lib/libc.a(lib_a-mprec.o)
 .reginfo       0x0000000000000000       0x18 /opt/toolchains/n64/mips64-elf/mips64-elf/lib/libc.a(lib_a-readr.o)
 .reginfo       0x0000000000000000       0x18 /opt/toolchains/n64/mips64-elf/mips64-elf/lib/libc.a(lib_a-signal.o)
 .reginfo       0x0000000000000000       0x18 /opt/toolchains/n64/mips64-elf/mips64-elf/lib/libc.a(lib_a-signalr.o)
 .reginfo       0x0000000000000000       0x18 /opt/toolchains/n64/mips64-elf/mips64-elf/lib/libc.a(lib_a-svfiprintf.o)
 .reginfo       0x0000000000000000       0x18 /opt/toolchains/n64/mips64-elf/mips64-elf/lib/libc.a(lib_a-wbuf.o)
 .reginfo       0x0000000000000000       0x18 /opt/toolchains/n64/mips64-elf/mips64-elf/lib/libc.a(lib_a-wcrtomb.o)
 .reginfo       0x0000000000000000       0x18 /opt/toolchains/n64/mips64-elf/mips64-elf/lib/libc.a(lib_a-wctomb_r.o)
 .reginfo       0x0000000000000000       0x18 /opt/toolchains/n64/mips64-elf/mips64-elf/lib/libc.a(lib_a-callocr.o)
 .reginfo       0x0000000000000000       0x18 /opt/toolchains/n64/mips64-elf/lib/libdragonsys.a(system.o)
 .reginfo       0x0000000000000000       0x18 /opt/toolchains/n64/mips64-elf/mips64-elf/lib/libnosys.a(_exit.o)

Memory Configuration

Name             Origin             Length             Attributes
ram              0x0000000080000400 0x00000000007ffc00 xw
*default*        0x0000000000000000 0xffffffffffffffff

Linker script and memory map

LOAD main.o
LOAD stb_image.o
LOAD ../game/ai/boost.o
LOAD ../game/ai/bullet.o
LOAD ../game/ai/death.o
LOAD ../game/ai/explode.o
LOAD ../game/ai/pickup.o
LOAD ../game/ai/quad.o
LOAD ../game/ai/sheba.o
LOAD ../game/ai/static_model.o
LOAD ../game/ai/static_sprite.o
LOAD ../game/ai/teleporter.o
LOAD ../game/ai/torch.o
LOAD ../game/data.o
LOAD ../game/entities.o
LOAD ../game/game.o
LOAD ../game/maps.o
LOAD ../game/models.o
LOAD ../game/screens.o
LOAD ../game/sprites.o
LOAD ../y3d/y3d_animation.o
LOAD ../y3d/y3d_ansic.o
LOAD ../y3d/y3d_cell.o
LOAD ../y3d/y3d_draw.o
LOAD ../y3d/y3d_engine.o
LOAD ../y3d/y3d_entity.o
LOAD ../y3d/y3d_file.o
LOAD ../y3d/y3d_fixed.o
LOAD ../y3d/y3d_fruity.o
LOAD ../y3d/y3d_image.o
LOAD ../y3d/y3d_keyboard.o
LOAD ../y3d/y3d_map.o
LOAD ../y3d/y3d_matrix.o
LOAD ../y3d/y3d_pixel.o
LOAD ../y3d/y3d_record.o
LOAD ../y3d/y3d_sound.o
LOAD ../y3d/y3d_spanner.o
LOAD ../y3d/y3d_surface.o
LOAD ../y3d/y3d_vertex.o
LOAD ../y3d/y3d_yeti.o
                0x0000000000000000                __DYNAMIC = 0x0
                0x0000000080800000                PROVIDE (__stack, 0x80800000)

.text           0x0000000080000400    0x42ce8 load address 0x0000000000000000
 *(.boot)
 .boot          0x0000000080000400      0x154 /opt/toolchains/n64/mips64-elf/lib/libdragon.a(entrypoint.o)
                0x0000000080000400                _start
                0x0000000080000560                . = ALIGN (0x10)
 *fill*         0x0000000080000554        0xc 00
                0x0000000080000560                __text_start = .
 *(.text)
 .text          0x0000000080000560     0x1290 main.o
                0x0000000080000560                vblCallback
                0x0000000080000578                getButtons
                0x00000000800005d0                getAnalogX
                0x00000000800005e8                getAnalogY
                0x0000000080000600                drawText
                0x0000000080000620                printText
                0x00000000800006c8                delay
                0x00000000800006f0                debugText
                0x00000000800008a0                splash
                0x0000000080000ed8                init_n64
                0x0000000080001050                Yeti_Cleanup
                0x0000000080001088                Yeti_LoadMap
                0x00000000800012f8                Yeti_Frame
                0x00000000800013d8                fix_sprites
                0x0000000080001488                fix_model
                0x00000000800015d8                fix_models
                0x0000000080001750                Yeti_Go_Episode
                0x00000000800017d8                sound_play
                0x00000000800017e0                sound_loop
                0x00000000800017e8                sound_stop
 .text          0x00000000800017f0    0x136d0 stb_image.o
                0x00000000800144d0                stbi_failure_reason
                0x00000000800144e0                stbi_image_free
                0x00000000800144e8                stbi_load
                0x0000000080014600                stbi_load_from_file
                0x00000000800146e8                stbi_load_from_memory
                0x0000000080014738                stbi_load_from_callbacks
                0x0000000080014818                stbi_is_hdr_from_memory
                0x0000000080014820                stbi_is_hdr
                0x0000000080014858                stbi_is_hdr_from_file
                0x0000000080014860                stbi_is_hdr_from_callbacks
                0x0000000080014868                stbi_zlib_decode_malloc_guesssize
                0x0000000080014920                stbi_zlib_decode_malloc
                0x0000000080014928                stbi_zlib_decode_malloc_guesssize_headerflag
                0x00000000800149e0                stbi_zlib_decode_buffer
                0x0000000080014a40                stbi_zlib_decode_noheader_malloc
                0x0000000080014af0                stbi_zlib_decode_noheader_buffer
                0x0000000080014b50                stbi_set_unpremultiply_on_load
                0x0000000080014b60                stbi_convert_iphone_png_to_rgb
                0x0000000080014b70                stbi_info_from_file
                0x0000000080014ca0                stbi_info
                0x0000000080014d38                stbi_info_from_memory
                0x0000000080014dc8                stbi_info_from_callbacks
 .text          0x0000000080014ec0       0xb0 ../game/ai/boost.o
                0x0000000080014ec0                boost_tick
                0x0000000080014ec8                boost_hit
                0x0000000080014f28                boost_init
 .text          0x0000000080014f70      0x180 ../game/ai/bullet.o
                0x0000000080014f70                bullet_hit
                0x0000000080014f78                bullet_wall
                0x0000000080014f80                bullet_tick
                0x0000000080014fa8                bullet_shoot_at
                0x0000000080014fd0                bullet_shoot
 .text          0x00000000800150f0       0xd0 ../game/ai/death.o
                0x00000000800150f0                death_tick
                0x0000000080015128                death_init
 .text          0x00000000800151c0      0x2f0 ../game/ai/explode.o
                0x00000000800151c0                splat_tick
                0x0000000080015280                explode_tick
                0x0000000080015358                explode_init
                0x0000000080015420                splat_init
 .text          0x00000000800154b0       0x90 ../game/ai/pickup.o
                0x00000000800154b0                pickup_tick
 .text          0x0000000080015540       0xb0 ../game/ai/quad.o
                0x0000000080015540                quad_tick
                0x0000000080015548                quad_hit
                0x00000000800155a8                quad_init
 .text          0x00000000800155f0       0x90 ../game/ai/sheba.o
                0x00000000800155f0                sheba_tick
                0x0000000080015630                sheba_init
 .text          0x0000000080015680        0x0 ../game/ai/static_model.o
 .text          0x0000000080015680        0x0 ../game/ai/static_sprite.o
 .text          0x0000000080015680       0x58 ../game/ai/teleporter.o
                0x0000000080015680                teleporter_tick
                0x0000000080015688                teleporter_init
 .text          0x00000000800156d8      0x1c0 ../game/ai/torch.o
                0x00000000800156d8                torch0_tick
                0x0000000080015718                torch1_tick
                0x0000000080015758                torch0_init
                0x00000000800157f8                torch1_init
 .text          0x0000000080015898        0x0 ../game/data.o
 .text          0x0000000080015898      0x768 ../game/entities.o
                0x0000000080015898                static_model_init
                0x0000000080015938                static_sprite_init
                0x00000000800159f8                barrontree_init
                0x0000000080015a88                leafyplant_init
                0x0000000080015b18                cactus_init
                0x0000000080015ba8                potplant_init
                0x0000000080015c40                pillar_init
                0x0000000080015cd0                overpass_init
                0x0000000080015d80                bridge_init
                0x0000000080015e30                emptypot_init
                0x0000000080015ec8                pinechair_init
                0x0000000080015f60                crate_init
 .text          0x0000000080016000     0x23a0 ../game/game.o
                0x0000000080016000                light_tick
                0x0000000080016068                hud_init
                0x00000000800160a0                camera_exit_tick
                0x0000000080016368                guard_attack_tick
                0x00000000800163c8                guard_stand_tick
                0x00000000800164d8                guard_attack_hit
                0x00000000800165b8                guard_pain_tick
                0x0000000080016670                player_tick
                0x0000000080016bb8                entity_default
                0x0000000080016e50                camera_exit_init
                0x0000000080016e60                player_init
                0x0000000080016eb0                guard_base_init
                0x0000000080016ec8                guard_pain_init
                0x0000000080016f28                guard_attack_init
                0x0000000080016f68                entity_line_of_sight
                0x0000000080016fa0                guard_stand_init
                0x0000000080016fe0                guard_init
                0x0000000080017020                bauul_init
                0x0000000080017070                ogro_init
                0x00000000800170c0                rat_init
                0x0000000080017110                light_init
                0x0000000080017198                game_spawn_entities
                0x0000000080017740                game_load_map
                0x0000000080017838                game_mode
                0x0000000080017840                game_goto
                0x0000000080017858                game_goback
                0x0000000080017878                game_cycle
                0x0000000080017898                game_menu
                0x0000000080017940                game_init
                0x0000000080017950                game_draw
                0x00000000800179f0                game_tick
                0x0000000080018378                game_loop
 .text          0x00000000800183a0        0x0 ../game/maps.o
 .text          0x00000000800183a0        0x0 ../game/models.o
 .text          0x00000000800183a0     0x19a8 ../game/screens.o
                0x00000000800183a0                draw_menu_item
                0x0000000080018480                screen_monster
                0x0000000080018580                screen_flames
                0x0000000080018690                screen_yeti3d
                0x0000000080018730                screen_publisher
                0x00000000800187c8                screen_title
                0x0000000080018888                screen_menu
                0x0000000080018bc0                screen_episode
                0x0000000080018df0                screen_skill
                0x0000000080019020                screen_credits
                0x00000000800191c8                draw_option
                0x0000000080019338                screen_view_options
                0x0000000080019850                screen_load_game
                0x00000000800198d8                screen_quit_game
                0x0000000080019960                screen_play
                0x0000000080019a18                screen_paused
                0x0000000080019d40                screen_end_level
 .text          0x0000000080019d48        0x0 ../game/sprites.o
 .text          0x0000000080019d48      0x220 ../y3d/y3d_animation.o
                0x0000000080019d48                animation_init
                0x0000000080019d88                animation_tick
                0x0000000080019e40                animation_mode
                0x0000000080019ec8                animation_get_frames
                0x0000000080019f20                keyframe_init
 .text          0x0000000080019f68      0x300 ../y3d/y3d_ansic.o
                0x0000000080019f68                ansic_stpcpy
                0x0000000080019f88                ansic_itos
                0x0000000080019ff8                ansic_friction
                0x000000008001a028                isqrt
 .text          0x000000008001a268      0x120 ../y3d/y3d_cell.o
                0x000000008001a268                cell_init
                0x000000008001a2f0                cells_are_equal
 .text          0x000000008001a388     0x9ed0 ../y3d/y3d_draw.o
                0x000000008001a388                fill_rect
                0x000000008001a4b8                draw_line_nc
                0x000000008001a568                draw_poly_line_nc
                0x000000008001a6f0                draw_char
                0x000000008001a770                draw_string
                0x000000008001a868                tmap_16_cs
                0x000000008001b5a8                tmap_16
                0x000000008001d3d0                draw_poly_flat
                0x000000008001d720                tmap_16_sky
                0x000000008001dad0                texcoord_fixup
                0x000000008001db80                tmap_8_horz_pc
                0x00000000800228a0                tmap_8_horz
 .text          0x0000000080024258     0x3238 ../y3d/y3d_engine.o
                0x0000000080024258                yeti_sprite_draw
                0x00000000800242e8                yeti_model_draw
                0x0000000080024d30                yeti_quad_draw
                0x0000000080025888                yeti_quad
                0x0000000080025b30                yeti_build_vis
                0x0000000080025d48                yeti_draw
                0x0000000080026828                cell_bot
                0x00000000800268b8                cell_top
                0x0000000080026958                yeti_tick
 .text          0x0000000080027490      0x5b0 ../y3d/y3d_entity.o
                0x0000000080027490                entity_visual_init
                0x00000000800274c8                entity_destroy
                0x00000000800274d8                entity_init
                0x0000000080027548                entity_reinit
                0x00000000800275c0                entity_freeze
                0x00000000800275e0                entity_friction
                0x0000000080027628                entity_move_forward
                0x0000000080027680                entity_move_backwards
                0x00000000800276d8                entity_move_right
                0x0000000080027738                entity_move_left
                0x0000000080027790                entity_turn_right
                0x00000000800277a0                entity_turn_left
                0x00000000800277b0                entity_turn_towards
                0x0000000080027890                entity_look_at
                0x0000000080027920                entity_look_at2
                0x00000000800279b0                entity_set_velocity
                0x0000000080027a08                entity_force_towards
 .text          0x0000000080027a40       0xb0 ../y3d/y3d_file.o
                0x0000000080027a40                file_load
 .text          0x0000000080027af0      0x110 ../y3d/y3d_fixed.o
                0x0000000080027af0                lupin_arctan2
                0x0000000080027b70                fixangle
 .text          0x0000000080027c00      0xb00 ../y3d/y3d_fruity.o
                0x0000000080027c00                fruity_poly
                0x0000000080028188                fruity_draw
 .text          0x0000000080028700     0x11f0 ../y3d/y3d_image.o
                0x0000000080028700                image_draw
                0x0000000080029780                image_draw_at
                0x00000000800297d8                image_draw_di
 .text          0x00000000800298f0       0x38 ../y3d/y3d_keyboard.o
                0x00000000800298f0                keyboard_init
                0x0000000080029900                keyboard_tick
 .text          0x0000000080029928     0x1c40 ../y3d/y3d_map.o
                0x0000000080029928                map_ungroup
                0x0000000080029998                map_group
                0x0000000080029ac0                map_cells_are_equal
                0x0000000080029bb0                map_cells_are_group
                0x0000000080029e78                map_init_lod
                0x000000008002a148                map_draw_light
                0x000000008002a2a0                map_ambient_lit
                0x000000008002a310                map_smooth_lit
                0x000000008002a4d8                map_smooth_slopes
                0x000000008002a790                map_calc_lights
                0x000000008002ac38                map_init_slopes
                0x000000008002b0a8                map_init
                0x000000008002b330                map_precalc_data
                0x000000008002b368                map_find_ent
                0x000000008002b400                map_line_of_sight
 .text          0x000000008002b568      0x640 ../y3d/y3d_matrix.o
                0x000000008002b568                matrix_rotate_world
                0x000000008002b6d8                matrix_rotate_object
                0x000000008002b858                matrix_multiply
 .text          0x000000008002bba8      0x858 ../y3d/y3d_pixel.o
                0x000000008002bba8                pixel_converter_init
                0x000000008002bec0                pixel555_convert
                0x000000008002bf70                pixel555_convert_array
                0x000000008002c048                pixel_convert
                0x000000008002c0f8                pixel_convert_array
                0x000000008002c1f8                pixel_convert_image
                0x000000008002c310                pixel_buffer_draw
                0x000000008002c3f0                pixel_buffer_clear
 .text          0x000000008002c400      0x1a0 ../y3d/y3d_record.o
                0x000000008002c400                record_write
                0x000000008002c428                record_read
                0x000000008002c450                record_start
                0x000000008002c488                record_rewind
                0x000000008002c4a8                record_play
                0x000000008002c4e8                record_play_or_record
                0x000000008002c568                record_stop
 .text          0x000000008002c5a0        0x0 ../y3d/y3d_sound.o
 .text          0x000000008002c5a0      0x248 ../y3d/y3d_spanner.o
                0x000000008002c5a0                spanarray_init
                0x000000008002c5b8                spanarray_validate
                0x000000008002c6b8                spanner_invalidate
                0x000000008002c710                spanner_validate
 .text          0x000000008002c7e8     0x1028 ../y3d/y3d_surface.o
                0x000000008002c7e8                surface_init
                0x000000008002c818                surface_array_init
 .text          0x000000008002d810      0x268 ../y3d/y3d_vertex.o
                0x000000008002d810                polycliper
 .text          0x000000008002da78      0xd10 ../y3d/y3d_yeti.o
                0x000000008002da78                palette_overbright
                0x000000008002db58                yeti_entity
                0x000000008002dbb8                yeti_load_cell
                0x000000008002dcb8                yeti_save_cell
                0x000000008002dd48                yeti_load_map
                0x000000008002e130                yeti_save_map
                0x000000008002e210                visual_init
                0x000000008002e260                yeti_init
                0x000000008002e3f0                message_init
                0x000000008002e400                lua_init
                0x000000008002e690                yeti_init_lua
 .text          0x000000008002e788      0x108 /opt/toolchains/n64/mips64-elf/mips64-elf/lib/libm.a(lib_a-s_sin.o)
                0x000000008002e788                sin
 .text          0x000000008002e890      0x408 /opt/toolchains/n64/mips64-elf/mips64-elf/lib/libm.a(lib_a-w_pow.o)
                0x000000008002e890                pow
 .text          0x000000008002ec98      0x908 /opt/toolchains/n64/mips64-elf/mips64-elf/lib/libm.a(lib_a-e_pow.o)
                0x000000008002ec98                __ieee754_pow
 .text          0x000000008002f5a0      0x378 /opt/toolchains/n64/mips64-elf/mips64-elf/lib/libm.a(lib_a-e_rem_pio2.o)
                0x000000008002f5a0                __ieee754_rem_pio2
 .text          0x000000008002f918      0x2c0 /opt/toolchains/n64/mips64-elf/mips64-elf/lib/libm.a(lib_a-e_sqrt.o)
                0x000000008002f918                __ieee754_sqrt
 .text          0x000000008002fbd8      0x178 /opt/toolchains/n64/mips64-elf/mips64-elf/lib/libm.a(lib_a-k_cos.o)
                0x000000008002fbd8                __kernel_cos
 .text          0x000000008002fd50      0x908 /opt/toolchains/n64/mips64-elf/mips64-elf/lib/libm.a(lib_a-k_rem_pio2.o)
                0x000000008002fd50                __kernel_rem_pio2
 .text          0x0000000080030658       0xb8 /opt/toolchains/n64/mips64-elf/mips64-elf/lib/libm.a(lib_a-k_sin.o)
                0x0000000080030658                __kernel_sin
 .text          0x0000000080030710       0x30 /opt/toolchains/n64/mips64-elf/mips64-elf/lib/libm.a(lib_a-s_fabs.o)
                0x0000000080030710                fabs
 .text          0x0000000080030740       0x20 /opt/toolchains/n64/mips64-elf/mips64-elf/lib/libm.a(lib_a-s_finite.o)
                0x0000000080030740                finite
 .text          0x0000000080030760      0x198 /opt/toolchains/n64/mips64-elf/mips64-elf/lib/libm.a(lib_a-s_floor.o)
                0x0000000080030760                floor
 .text          0x00000000800308f8       0xa0 /opt/toolchains/n64/mips64-elf/mips64-elf/lib/libm.a(lib_a-s_fpclassify.o)
                0x00000000800308f8                __fpclassifyd
 .text          0x0000000080030998        0x0 /opt/toolchains/n64/mips64-elf/mips64-elf/lib/libm.a(lib_a-s_lib_ver.o)
 .text          0x0000000080030998        0x8 /opt/toolchains/n64/mips64-elf/mips64-elf/lib/libm.a(lib_a-s_matherr.o)
                0x0000000080030998                matherr
 .text          0x00000000800309a0       0x18 /opt/toolchains/n64/mips64-elf/mips64-elf/lib/libm.a(lib_a-s_nan.o)
                0x00000000800309a0                nan
 .text          0x00000000800309b8      0x1e0 /opt/toolchains/n64/mips64-elf/mips64-elf/lib/libm.a(lib_a-s_rint.o)
                0x00000000800309b8                rint
 .text          0x0000000080030b98      0x1a8 /opt/toolchains/n64/mips64-elf/mips64-elf/lib/libm.a(lib_a-s_scalbn.o)
                0x0000000080030b98                scalbn
 .text          0x0000000080030d40       0x40 /opt/toolchains/n64/mips64-elf/mips64-elf/lib/libm.a(lib_a-s_copysign.o)
                0x0000000080030d40                copysign
 .text          0x0000000080030d80      0x1d0 /opt/toolchains/n64/mips64-elf/lib/libdragon.a(n64sys.o)
                0x0000000080030d80                sys_get_boot_cic
                0x0000000080030d90                sys_set_boot_cic
                0x0000000080030db0                get_ticks
                0x0000000080030dc0                get_ticks_ms
                0x0000000080030de0                wait_ticks
                0x0000000080030e00                wait_ms
                0x0000000080030e38                data_cache_hit_writeback
                0x0000000080030e60                data_cache_hit_invalidate
                0x0000000080030e88                data_cache_hit_writeback_invalidate
                0x0000000080030eb0                data_cache_index_writeback_invalidate
                0x0000000080030ed8                inst_cache_hit_writeback
                0x0000000080030f00                inst_cache_hit_invalidate
                0x0000000080030f28                inst_cache_index_invalidate
 .text          0x0000000080030f50      0x5a8 /opt/toolchains/n64/mips64-elf/lib/libdragon.a(interrupt.o)
                0x0000000080031000                __MI_handler
                0x00000000800311d8                __TI_handler
                0x0000000080031220                register_AI_handler
                0x0000000080031230                unregister_AI_handler
                0x0000000080031240                register_VI_handler
                0x0000000080031250                unregister_VI_handler
                0x0000000080031260                register_PI_handler
                0x0000000080031270                unregister_PI_handler
                0x0000000080031280                register_DP_handler
                0x0000000080031290                unregister_DP_handler
                0x00000000800312a0                register_TI_handler
                0x00000000800312b0                unregister_TI_handler
                0x00000000800312c0                register_SI_handler
                0x00000000800312d0                unregister_SI_handler
                0x00000000800312e0                register_SP_handler
                0x00000000800312f0                unregister_SP_handler
                0x0000000080031300                set_AI_interrupt
                0x0000000080031330                set_VI_interrupt
                0x0000000080031368                set_PI_interrupt
                0x0000000080031398                set_DP_interrupt
                0x00000000800313c8                set_SI_interrupt
                0x00000000800313f8                set_SP_interrupt
                0x0000000080031428                init_interrupts
                0x0000000080031460                disable_interrupts
                0x00000000800314a0                enable_interrupts
                0x00000000800314d0                get_interrupts_state
 .text          0x00000000800314f8        0x0 /opt/toolchains/n64/mips64-elf/lib/libdragon.a(entrypoint.o)
 .text          0x00000000800314f8      0xfd0 /opt/toolchains/n64/mips64-elf/lib/libdragon.a(dragonfs.o)
                0x0000000080031ac8                dfs_chdir
                0x0000000080031af0                dfs_dir_findfirst
                0x0000000080031c58                dfs_dir_findnext
                0x0000000080031d88                dfs_open
                0x0000000080031f18                dfs_close
                0x0000000080031f90                dfs_seek
                0x00000000800320d8                dfs_tell
                0x0000000080032130                dfs_read
                0x0000000080032340                dfs_size
                0x0000000080032398                dfs_eof
                0x0000000080032400                dfs_init
 .text          0x00000000800324c8      0x628 /opt/toolchains/n64/mips64-elf/lib/libdragon.a(audio.o)
                0x00000000800325f0                audio_init
                0x0000000080032778                audio_close
                0x0000000080032828                audio_write
                0x0000000080032960                audio_write_silence
                0x0000000080032a80                audio_can_write
                0x0000000080032ad0                audio_get_frequency
                0x0000000080032ae0                audio_get_buffer_length
 .text          0x0000000080032af0      0x608 /opt/toolchains/n64/mips64-elf/lib/libdragon.a(display.o)
                0x0000000080032b40                display_init
                0x0000000080032f20                display_close
                0x0000000080032ff8                display_lock
                0x0000000080033098                display_show
 .text          0x00000000800330f8      0xe48 /opt/toolchains/n64/mips64-elf/lib/libdragon.a(controller.o)
                0x0000000080033308                controller_init
                0x0000000080033340                eeprom_present
                0x0000000080033380                eeprom_read
                0x00000000800333d8                eeprom_write
                0x0000000080033410                controller_read
                0x0000000080033420                controller_scan
                0x0000000080033498                get_keys_down
                0x0000000080033538                get_keys_up
                0x00000000800335d8                get_keys_held
                0x0000000080033670                get_keys_pressed
                0x00000000800336c8                get_dpad_direction
                0x0000000080033790                execute_raw_command
                0x0000000080033878                get_controllers_present
                0x00000000800338e0                get_accessories_present
                0x00000000800339f0                read_mempak_address
                0x0000000080033ba8                write_mempak_address
                0x0000000080033d60                identify_accessory
                0x0000000080033e68                rumble_start
                0x0000000080033ee0                rumble_stop
 .text          0x0000000080033f40     0x1320 /opt/toolchains/n64/mips64-elf/lib/libdragon.a(graphics.o)
                0x0000000080033f40                graphics_convert_color
                0x0000000080033fc8                graphics_make_color
                0x0000000080033ff8                graphics_set_color
                0x0000000080034010                graphics_draw_pixel
                0x00000000800340a0                graphics_draw_pixel_trans
                0x00000000800341e8                graphics_draw_line
                0x0000000080034390                graphics_draw_line_trans
                0x0000000080034538                graphics_draw_box
                0x0000000080034648                graphics_draw_box_trans
                0x0000000080034810                graphics_fill_screen
                0x00000000800348f8                graphics_draw_character
                0x0000000080034b28                graphics_draw_text
                0x0000000080034c28                graphics_draw_sprite_stride
                0x0000000080034eb8                graphics_draw_sprite
                0x0000000080034ed8                graphics_draw_sprite_trans_stride
                0x0000000080035240                graphics_draw_sprite_trans
 .text          0x0000000080035260      0xc38 /opt/toolchains/n64/mips64-elf/lib/libdragon.a(rdp.o)
                0x00000000800357b0                rdp_init
                0x00000000800357f0                rdp_close
                0x0000000080035818                rdp_attach_display
                0x0000000080035898                rdp_sync
                0x0000000080035940                rdp_detach_display
                0x00000000800359a8                rdp_set_clipping
                0x00000000800359f8                rdp_set_default_clipping
                0x0000000080035a18                rdp_enable_primitive_fill
                0x0000000080035a40                rdp_enable_texture_copy
                0x0000000080035a68                rdp_load_texture
                0x0000000080035aa8                rdp_load_texture_stride
                0x0000000080035b50                rdp_draw_textured_rectangle_scaled
                0x0000000080035ce8                rdp_draw_textured_rectangle
                0x0000000080035d18                rdp_draw_sprite
                0x0000000080035d68                rdp_draw_sprite_scaled
                0x0000000080035df0                rdp_set_primitive_color
                0x0000000080035e20                rdp_draw_filled_rectangle
                0x0000000080035e88                rdp_set_texture_flush
 .text          0x0000000080035e98      0x1b0 /opt/toolchains/n64/mips64-elf/lib/libdragon.a(dma.o)
                0x0000000080035e98                dma_busy
                0x0000000080035ea8                dma_read
                0x0000000080035f28                dma_write
                0x0000000080035fa8                io_read
                0x0000000080035ff8                io_write
 .text          0x0000000080036048      0x4d0 /opt/toolchains/n64/mips64-elf/lib/libdragon.a(timer.o)
                0x0000000080036240                timer_init
                0x0000000080036270                new_timer
                0x0000000080036310                start_timer
                0x0000000080036390                stop_timer
                0x0000000080036418                delete_timer
                0x0000000080036458                timer_close
                0x00000000800364e0                timer_ticks
 .text          0x0000000080036518      0x2e0 /opt/toolchains/n64/mips64-elf/lib/libdragon.a(inthandler.o)
                0x0000000080036518                inthandler
 .text          0x00000000800367f8       0xb0 /opt/toolchains/n64/mips64-elf/lib/libdragon.a(exception.o)
                0x00000000800367f8                register_exception_handler
                0x0000000080036808                __onCriticalException
                0x0000000080036858                __onResetException
 .text          0x00000000800368a8       0x78 /opt/toolchains/n64/mips64-elf/mips64-elf/lib/libc.a(lib_a-assert.o)
                0x00000000800368a8                __assert_func
                0x0000000080036908                __assert
 .text          0x0000000080036920        0x8 /opt/toolchains/n64/mips64-elf/mips64-elf/lib/libc.a(lib_a-errno.o)
                0x0000000080036920                __errno
 .text          0x0000000080036928      0x138 /opt/toolchains/n64/mips64-elf/mips64-elf/lib/libc.a(lib_a-fclose.o)
                0x0000000080036928                _fclose_r
                0x0000000080036a50                fclose
 .text          0x0000000080036a60      0x2f8 /opt/toolchains/n64/mips64-elf/mips64-elf/lib/libc.a(lib_a-fflush.o)
                0x0000000080036a60                __sflush_r
                0x0000000080036cd8                _fflush_r
                0x0000000080036d38                fflush
 .text          0x0000000080036d58      0x320 /opt/toolchains/n64/mips64-elf/mips64-elf/lib/libc.a(lib_a-findfp.o)
                0x0000000080036d68                _cleanup_r
                0x0000000080036e00                __sfmoreglue
                0x0000000080036e70                _cleanup
                0x0000000080036e78                __sinit
                0x0000000080036f08                __sfp
                0x0000000080037038                __sfp_lock_acquire
                0x0000000080037040                __sfp_lock_release
                0x0000000080037048                __sinit_lock_acquire
                0x0000000080037050                __sinit_lock_release
                0x0000000080037058                __fp_lock_all
                0x0000000080037068                __fp_unlock_all
 .text          0x0000000080037078       0x68 /opt/toolchains/n64/mips64-elf/mips64-elf/lib/libc.a(lib_a-fiprintf.o)
                0x0000000080037078                _fiprintf_r
                0x00000000800370a0                fiprintf
 .text          0x00000000800370e0      0x138 /opt/toolchains/n64/mips64-elf/mips64-elf/lib/libc.a(lib_a-fopen.o)
                0x00000000800370e0                _fopen_r
                0x0000000080037200                fopen
 .text          0x0000000080037218      0x320 /opt/toolchains/n64/mips64-elf/mips64-elf/lib/libc.a(lib_a-fread.o)
                0x0000000080037218                _fread_r
                0x0000000080037500                fread
 .text          0x0000000080037538      0x408 /opt/toolchains/n64/mips64-elf/mips64-elf/lib/libc.a(lib_a-freer.o)
                0x0000000080037538                _malloc_trim_r
                0x0000000080037670                _free_r
 .text          0x0000000080037940      0x500 /opt/toolchains/n64/mips64-elf/mips64-elf/lib/libc.a(lib_a-fseek.o)
                0x0000000080037940                _fseek_r
                0x0000000080037e20                fseek
 .text          0x0000000080037e40       0x58 /opt/toolchains/n64/mips64-elf/mips64-elf/lib/libc.a(lib_a-fstatr.o)
                0x0000000080037e40                _fstat_r
 .text          0x0000000080037e98      0x128 /opt/toolchains/n64/mips64-elf/mips64-elf/lib/libc.a(lib_a-ftell.o)
                0x0000000080037e98                _ftell_r
                0x0000000080037fb0                ftell
 .text          0x0000000080037fc0      0x188 /opt/toolchains/n64/mips64-elf/mips64-elf/lib/libc.a(lib_a-fwalk.o)
                0x0000000080037fc0                _fwalk
                0x0000000080038080                _fwalk_reent
 .text          0x0000000080038148      0x118 /opt/toolchains/n64/mips64-elf/mips64-elf/lib/libc.a(lib_a-fwrite.o)
                0x0000000080038148                _fwrite_r
                0x0000000080038228                fwrite
 .text          0x0000000080038260        0x0 /opt/toolchains/n64/mips64-elf/mips64-elf/lib/libc.a(lib_a-impure.o)
 .text          0x0000000080038260      0x1c0 /opt/toolchains/n64/mips64-elf/mips64-elf/lib/libc.a(lib_a-makebuf.o)
                0x0000000080038260                __smakebuf_r
 .text          0x0000000080038420       0x20 /opt/toolchains/n64/mips64-elf/mips64-elf/lib/libc.a(lib_a-malloc.o)
                0x0000000080038420                malloc
                0x0000000080038430                free
 .text          0x0000000080038440      0x8a8 /opt/toolchains/n64/mips64-elf/mips64-elf/lib/libc.a(lib_a-mallocr.o)
                0x0000000080038440                _malloc_r
 .text          0x0000000080038ce8      0x160 /opt/toolchains/n64/mips64-elf/mips64-elf/lib/libc.a(lib_a-memcpy.o)
                0x0000000080038ce8                memcpy
 .text          0x0000000080038e48       0xf0 /opt/toolchains/n64/mips64-elf/mips64-elf/lib/libc.a(lib_a-memset.o)
                0x0000000080038e48                memset
 .text          0x0000000080038f38       0x10 /opt/toolchains/n64/mips64-elf/mips64-elf/lib/libc.a(lib_a-mlock.o)
                0x0000000080038f38                __malloc_lock
                0x0000000080038f40                __malloc_unlock
 .text          0x0000000080038f48       0x58 /opt/toolchains/n64/mips64-elf/mips64-elf/lib/libc.a(lib_a-openr.o)
                0x0000000080038f48                _open_r
 .text          0x0000000080038fa0       0x18 /opt/toolchains/n64/mips64-elf/mips64-elf/lib/libc.a(lib_a-realloc.o)
                0x0000000080038fa0                realloc
 .text          0x0000000080038fb8      0x6c0 /opt/toolchains/n64/mips64-elf/mips64-elf/lib/libc.a(lib_a-reallocr.o)
                0x0000000080038fb8                _realloc_r
 .text          0x0000000080039678      0x250 /opt/toolchains/n64/mips64-elf/mips64-elf/lib/libc.a(lib_a-reent.o)
                0x0000000080039678                cleanup_glue
                0x00000000800396c0                _reclaim_reent
                0x0000000080039800                _wrapup_reent
 .text          0x00000000800398c8      0x270 /opt/toolchains/n64/mips64-elf/mips64-elf/lib/libc.a(lib_a-refill.o)
                0x00000000800398f0                __srefill_r
 .text          0x0000000080039b38       0x50 /opt/toolchains/n64/mips64-elf/mips64-elf/lib/libc.a(lib_a-sbrkr.o)
                0x0000000080039b38                _sbrk_r
 .text          0x0000000080039b88       0xd0 /opt/toolchains/n64/mips64-elf/mips64-elf/lib/libc.a(lib_a-sprintf.o)
                0x0000000080039b88                _sprintf_r
                0x0000000080039be8                sprintf
 .text          0x0000000080039c58      0x148 /opt/toolchains/n64/mips64-elf/mips64-elf/lib/libc.a(lib_a-stdio.o)
                0x0000000080039c58                __sread
                0x0000000080039cb0                __seofread
                0x0000000080039cb8                __swrite
                0x0000000080039d38                __sseek
                0x0000000080039d98                __sclose
 .text          0x0000000080039da0       0x68 /opt/toolchains/n64/mips64-elf/mips64-elf/lib/libc.a(lib_a-strcmp.o)
                0x0000000080039da0                strcmp
 .text          0x0000000080039e08       0xa8 /opt/toolchains/n64/mips64-elf/mips64-elf/lib/libc.a(lib_a-strcpy.o)
                0x0000000080039e08                strcpy
 .text          0x0000000080039eb0       0x18 /opt/toolchains/n64/mips64-elf/mips64-elf/lib/libc.a(lib_a-strlen.o)
                0x0000000080039eb0                strlen
 .text          0x0000000080039ec8     0x1d08 /opt/toolchains/n64/mips64-elf/mips64-elf/lib/libc.a(lib_a-svfprintf.o)
                0x0000000080039ec8                _svfprintf_r
 .text          0x000000008003bbd0     0x1080 /opt/toolchains/n64/mips64-elf/mips64-elf/lib/libc.a(lib_a-vfiprintf.o)
                0x000000008003bbd0                __sprint_r
                0x000000008003bcc0                _vfiprintf_r
                0x000000008003cc30                vfiprintf
 .text          0x000000008003cc50       0x58 /opt/toolchains/n64/mips64-elf/mips64-elf/lib/libc.a(lib_a-writer.o)
                0x000000008003cc50                _write_r
 .text          0x000000008003cca8      0x178 /opt/toolchains/n64/mips64-elf/mips64-elf/lib/libc.a(lib_a-wsetup.o)
                0x000000008003cca8                __swsetup_r
 .text          0x000000008003ce20       0x18 /opt/toolchains/n64/mips64-elf/mips64-elf/lib/libc.a(lib_a-abort.o)
                0x000000008003ce20                abort
 .text          0x000000008003ce38       0x50 /opt/toolchains/n64/mips64-elf/mips64-elf/lib/libc.a(lib_a-closer.o)
                0x000000008003ce38                _close_r
 .text          0x000000008003ce88     0x1510 /opt/toolchains/n64/mips64-elf/mips64-elf/lib/libc.a(lib_a-dtoa.o)
                0x000000008003d0d0                _dtoa_r
 .text          0x000000008003e398       0xa8 /opt/toolchains/n64/mips64-elf/mips64-elf/lib/libc.a(lib_a-flags.o)
                0x000000008003e398                __sflags
 .text          0x000000008003e440      0x260 /opt/toolchains/n64/mips64-elf/mips64-elf/lib/libc.a(lib_a-fputwc.o)
                0x000000008003e440                _fputwc_r
                0x000000008003e648                fputwc
 .text          0x000000008003e6a0      0x548 /opt/toolchains/n64/mips64-elf/mips64-elf/lib/libc.a(lib_a-fvwrite.o)
                0x000000008003e6a0                __sfvwrite_r
 .text          0x000000008003ebe8       0x50 /opt/toolchains/n64/mips64-elf/mips64-elf/lib/libc.a(lib_a-isattyr.o)
                0x000000008003ebe8                _isatty_r
 .text          0x000000008003ec38       0xf0 /opt/toolchains/n64/mips64-elf/mips64-elf/lib/libc.a(lib_a-locale.o)
                0x000000008003ec38                _setlocale_r
                0x000000008003ecc0                __locale_charset
                0x000000008003ecd0                __locale_mb_cur_max
                0x000000008003ecd8                __locale_msgcharset
                0x000000008003ece8                __locale_cjk_lang
                0x000000008003ecf0                _localeconv_r
                0x000000008003ed00                setlocale
                0x000000008003ed18                localeconv
 .text          0x000000008003ed28       0x58 /opt/toolchains/n64/mips64-elf/mips64-elf/lib/libc.a(lib_a-lseekr.o)
                0x000000008003ed28                _lseek_r
 .text          0x000000008003ed80      0x100 /opt/toolchains/n64/mips64-elf/mips64-elf/lib/libc.a(lib_a-memchr.o)
                0x000000008003ed80                memchr
 .text          0x000000008003ee80      0x150 /opt/toolchains/n64/mips64-elf/mips64-elf/lib/libc.a(lib_a-memmove.o)
                0x000000008003ee80                memmove
 .text          0x000000008003efd0     0x11f0 /opt/toolchains/n64/mips64-elf/mips64-elf/lib/libc.a(lib_a-mprec.o)
                0x000000008003efd0                _Balloc
                0x000000008003f088                _Bfree
                0x000000008003f0b8                __multadd
                0x000000008003f1e0                __s2b
                0x000000008003f330                __hi0bits
                0x000000008003f3b0                __lo0bits
                0x000000008003f470                __i2b
                0x000000008003f4a8                __multiply
                0x000000008003f6f0                __pow5mult
                0x000000008003f828                __lshift
                0x000000008003f9a8                __mcmp
                0x000000008003fa08                __mdiff
                0x000000008003fbd0                __ulp
                0x000000008003fc60                __b2d
                0x000000008003fde0                __d2b
                0x000000008003ff48                __ratio
                0x0000000080040028                _mprec_log10
                0x0000000080040068                __copybits
                0x00000000800400f8                __any_on
 .text          0x00000000800401c0       0x58 /opt/toolchains/n64/mips64-elf/mips64-elf/lib/libc.a(lib_a-readr.o)
                0x00000000800401c0                _read_r
 .text          0x0000000080040218      0x2a8 /opt/toolchains/n64/mips64-elf/mips64-elf/lib/libc.a(lib_a-signal.o)
                0x0000000080040218                _init_signal_r
                0x0000000080040298                _signal_r
                0x0000000080040320                _raise_r
                0x00000000800403e8                __sigtramp_r
                0x0000000080040480                raise
                0x0000000080040490                signal
                0x00000000800404a8                _init_signal
                0x00000000800404b0                __sigtramp
 .text          0x00000000800404c0       0x60 /opt/toolchains/n64/mips64-elf/mips64-elf/lib/libc.a(lib_a-signalr.o)
                0x00000000800404c0                _kill_r
                0x0000000080040518                _getpid_r
 .text          0x0000000080040520     0x10b0 /opt/toolchains/n64/mips64-elf/mips64-elf/lib/libc.a(lib_a-svfiprintf.o)
                0x0000000080040520                __ssprint_r
                0x0000000080040768                _svfiprintf_r
 .text          0x00000000800415d0      0x1c0 /opt/toolchains/n64/mips64-elf/mips64-elf/lib/libc.a(lib_a-wbuf.o)
                0x00000000800415d0                __swbuf_r
                0x0000000080041778                __swbuf
 .text          0x0000000080041790      0x158 /opt/toolchains/n64/mips64-elf/mips64-elf/lib/libc.a(lib_a-wcrtomb.o)
                0x0000000080041790                _wcrtomb_r
                0x0000000080041830                wcrtomb
 .text          0x00000000800418e8       0x90 /opt/toolchains/n64/mips64-elf/mips64-elf/lib/libc.a(lib_a-wctomb_r.o)
                0x00000000800418e8                __ascii_wctomb
                0x0000000080041920                _wctomb_r
 .text          0x0000000080041978       0xc8 /opt/toolchains/n64/mips64-elf/mips64-elf/lib/libc.a(lib_a-callocr.o)
                0x0000000080041978                _calloc_r
 .text          0x0000000080041a40      0xff8 /opt/toolchains/n64/mips64-elf/lib/libdragonsys.a(system.o)
                0x0000000080041ba0                attach_filesystem
                0x0000000080041da8                chown
                0x0000000080041dc0                close
                0x0000000080041ea8                detach_filesystem
                0x0000000080041fd0                execve
                0x0000000080041fe8                exit
                0x0000000080041ff0                fork
                0x0000000080042008                fstat
                0x00000000800420f8                getpid
                0x0000000080042110                gettimeofday
                0x0000000080042128                isatty
                0x0000000080042150                kill
                0x0000000080042168                link
                0x0000000080042180                lseek
                0x0000000080042268                open
                0x0000000080042410                read
                0x0000000080042530                readlink
                0x0000000080042548                sbrk
                0x00000000800425f8                stat
                0x0000000080042668                symlink
                0x0000000080042680                times
                0x0000000080042698                unlink
                0x0000000080042760                wait
                0x0000000080042778                write
                0x00000000800428b8                dir_findfirst
                0x0000000080042978                dir_findnext
                0x00000000800429e0                hook_stdio_calls
                0x0000000080042a18                unhook_stdio_calls
 .text          0x0000000080042a38        0x8 /opt/toolchains/n64/mips64-elf/mips64-elf/lib/libnosys.a(_exit.o)
                0x0000000080042a38                _exit
 *(.text.*)
 .text.startup  0x0000000080042a40      0x3a8 main.o
                0x0000000080042a40                main
 .text.unlikely
                0x0000000080042de8      0x2dc stb_image.o
 *(.gnu.linkonce.t.*)
                0x00000000800430d0                . = ALIGN (0x10)
 *fill*         0x00000000800430c4        0xc 00
                0x00000000800430d0                __INIT_SECTION__ = .
 *(.init)
                0x00000000800430d0        0x4 LONG 0x3e00008
                0x00000000800430d4        0x4 LONG 0x0
                0x00000000800430e0                . = ALIGN (0x10)
 *fill*         0x00000000800430d8        0x8 00
                0x00000000800430e0                __FINI_SECTION__ = .
 *(.fini)
                0x00000000800430e0        0x4 LONG 0x3e00008
                0x00000000800430e4        0x4 LONG 0x0

.eh_frame_hdr
 *(.eh_frame_hdr)

.eh_frame
 *(.eh_frame)

.gcc_except_table
 *(.gcc_except_table)

.jcr
 *(.jcr)

.ctors          0x00000000800430e8       0x10 load address 0x0000000000042ce8
                0x00000000800430f0                . = ALIGN (0x10)
 *fill*         0x00000000800430e8        0x8 00
                0x00000000800430f0                __CTOR_LIST__ = .
                0x00000000800430f0                ___CTOR_LIST__ = .
                0x00000000800430f0        0x4 LONG 0x0 (((__CTOR_END__ - __CTOR_LIST__) / 0x4) - 0x2)
 *(SORT(.ctors.*))
 *(.ctors)
                0x00000000800430f4        0x4 LONG 0x0
                0x00000000800430f8                __CTOR_END__ = .

.dtors          0x00000000800430f8       0x10 load address 0x0000000000042cf8
                0x0000000080043100                . = ALIGN (0x10)
 *fill*         0x00000000800430f8        0x8 00
                0x0000000080043100                __DTOR_LIST__ = .
                0x0000000080043100                ___DTOR_LIST__ = .
                0x0000000080043100        0x4 LONG 0x0 (((__DTOR_END__ - __DTOR_LIST__) / 0x4) - 0x2)
 *(SORT(.dtors.*))
 *(.dtors)
                0x0000000080043104        0x4 LONG 0x0
                0x0000000080043108                __DTOR_END__ = .
                0x0000000080043108                . = .

.rodata         0x0000000080043108     0x2ba0 load address 0x0000000000042d08
 *(.rdata)
 *(.rodata)
 .rodata        0x0000000080043108      0x4e8 stb_image.o
 .rodata        0x00000000800435f0       0xc0 ../game/ai/explode.o
 .rodata        0x00000000800436b0       0x10 ../game/ai/sheba.o
 .rodata        0x00000000800436c0       0x20 ../game/ai/torch.o
 .rodata        0x00000000800436e0       0x78 ../game/game.o
 .rodata        0x0000000080043758       0x20 ../game/screens.o
 .rodata        0x0000000080043778       0x28 ../y3d/y3d_animation.o
 .rodata        0x00000000800437a0      0x300 ../y3d/y3d_draw.o
 .rodata        0x0000000080043aa0       0x3c ../y3d/y3d_engine.o
 .rodata        0x0000000080043adc       0x20 ../y3d/y3d_fruity.o
 .rodata        0x0000000080043afc       0x98 ../y3d/y3d_image.o
 .rodata        0x0000000080043b94       0x18 ../y3d/y3d_pixel.o
 *fill*         0x0000000080043bac        0x4 00
 .rodata        0x0000000080043bb0       0x18 ../y3d/y3d_spanner.o
 .rodata        0x0000000080043bc8       0x30 /opt/toolchains/n64/mips64-elf/mips64-elf/lib/libm.a(lib_a-e_pow.o)
 .rodata        0x0000000080043bf8      0x188 /opt/toolchains/n64/mips64-elf/mips64-elf/lib/libm.a(lib_a-e_rem_pio2.o)
 .rodata        0x0000000080043d80       0x50 /opt/toolchains/n64/mips64-elf/mips64-elf/lib/libm.a(lib_a-k_rem_pio2.o)
 .rodata        0x0000000080043dd0       0x10 /opt/toolchains/n64/mips64-elf/mips64-elf/lib/libm.a(lib_a-s_rint.o)
 .rodata        0x0000000080043de0       0x10 /opt/toolchains/n64/mips64-elf/lib/libdragon.a(audio.o)
 .rodata        0x0000000080043df0      0x2d0 /opt/toolchains/n64/mips64-elf/lib/libdragon.a(display.o)
 .rodata        0x00000000800440c0       0x20 /opt/toolchains/n64/mips64-elf/lib/libdragon.a(controller.o)
 .rodata        0x00000000800440e0      0x800 /opt/toolchains/n64/mips64-elf/lib/libdragon.a(graphics.o)
 .rodata        0x00000000800448e0      0x188 /opt/toolchains/n64/mips64-elf/mips64-elf/lib/libc.a(lib_a-svfprintf.o)
 .rodata        0x0000000080044a68      0x188 /opt/toolchains/n64/mips64-elf/mips64-elf/lib/libc.a(lib_a-vfiprintf.o)
 .rodata        0x0000000080044bf0      0x128 /opt/toolchains/n64/mips64-elf/mips64-elf/lib/libc.a(lib_a-mprec.o)
                0x0000000080044bf0                __mprec_tinytens
                0x0000000080044c18                __mprec_bigtens
                0x0000000080044c40                __mprec_tens
 .rodata        0x0000000080044d18      0x188 /opt/toolchains/n64/mips64-elf/mips64-elf/lib/libc.a(lib_a-svfiprintf.o)
 *(.rodata.*)
 .rodata.str1.8
                0x0000000080044ea0      0x34b main.o
                                        0x350 (size before relaxing)
 *fill*         0x00000000800451eb        0x1 00
 .rodata.cst4   0x00000000800451ec        0x4 main.o
 .rodata.str1.8
                0x00000000800451f0      0x6cc stb_image.o
                                        0x6d8 (size before relaxing)
 *fill*         0x00000000800458bc        0x4 00
 .rodata.str1.8
                0x00000000800458c0       0x30 ../game/game.o
 .rodata.str1.8
                0x00000000800458f0      0x1f2 ../game/screens.o
                                        0x1f8 (size before relaxing)
 *fill*         0x0000000080045ae2        0x6 00
 .rodata.str1.8
                0x0000000080045ae8        0x5 ../y3d/y3d_engine.o
                                          0x8 (size before relaxing)
 .rodata.str1.8
                0x0000000000000000        0x8 ../y3d/y3d_file.o
 *fill*         0x0000000080045aed        0x3 00
 .rodata.str1.8
                0x0000000080045af0        0x3 ../y3d/y3d_record.o
                                         0x10 (size before relaxing)
 *fill*         0x0000000080045af3        0x5 00
 .rodata.str1.8
                0x0000000080045af8       0x41 ../y3d/y3d_spanner.o
                                         0x48 (size before relaxing)
 *fill*         0x0000000080045b39        0x7 00
 .rodata.cst8   0x0000000080045b40       0x28 ../y3d/y3d_yeti.o
 .rodata.cst4   0x0000000080045b68       0x18 ../y3d/y3d_yeti.o
 .rodata.str1.8
                0x0000000080045b80        0x4 /opt/toolchains/n64/mips64-elf/mips64-elf/lib/libm.a(lib_a-w_pow.o)
                                          0x8 (size before relaxing)
 .rodata.str1.8
                0x0000000000000000        0x8 /opt/toolchains/n64/mips64-elf/mips64-elf/lib/libm.a(lib_a-e_pow.o)
 *fill*         0x0000000080045b84        0x4 00
 .rodata.str1.8
                0x0000000080045b88       0x1e /opt/toolchains/n64/mips64-elf/lib/libdragon.a(dragonfs.o)
                                         0x20 (size before relaxing)
 *fill*         0x0000000080045ba6        0x2 00
 .rodata.cst8   0x0000000080045ba8       0x18 /opt/toolchains/n64/mips64-elf/lib/libdragon.a(rdp.o)
                                         0x20 (size before relaxing)
 .rodata.str1.8
                0x0000000080045bc0       0x22 /opt/toolchains/n64/mips64-elf/lib/libdragon.a(exception.o)
                                         0x28 (size before relaxing)
 *fill*         0x0000000080045be2        0x6 00
 .rodata.str1.8
                0x0000000080045be8       0x3f /opt/toolchains/n64/mips64-elf/mips64-elf/lib/libc.a(lib_a-assert.o)
                                         0x48 (size before relaxing)
 *fill*         0x0000000080045c27        0x1 00
 .rodata.str1.8
                0x0000000080045c28        0x2 /opt/toolchains/n64/mips64-elf/mips64-elf/lib/libc.a(lib_a-impure.o)
                                          0x8 (size before relaxing)
 *fill*         0x0000000080045c2a        0x6 00
 .rodata.str1.8
                0x0000000080045c30       0x57 /opt/toolchains/n64/mips64-elf/mips64-elf/lib/libc.a(lib_a-svfprintf.o)
                                         0x60 (size before relaxing)
 .rodata.str1.8
                0x0000000000000000       0x38 /opt/toolchains/n64/mips64-elf/mips64-elf/lib/libc.a(lib_a-vfiprintf.o)
 *fill*         0x0000000080045c87        0x1 00
 .rodata.str1.8
                0x0000000080045c88       0x14 /opt/toolchains/n64/mips64-elf/mips64-elf/lib/libc.a(lib_a-dtoa.o)
                                         0x20 (size before relaxing)
 *fill*         0x0000000080045c9c        0x4 00
 .rodata.str1.8
                0x0000000080045ca0        0x8 /opt/toolchains/n64/mips64-elf/mips64-elf/lib/libc.a(lib_a-locale.o)
                                         0x20 (size before relaxing)
 .rodata.str1.8
                0x0000000000000000       0x38 /opt/toolchains/n64/mips64-elf/mips64-elf/lib/libc.a(lib_a-svfiprintf.o)
 *(.gnu.linkonce.r.*)

.rel.dyn        0x0000000080045ca8        0x0 load address 0x00000000000458a8
 .rel.dyn       0x0000000000000000        0x0 ../game/maps.o
                0x0000000080045cb0                . = ALIGN (0x10)
                0x0000000080045cb0                __text_end = .

.data           0x0000000080045ca8   0x3a3ea0 load address 0x00000000000458a8
                0x0000000080045ca8                __data_start = .
 *(.data)
 .data          0x0000000080045ca8       0x80 main.o
                0x0000000080045ca8                mapnames
 .data          0x0000000080045d28       0x18 stb_image.o
 .data          0x0000000080045d40        0x0 ../game/ai/boost.o
 .data          0x0000000080045d40        0x0 ../game/ai/bullet.o
 .data          0x0000000080045d40        0x0 ../game/ai/death.o
 .data          0x0000000080045d40        0x0 ../game/ai/explode.o
 .data          0x0000000080045d40        0x0 ../game/ai/pickup.o
 .data          0x0000000080045d40        0x0 ../game/ai/quad.o
 .data          0x0000000080045d40        0x0 ../game/ai/sheba.o
 .data          0x0000000080045d40        0x0 ../game/ai/static_model.o
 .data          0x0000000080045d40        0x0 ../game/ai/static_sprite.o
 .data          0x0000000080045d40        0x0 ../game/ai/teleporter.o
 .data          0x0000000080045d40        0x0 ../game/ai/torch.o
 .data          0x0000000080045d40    0x80300 ../game/data.o
                0x0000000080045d40                palette
                0x0000000080046040                textures
 .data          0x00000000800c6040        0x0 ../game/entities.o
 .data          0x00000000800c6040        0x0 ../game/game.o
 .data          0x00000000800c6040    0x10088 ../game/maps.o
                0x00000000800c6040                maps
                0x00000000800c6048                map_cave
 .data          0x00000000800d60c8   0x1ceeb8 ../game/models.o
                0x00000000800d60c8                size_teleporter
                0x00000000800d60cc                size_box
                0x00000000800d60d0                size_quad
                0x00000000800d60d4                size_boost
                0x00000000800d60d8                size_emptypot
                0x00000000800d60dc                size_pillar
                0x00000000800d60e0                size_bridge
                0x00000000800d60e4                size_overpass
                0x00000000800d60e8                size_crate
                0x00000000800d60ec                size_pinechair
                0x00000000800d60f0                size_potplant
                0x00000000800d60f4                size_cactus
                0x00000000800d60f8                size_leafyplant
                0x00000000800d60fc                size_barrontree
                0x00000000800d6100                size_ogro
                0x00000000800d6104                size_bauul
                0x00000000800d6108                size_rat
                0x00000000800d610c                size_rocket
                0x00000000800d6110                model_teleporter
                0x00000000800de1d0                model_box
                0x00000000800e6308                model_quad
                0x00000000800eec58                model_boost
                0x00000000800f72f0                model_emptypot
                0x00000000800ffa28                model_pillar
                0x0000000080108438                model_bridge
                0x0000000080110678                model_overpass
                0x00000000801187b0                model_crate
                0x00000000801208e8                model_pinechair
                0x0000000080129398                model_potplant
                0x00000000801331e8                model_cactus
                0x000000008013bab0                model_leafyplant
                0x0000000080144be8                model_barrontree
                0x000000008014da78                model_ogro
                0x00000000801c0700                model_bauul
                0x0000000080220070                model_rat
                0x000000008028e170                model_rocket
 .data          0x00000000802a4f80        0x0 ../game/screens.o
 .data          0x00000000802a4f80   0x144120 ../game/sprites.o
                0x00000000802a4f80                sprites
                0x00000000802a50d8                spr_yeti3d
                0x00000000802a9be0                spr_tree1
                0x00000000802b1be8                spr_torch7
                0x00000000802b3048                spr_torch6
                0x00000000802b44a8                spr_torch5
                0x00000000802b5908                spr_torch4
                0x00000000802b6d68                spr_torch3
                0x00000000802b9480                spr_torch2
                0x00000000802bbb98                spr_torch1
                0x00000000802be2b0                spr_torch0
                0x00000000802c09c8                spr_test
                0x00000000802c57f0                spr_temple
                0x00000000802ca2f8                spr_splat31
                0x00000000802cc300                spr_splat30
                0x00000000802ce308                spr_splat29
                0x00000000802d0310                spr_splat28
                0x00000000802d2318                spr_splat27
                0x00000000802d4320                spr_splat26
                0x00000000802d6328                spr_splat25
                0x00000000802d8330                spr_splat24
                0x00000000802da338                spr_splat23
                0x00000000802dc340                spr_splat22
                0x00000000802de348                spr_splat21
                0x00000000802e0350                spr_splat20
                0x00000000802e2358                spr_splat19
                0x00000000802e4360                spr_splat18
                0x00000000802e6368                spr_splat17
                0x00000000802e8370                spr_splat16
                0x00000000802ea378                spr_splat15
                0x00000000802ec380                spr_splat14
                0x00000000802ee388                spr_splat13
                0x00000000802f0390                spr_splat12
                0x00000000802f2398                spr_splat11
                0x00000000802f43a0                spr_splat10
                0x00000000802f63a8                spr_splat09
                0x00000000802f83b0                spr_splat08
                0x00000000802fa3b8                spr_splat07
                0x00000000802fc3c0                spr_splat06
                0x00000000802fe3c8                spr_splat05
                0x00000000803003d0                spr_splat04
                0x00000000803023d8                spr_splat03
                0x00000000803043e0                spr_splat02
                0x00000000803063e8                spr_splat01
                0x00000000803083f0                spr_splat00
                0x000000008030a3f8                spr_sky2
                0x000000008034a400                spr_sheba3
                0x0000000080350080                spr_sheba2
                0x0000000080355d00                spr_sheba1
                0x000000008035b980                spr_sheba0
                0x0000000080361600                spr_publisher
                0x0000000080366108                spr_menu
                0x0000000080366190                spr_hud
                0x0000000080366e18                spr_horror
                0x000000008036a020                spr_font
                0x0000000080372028                spr_flare3
                0x0000000080373eb0                spr_flare2
                0x000000008037beb8                spr_flare1
                0x0000000080383ec0                spr_flare0
                0x000000008038bec8                spr_flames3
                0x00000000803909d0                spr_flames2
                0x00000000803954d8                spr_flames1
                0x0000000080399fe0                spr_flames0
                0x000000008039eae8                spr_face
                0x00000000803a35f0                spr_explode0
                0x00000000803ab5f8                spr_expl9
                0x00000000803ad600                spr_expl8
                0x00000000803af608                spr_expl7
                0x00000000803b1610                spr_expl6
                0x00000000803b3618                spr_expl5
                0x00000000803b5620                spr_expl4
                0x00000000803b7628                spr_expl3
                0x00000000803b9630                spr_expl2
                0x00000000803bb638                spr_expl15
                0x00000000803bd640                spr_expl14
                0x00000000803bf648                spr_expl13
                0x00000000803c1650                spr_expl12
                0x00000000803c3658                spr_expl11
                0x00000000803c5660                spr_expl10
                0x00000000803c7668                spr_expl1
                0x00000000803c9670                spr_expl0
                0x00000000803cb678                spr_credits
                0x00000000803d0180                spr_blood3
                0x00000000803d6548                spr_blood2
                0x00000000803dc910                spr_blood1
                0x00000000803e2cd8                spr_blood0
 .data          0x00000000803e90a0        0x0 ../y3d/y3d_animation.o
 .data          0x00000000803e90a0        0x0 ../y3d/y3d_ansic.o
 .data          0x00000000803e90a0        0x0 ../y3d/y3d_cell.o
 .data          0x00000000803e90a0       0x20 ../y3d/y3d_draw.o
                0x00000000803e90a0                dither_kernals
 .data          0x00000000803e90c0        0x0 ../y3d/y3d_engine.o
 .data          0x00000000803e90c0        0x0 ../y3d/y3d_entity.o
 .data          0x00000000803e90c0        0x0 ../y3d/y3d_file.o
 .data          0x00000000803e90c0        0x0 ../y3d/y3d_fixed.o
 .data          0x00000000803e90c0        0x0 ../y3d/y3d_fruity.o
 .data          0x00000000803e90c0        0x0 ../y3d/y3d_image.o
 .data          0x00000000803e90c0        0x0 ../y3d/y3d_keyboard.o
 .data          0x00000000803e90c0        0x0 ../y3d/y3d_map.o
 .data          0x00000000803e90c0        0x0 ../y3d/y3d_matrix.o
 .data          0x00000000803e90c0        0x0 ../y3d/y3d_pixel.o
 .data          0x00000000803e90c0        0x0 ../y3d/y3d_record.o
 .data          0x00000000803e90c0        0x0 ../y3d/y3d_sound.o
 .data          0x00000000803e90c0        0x0 ../y3d/y3d_spanner.o
 .data          0x00000000803e90c0        0x0 ../y3d/y3d_surface.o
 .data          0x00000000803e90c0        0x0 ../y3d/y3d_vertex.o
 .data          0x00000000803e90c0        0x0 ../y3d/y3d_yeti.o
 .data          0x00000000803e90c0        0x0 /opt/toolchains/n64/mips64-elf/mips64-elf/lib/libm.a(lib_a-s_sin.o)
 .data          0x00000000803e90c0        0x0 /opt/toolchains/n64/mips64-elf/mips64-elf/lib/libm.a(lib_a-w_pow.o)
 .data          0x00000000803e90c0        0x0 /opt/toolchains/n64/mips64-elf/mips64-elf/lib/libm.a(lib_a-e_pow.o)
 .data          0x00000000803e90c0        0x0 /opt/toolchains/n64/mips64-elf/mips64-elf/lib/libm.a(lib_a-e_rem_pio2.o)
 .data          0x00000000803e90c0        0x0 /opt/toolchains/n64/mips64-elf/mips64-elf/lib/libm.a(lib_a-e_sqrt.o)
 .data          0x00000000803e90c0        0x0 /opt/toolchains/n64/mips64-elf/mips64-elf/lib/libm.a(lib_a-k_cos.o)
 .data          0x00000000803e90c0        0x0 /opt/toolchains/n64/mips64-elf/mips64-elf/lib/libm.a(lib_a-k_rem_pio2.o)
 .data          0x00000000803e90c0        0x0 /opt/toolchains/n64/mips64-elf/mips64-elf/lib/libm.a(lib_a-k_sin.o)
 .data          0x00000000803e90c0        0x0 /opt/toolchains/n64/mips64-elf/mips64-elf/lib/libm.a(lib_a-s_fabs.o)
 .data          0x00000000803e90c0        0x0 /opt/toolchains/n64/mips64-elf/mips64-elf/lib/libm.a(lib_a-s_finite.o)
 .data          0x00000000803e90c0        0x0 /opt/toolchains/n64/mips64-elf/mips64-elf/lib/libm.a(lib_a-s_floor.o)
 .data          0x00000000803e90c0        0x0 /opt/toolchains/n64/mips64-elf/mips64-elf/lib/libm.a(lib_a-s_fpclassify.o)
 .data          0x00000000803e90c0        0x0 /opt/toolchains/n64/mips64-elf/mips64-elf/lib/libm.a(lib_a-s_lib_ver.o)
 .data          0x00000000803e90c0        0x0 /opt/toolchains/n64/mips64-elf/mips64-elf/lib/libm.a(lib_a-s_matherr.o)
 .data          0x00000000803e90c0        0x0 /opt/toolchains/n64/mips64-elf/mips64-elf/lib/libm.a(lib_a-s_nan.o)
 .data          0x00000000803e90c0        0x0 /opt/toolchains/n64/mips64-elf/mips64-elf/lib/libm.a(lib_a-s_rint.o)
 .data          0x00000000803e90c0        0x0 /opt/toolchains/n64/mips64-elf/mips64-elf/lib/libm.a(lib_a-s_scalbn.o)
 .data          0x00000000803e90c0        0x0 /opt/toolchains/n64/mips64-elf/mips64-elf/lib/libm.a(lib_a-s_copysign.o)
 .data          0x00000000803e90c0        0x4 /opt/toolchains/n64/mips64-elf/lib/libdragon.a(n64sys.o)
                0x00000000803e90c0                __bootcic
 .data          0x00000000803e90c4        0x4 /opt/toolchains/n64/mips64-elf/lib/libdragon.a(interrupt.o)
 .data          0x00000000803e90c8        0x0 /opt/toolchains/n64/mips64-elf/lib/libdragon.a(entrypoint.o)
 .data          0x00000000803e90c8       0x30 /opt/toolchains/n64/mips64-elf/lib/libdragon.a(dragonfs.o)
 .data          0x00000000803e90f8        0x4 /opt/toolchains/n64/mips64-elf/lib/libdragon.a(audio.o)
 .data          0x00000000803e90fc       0x10 /opt/toolchains/n64/mips64-elf/lib/libdragon.a(display.o)
                0x00000000803e90fc                __buffers
 *fill*         0x00000000803e910c        0x4 00
 .data          0x00000000803e9110      0x180 /opt/toolchains/n64/mips64-elf/lib/libdragon.a(controller.o)
 .data          0x00000000803e9290        0x4 /opt/toolchains/n64/mips64-elf/lib/libdragon.a(graphics.o)
 .data          0x00000000803e9294        0x4 /opt/toolchains/n64/mips64-elf/lib/libdragon.a(rdp.o)
 .data          0x00000000803e9298        0x0 /opt/toolchains/n64/mips64-elf/lib/libdragon.a(dma.o)
 .data          0x00000000803e9298        0x0 /opt/toolchains/n64/mips64-elf/lib/libdragon.a(timer.o)
 .data          0x00000000803e9298        0x0 /opt/toolchains/n64/mips64-elf/lib/libdragon.a(inthandler.o)
 .data          0x00000000803e9298        0x0 /opt/toolchains/n64/mips64-elf/lib/libdragon.a(exception.o)
 .data          0x00000000803e9298        0x0 /opt/toolchains/n64/mips64-elf/mips64-elf/lib/libc.a(lib_a-assert.o)
 .data          0x00000000803e9298        0x0 /opt/toolchains/n64/mips64-elf/mips64-elf/lib/libc.a(lib_a-errno.o)
 .data          0x00000000803e9298        0x0 /opt/toolchains/n64/mips64-elf/mips64-elf/lib/libc.a(lib_a-fclose.o)
 .data          0x00000000803e9298        0x0 /opt/toolchains/n64/mips64-elf/mips64-elf/lib/libc.a(lib_a-fflush.o)
 .data          0x00000000803e9298        0x0 /opt/toolchains/n64/mips64-elf/mips64-elf/lib/libc.a(lib_a-findfp.o)
 .data          0x00000000803e9298        0x0 /opt/toolchains/n64/mips64-elf/mips64-elf/lib/libc.a(lib_a-fiprintf.o)
 .data          0x00000000803e9298        0x0 /opt/toolchains/n64/mips64-elf/mips64-elf/lib/libc.a(lib_a-fopen.o)
 .data          0x00000000803e9298        0x0 /opt/toolchains/n64/mips64-elf/mips64-elf/lib/libc.a(lib_a-fread.o)
 .data          0x00000000803e9298        0x0 /opt/toolchains/n64/mips64-elf/mips64-elf/lib/libc.a(lib_a-freer.o)
 .data          0x00000000803e9298        0x0 /opt/toolchains/n64/mips64-elf/mips64-elf/lib/libc.a(lib_a-fseek.o)
 .data          0x00000000803e9298        0x0 /opt/toolchains/n64/mips64-elf/mips64-elf/lib/libc.a(lib_a-fstatr.o)
 .data          0x00000000803e9298        0x0 /opt/toolchains/n64/mips64-elf/mips64-elf/lib/libc.a(lib_a-ftell.o)
 .data          0x00000000803e9298        0x0 /opt/toolchains/n64/mips64-elf/mips64-elf/lib/libc.a(lib_a-fwalk.o)
 .data          0x00000000803e9298        0x0 /opt/toolchains/n64/mips64-elf/mips64-elf/lib/libc.a(lib_a-fwrite.o)
 .data          0x00000000803e9298      0x428 /opt/toolchains/n64/mips64-elf/mips64-elf/lib/libc.a(lib_a-impure.o)
 .data          0x00000000803e96c0        0x0 /opt/toolchains/n64/mips64-elf/mips64-elf/lib/libc.a(lib_a-makebuf.o)
 .data          0x00000000803e96c0        0x0 /opt/toolchains/n64/mips64-elf/mips64-elf/lib/libc.a(lib_a-malloc.o)
 .data          0x00000000803e96c0      0x408 /opt/toolchains/n64/mips64-elf/mips64-elf/lib/libc.a(lib_a-mallocr.o)
                0x00000000803e96c0                __malloc_av_
 .data          0x00000000803e9ac8        0x0 /opt/toolchains/n64/mips64-elf/mips64-elf/lib/libc.a(lib_a-memcpy.o)
 .data          0x00000000803e9ac8        0x0 /opt/toolchains/n64/mips64-elf/mips64-elf/lib/libc.a(lib_a-memset.o)
 .data          0x00000000803e9ac8        0x0 /opt/toolchains/n64/mips64-elf/mips64-elf/lib/libc.a(lib_a-mlock.o)
 .data          0x00000000803e9ac8        0x0 /opt/toolchains/n64/mips64-elf/mips64-elf/lib/libc.a(lib_a-openr.o)
 .data          0x00000000803e9ac8        0x0 /opt/toolchains/n64/mips64-elf/mips64-elf/lib/libc.a(lib_a-realloc.o)
 .data          0x00000000803e9ac8        0x0 /opt/toolchains/n64/mips64-elf/mips64-elf/lib/libc.a(lib_a-reallocr.o)
 .data          0x00000000803e9ac8        0x0 /opt/toolchains/n64/mips64-elf/mips64-elf/lib/libc.a(lib_a-reent.o)
 .data          0x00000000803e9ac8        0x0 /opt/toolchains/n64/mips64-elf/mips64-elf/lib/libc.a(lib_a-refill.o)
 .data          0x00000000803e9ac8        0x0 /opt/toolchains/n64/mips64-elf/mips64-elf/lib/libc.a(lib_a-sbrkr.o)
 .data          0x00000000803e9ac8        0x0 /opt/toolchains/n64/mips64-elf/mips64-elf/lib/libc.a(lib_a-sprintf.o)
 .data          0x00000000803e9ac8        0x0 /opt/toolchains/n64/mips64-elf/mips64-elf/lib/libc.a(lib_a-stdio.o)
 .data          0x00000000803e9ac8        0x0 /opt/toolchains/n64/mips64-elf/mips64-elf/lib/libc.a(lib_a-strcmp.o)
 .data          0x00000000803e9ac8        0x0 /opt/toolchains/n64/mips64-elf/mips64-elf/lib/libc.a(lib_a-strcpy.o)
 .data          0x00000000803e9ac8        0x0 /opt/toolchains/n64/mips64-elf/mips64-elf/lib/libc.a(lib_a-strlen.o)
 .data          0x00000000803e9ac8        0x0 /opt/toolchains/n64/mips64-elf/mips64-elf/lib/libc.a(lib_a-svfprintf.o)
 .data          0x00000000803e9ac8        0x0 /opt/toolchains/n64/mips64-elf/mips64-elf/lib/libc.a(lib_a-vfiprintf.o)
 .data          0x00000000803e9ac8        0x0 /opt/toolchains/n64/mips64-elf/mips64-elf/lib/libc.a(lib_a-writer.o)
 .data          0x00000000803e9ac8        0x0 /opt/toolchains/n64/mips64-elf/mips64-elf/lib/libc.a(lib_a-wsetup.o)
 .data          0x00000000803e9ac8        0x0 /opt/toolchains/n64/mips64-elf/mips64-elf/lib/libc.a(lib_a-abort.o)
 .data          0x00000000803e9ac8        0x0 /opt/toolchains/n64/mips64-elf/mips64-elf/lib/libc.a(lib_a-closer.o)
 .data          0x00000000803e9ac8        0x0 /opt/toolchains/n64/mips64-elf/mips64-elf/lib/libc.a(lib_a-dtoa.o)
 .data          0x00000000803e9ac8        0x0 /opt/toolchains/n64/mips64-elf/mips64-elf/lib/libc.a(lib_a-flags.o)
 .data          0x00000000803e9ac8        0x0 /opt/toolchains/n64/mips64-elf/mips64-elf/lib/libc.a(lib_a-fputwc.o)
 .data          0x00000000803e9ac8        0x0 /opt/toolchains/n64/mips64-elf/mips64-elf/lib/libc.a(lib_a-fvwrite.o)
 .data          0x00000000803e9ac8        0x0 /opt/toolchains/n64/mips64-elf/mips64-elf/lib/libc.a(lib_a-isattyr.o)
 .data          0x00000000803e9ac8       0x78 /opt/toolchains/n64/mips64-elf/mips64-elf/lib/libc.a(lib_a-locale.o)
 .data          0x00000000803e9b40        0x0 /opt/toolchains/n64/mips64-elf/mips64-elf/lib/libc.a(lib_a-lseekr.o)
 .data          0x00000000803e9b40        0x0 /opt/toolchains/n64/mips64-elf/mips64-elf/lib/libc.a(lib_a-memchr.o)
 .data          0x00000000803e9b40        0x0 /opt/toolchains/n64/mips64-elf/mips64-elf/lib/libc.a(lib_a-memmove.o)
 .data          0x00000000803e9b40        0x0 /opt/toolchains/n64/mips64-elf/mips64-elf/lib/libc.a(lib_a-mprec.o)
 .data          0x00000000803e9b40        0x0 /opt/toolchains/n64/mips64-elf/mips64-elf/lib/libc.a(lib_a-readr.o)
 .data          0x00000000803e9b40        0x0 /opt/toolchains/n64/mips64-elf/mips64-elf/lib/libc.a(lib_a-signal.o)
 .data          0x00000000803e9b40        0x0 /opt/toolchains/n64/mips64-elf/mips64-elf/lib/libc.a(lib_a-signalr.o)
 .data          0x00000000803e9b40        0x0 /opt/toolchains/n64/mips64-elf/mips64-elf/lib/libc.a(lib_a-svfiprintf.o)
 .data          0x00000000803e9b40        0x0 /opt/toolchains/n64/mips64-elf/mips64-elf/lib/libc.a(lib_a-wbuf.o)
 .data          0x00000000803e9b40        0x0 /opt/toolchains/n64/mips64-elf/mips64-elf/lib/libc.a(lib_a-wcrtomb.o)
 .data          0x00000000803e9b40        0x0 /opt/toolchains/n64/mips64-elf/mips64-elf/lib/libc.a(lib_a-wctomb_r.o)
 .data          0x00000000803e9b40        0x0 /opt/toolchains/n64/mips64-elf/mips64-elf/lib/libc.a(lib_a-callocr.o)
 .data          0x00000000803e9b40        0x8 /opt/toolchains/n64/mips64-elf/lib/libdragonsys.a(system.o)
                0x00000000803e9b40                environ
 .data          0x00000000803e9b48        0x0 /opt/toolchains/n64/mips64-elf/mips64-elf/lib/libnosys.a(_exit.o)
 *(.data.*)
 *(.gnu.linkonce.d.*)
                0x00000000803e9b48                . = ALIGN (0x8)
                0x00000000803f1b48                _gp = (. + 0x8000)
                0x00000000803f1b48                __global = _gp

.lit8
 *(.lit8)

.lit4
 *(.lit4)

.sdata          0x00000000803e9b48      0x2cc load address 0x00000000003e9748
 *(.sdata)
 .sdata         0x00000000803e9b48       0x30 /opt/toolchains/n64/mips64-elf/mips64-elf/lib/libm.a(lib_a-w_pow.o)
 .sdata         0x00000000803e9b78       0xf8 /opt/toolchains/n64/mips64-elf/mips64-elf/lib/libm.a(lib_a-e_pow.o)
 .sdata         0x00000000803e9c70       0x48 /opt/toolchains/n64/mips64-elf/mips64-elf/lib/libm.a(lib_a-e_rem_pio2.o)
 .sdata         0x00000000803e9cb8       0x50 /opt/toolchains/n64/mips64-elf/mips64-elf/lib/libm.a(lib_a-k_cos.o)
 .sdata         0x00000000803e9d08       0x30 /opt/toolchains/n64/mips64-elf/mips64-elf/lib/libm.a(lib_a-k_rem_pio2.o)
 .sdata         0x00000000803e9d38       0x38 /opt/toolchains/n64/mips64-elf/mips64-elf/lib/libm.a(lib_a-k_sin.o)
 .sdata         0x00000000803e9d70        0x8 /opt/toolchains/n64/mips64-elf/mips64-elf/lib/libm.a(lib_a-s_floor.o)
 .sdata         0x00000000803e9d78        0x4 /opt/toolchains/n64/mips64-elf/mips64-elf/lib/libm.a(lib_a-s_lib_ver.o)
                0x00000000803e9d78                __fdlib_version
 *fill*         0x00000000803e9d7c        0x4 00
 .sdata         0x00000000803e9d80       0x20 /opt/toolchains/n64/mips64-elf/mips64-elf/lib/libm.a(lib_a-s_scalbn.o)
 .sdata         0x00000000803e9da0        0x8 /opt/toolchains/n64/mips64-elf/mips64-elf/lib/libc.a(lib_a-impure.o)
                0x00000000803e9da0                _global_impure_ptr
                0x00000000803e9da4                _impure_ptr
 .sdata         0x00000000803e9da8        0x8 /opt/toolchains/n64/mips64-elf/mips64-elf/lib/libc.a(lib_a-mallocr.o)
                0x00000000803e9da8                __malloc_sbrk_base
                0x00000000803e9dac                __malloc_trim_threshold
 .sdata         0x00000000803e9db0       0x48 /opt/toolchains/n64/mips64-elf/mips64-elf/lib/libc.a(lib_a-dtoa.o)
 .sdata         0x00000000803e9df8        0x4 /opt/toolchains/n64/mips64-elf/mips64-elf/lib/libc.a(lib_a-locale.o)
                0x00000000803e9df8                __mb_cur_max
 *fill*         0x00000000803e9dfc        0x4 00
 .sdata         0x00000000803e9e00       0x10 /opt/toolchains/n64/mips64-elf/mips64-elf/lib/libc.a(lib_a-mprec.o)
 .sdata         0x00000000803e9e10        0x4 /opt/toolchains/n64/mips64-elf/mips64-elf/lib/libc.a(lib_a-wctomb_r.o)
                0x00000000803e9e10                __wctomb
 *(.sdata.*)
 *(.gnu.linkonce.s.*)
                0x00000000803e9e18                . = ALIGN (0x8)
                0x00000000803e9e18                __data_end = .

.sbss           0x00000000803e9e18      0x26c load address 0x00000000003e9a18
                0x00000000803e9e18                __bss_start = .
 *(.sbss)
 .sbss          0x00000000803e9e18      0x218 /opt/toolchains/n64/mips64-elf/lib/libdragon.a(inthandler.o)
 .sbss          0x00000000803ea030        0xc /opt/toolchains/n64/mips64-elf/mips64-elf/lib/libc.a(lib_a-mallocr.o)
                0x00000000803ea030                __malloc_max_total_mem
                0x00000000803ea034                __malloc_max_sbrked_mem
                0x00000000803ea038                __malloc_top_pad
 .sbss          0x00000000803ea03c        0xc /opt/toolchains/n64/mips64-elf/mips64-elf/lib/libc.a(lib_a-locale.o)
                0x00000000803ea03c                _PathLocale
                0x00000000803ea040                __mlocale_changed
                0x00000000803ea044                __nlocale_changed
 *(.sbss.*)
 *(.gnu.linkonce.sb.*)
 *(.scommon)
 .scommon       0x00000000803ea048       0x24 main.o
                0x00000000803ea048                gTicks
                0x00000000803ea04c                tv_fps
                0x00000000803ea050                gCursorY
                0x00000000803ea054                buf_size
                0x00000000803ea058                lastticks
                0x00000000803ea060                gCursorX
                0x00000000803ea064                buf_ptr
                0x00000000803ea068                frameticks
 *fill*         0x00000000803ea06c        0x4 00
 .scommon       0x00000000803ea070        0x4 stb_image.o
                0x00000000803ea070                stbi_png_partial
 .scommon       0x00000000803ea074        0xc /opt/toolchains/n64/mips64-elf/lib/libdragon.a(display.o)
                0x00000000803ea074                __width
                0x00000000803ea078                __bitdepth
                0x00000000803ea07c                __height
 .scommon       0x00000000803ea080        0x4 /opt/toolchains/n64/mips64-elf/mips64-elf/lib/libc.a(lib_a-reent.o)
                0x00000000803ea080                errno
 .scommon       0x00000000803ea084        0x0 /opt/toolchains/n64/mips64-elf/lib/libdragonsys.a(system.o)

.bss            0x00000000803ea100    0xa947c load address 0x00000000003e9d00
 *(.bss)
 .bss           0x00000000803ea100       0x18 main.o
                0x00000000803ea100                gButtons
                0x00000000803ea108                dcon
                0x00000000803ea10c                done
 .bss           0x00000000803ea118      0x158 stb_image.o
 .bss           0x00000000803ea270        0x0 ../game/ai/boost.o
 .bss           0x00000000803ea270        0x0 ../game/ai/bullet.o
 .bss           0x00000000803ea270        0x0 ../game/ai/death.o
 .bss           0x00000000803ea270        0x0 ../game/ai/explode.o
 .bss           0x00000000803ea270        0x0 ../game/ai/pickup.o
 .bss           0x00000000803ea270        0x0 ../game/ai/quad.o
 .bss           0x00000000803ea270        0x0 ../game/ai/sheba.o
 .bss           0x00000000803ea270        0x0 ../game/ai/static_model.o
 .bss           0x00000000803ea270        0x0 ../game/ai/static_sprite.o
 .bss           0x00000000803ea270        0x0 ../game/ai/teleporter.o
 .bss           0x00000000803ea270        0x0 ../game/ai/torch.o
 .bss           0x00000000803ea270        0x0 ../game/data.o
 .bss           0x00000000803ea270        0x0 ../game/entities.o
 .bss           0x00000000803ea270       0x10 ../game/game.o
 .bss           0x00000000803ea280        0x0 ../game/maps.o
 .bss           0x00000000803ea280        0x0 ../game/models.o
 .bss           0x00000000803ea280        0x0 ../game/screens.o
 .bss           0x00000000803ea280        0x0 ../game/sprites.o
 .bss           0x00000000803ea280        0x0 ../y3d/y3d_animation.o
 .bss           0x00000000803ea280        0x0 ../y3d/y3d_ansic.o
 .bss           0x00000000803ea280        0x0 ../y3d/y3d_cell.o
 .bss           0x00000000803ea280        0x0 ../y3d/y3d_draw.o
 .bss           0x00000000803ea280        0x0 ../y3d/y3d_engine.o
 .bss           0x00000000803ea280        0x0 ../y3d/y3d_entity.o
 .bss           0x00000000803ea280        0x0 ../y3d/y3d_file.o
 .bss           0x00000000803ea280        0x0 ../y3d/y3d_fixed.o
 .bss           0x00000000803ea280        0x0 ../y3d/y3d_fruity.o
 .bss           0x00000000803ea280        0x0 ../y3d/y3d_image.o
 .bss           0x00000000803ea280        0x0 ../y3d/y3d_keyboard.o
 .bss           0x00000000803ea280        0x0 ../y3d/y3d_map.o
 .bss           0x00000000803ea280        0x0 ../y3d/y3d_matrix.o
 .bss           0x00000000803ea280        0x0 ../y3d/y3d_pixel.o
 .bss           0x00000000803ea280        0x0 ../y3d/y3d_record.o
 .bss           0x00000000803ea280        0x0 ../y3d/y3d_sound.o
 .bss           0x00000000803ea280        0x0 ../y3d/y3d_spanner.o
 .bss           0x00000000803ea280        0x0 ../y3d/y3d_surface.o
 .bss           0x00000000803ea280        0x0 ../y3d/y3d_vertex.o
 .bss           0x00000000803ea280        0x0 ../y3d/y3d_yeti.o
 .bss           0x00000000803ea280        0x0 /opt/toolchains/n64/mips64-elf/mips64-elf/lib/libm.a(lib_a-s_sin.o)
 .bss           0x00000000803ea280        0x0 /opt/toolchains/n64/mips64-elf/mips64-elf/lib/libm.a(lib_a-w_pow.o)
 .bss           0x00000000803ea280        0x0 /opt/toolchains/n64/mips64-elf/mips64-elf/lib/libm.a(lib_a-e_pow.o)
 .bss           0x00000000803ea280        0x0 /opt/toolchains/n64/mips64-elf/mips64-elf/lib/libm.a(lib_a-e_rem_pio2.o)
 .bss           0x00000000803ea280        0x0 /opt/toolchains/n64/mips64-elf/mips64-elf/lib/libm.a(lib_a-e_sqrt.o)
 .bss           0x00000000803ea280        0x0 /opt/toolchains/n64/mips64-elf/mips64-elf/lib/libm.a(lib_a-k_cos.o)
 .bss           0x00000000803ea280        0x0 /opt/toolchains/n64/mips64-elf/mips64-elf/lib/libm.a(lib_a-k_rem_pio2.o)
 .bss           0x00000000803ea280        0x0 /opt/toolchains/n64/mips64-elf/mips64-elf/lib/libm.a(lib_a-k_sin.o)
 .bss           0x00000000803ea280        0x0 /opt/toolchains/n64/mips64-elf/mips64-elf/lib/libm.a(lib_a-s_fabs.o)
 .bss           0x00000000803ea280        0x0 /opt/toolchains/n64/mips64-elf/mips64-elf/lib/libm.a(lib_a-s_finite.o)
 .bss           0x00000000803ea280        0x0 /opt/toolchains/n64/mips64-elf/mips64-elf/lib/libm.a(lib_a-s_floor.o)
 .bss           0x00000000803ea280        0x0 /opt/toolchains/n64/mips64-elf/mips64-elf/lib/libm.a(lib_a-s_fpclassify.o)
 .bss           0x00000000803ea280        0x0 /opt/toolchains/n64/mips64-elf/mips64-elf/lib/libm.a(lib_a-s_lib_ver.o)
 .bss           0x00000000803ea280        0x0 /opt/toolchains/n64/mips64-elf/mips64-elf/lib/libm.a(lib_a-s_matherr.o)
 .bss           0x00000000803ea280        0x0 /opt/toolchains/n64/mips64-elf/mips64-elf/lib/libm.a(lib_a-s_nan.o)
 .bss           0x00000000803ea280        0x0 /opt/toolchains/n64/mips64-elf/mips64-elf/lib/libm.a(lib_a-s_rint.o)
 .bss           0x00000000803ea280        0x0 /opt/toolchains/n64/mips64-elf/mips64-elf/lib/libm.a(lib_a-s_scalbn.o)
 .bss           0x00000000803ea280        0x0 /opt/toolchains/n64/mips64-elf/mips64-elf/lib/libm.a(lib_a-s_copysign.o)
 .bss           0x00000000803ea280        0x0 /opt/toolchains/n64/mips64-elf/lib/libdragon.a(n64sys.o)
 .bss           0x00000000803ea280       0x1c /opt/toolchains/n64/mips64-elf/lib/libdragon.a(interrupt.o)
                0x00000000803ea280                SP_callback
                0x00000000803ea284                SI_callback
                0x00000000803ea288                TI_callback
                0x00000000803ea28c                DP_callback
                0x00000000803ea290                PI_callback
                0x00000000803ea294                VI_callback
                0x00000000803ea298                AI_callback
 .bss           0x00000000803ea29c        0x0 /opt/toolchains/n64/mips64-elf/lib/libdragon.a(entrypoint.o)
 *fill*         0x00000000803ea29c        0x4 00
 .bss           0x00000000803ea2a0      0x9a0 /opt/toolchains/n64/mips64-elf/lib/libdragon.a(dragonfs.o)
 .bss           0x00000000803eac40       0x18 /opt/toolchains/n64/mips64-elf/lib/libdragon.a(audio.o)
 .bss           0x00000000803eac58       0x10 /opt/toolchains/n64/mips64-elf/lib/libdragon.a(display.o)
 .bss           0x00000000803eac68      0x200 /opt/toolchains/n64/mips64-elf/lib/libdragon.a(controller.o)
 .bss           0x00000000803eae68        0x4 /opt/toolchains/n64/mips64-elf/lib/libdragon.a(graphics.o)
 *fill*         0x00000000803eae6c        0x4 00
 .bss           0x00000000803eae70     0x1090 /opt/toolchains/n64/mips64-elf/lib/libdragon.a(rdp.o)
 .bss           0x00000000803ebf00        0x0 /opt/toolchains/n64/mips64-elf/lib/libdragon.a(dma.o)
 .bss           0x00000000803ebf00       0x10 /opt/toolchains/n64/mips64-elf/lib/libdragon.a(timer.o)
 *fill*         0x00000000803ebf10       0xf0 00
 .bss           0x00000000803ec000    0x10500 /opt/toolchains/n64/mips64-elf/lib/libdragon.a(inthandler.o)
                0x00000000803ec100                __baseRegAddr
 .bss           0x00000000803fc500        0x4 /opt/toolchains/n64/mips64-elf/lib/libdragon.a(exception.o)
 .bss           0x00000000803fc504        0x0 /opt/toolchains/n64/mips64-elf/mips64-elf/lib/libc.a(lib_a-assert.o)
 .bss           0x00000000803fc504        0x0 /opt/toolchains/n64/mips64-elf/mips64-elf/lib/libc.a(lib_a-errno.o)
 .bss           0x00000000803fc504        0x0 /opt/toolchains/n64/mips64-elf/mips64-elf/lib/libc.a(lib_a-fclose.o)
 .bss           0x00000000803fc504        0x0 /opt/toolchains/n64/mips64-elf/mips64-elf/lib/libc.a(lib_a-fflush.o)
 .bss           0x00000000803fc504        0x0 /opt/toolchains/n64/mips64-elf/mips64-elf/lib/libc.a(lib_a-findfp.o)
 .bss           0x00000000803fc504        0x0 /opt/toolchains/n64/mips64-elf/mips64-elf/lib/libc.a(lib_a-fiprintf.o)
 .bss           0x00000000803fc504        0x0 /opt/toolchains/n64/mips64-elf/mips64-elf/lib/libc.a(lib_a-fopen.o)
 .bss           0x00000000803fc504        0x0 /opt/toolchains/n64/mips64-elf/mips64-elf/lib/libc.a(lib_a-fread.o)
 .bss           0x00000000803fc504        0x0 /opt/toolchains/n64/mips64-elf/mips64-elf/lib/libc.a(lib_a-freer.o)
 .bss           0x00000000803fc504        0x0 /opt/toolchains/n64/mips64-elf/mips64-elf/lib/libc.a(lib_a-fseek.o)
 .bss           0x00000000803fc504        0x0 /opt/toolchains/n64/mips64-elf/mips64-elf/lib/libc.a(lib_a-fstatr.o)
 .bss           0x00000000803fc504        0x0 /opt/toolchains/n64/mips64-elf/mips64-elf/lib/libc.a(lib_a-ftell.o)
 .bss           0x00000000803fc504        0x0 /opt/toolchains/n64/mips64-elf/mips64-elf/lib/libc.a(lib_a-fwalk.o)
 .bss           0x00000000803fc504        0x0 /opt/toolchains/n64/mips64-elf/mips64-elf/lib/libc.a(lib_a-fwrite.o)
 .bss           0x00000000803fc504        0x0 /opt/toolchains/n64/mips64-elf/mips64-elf/lib/libc.a(lib_a-impure.o)
 .bss           0x00000000803fc504        0x0 /opt/toolchains/n64/mips64-elf/mips64-elf/lib/libc.a(lib_a-makebuf.o)
 .bss           0x00000000803fc504        0x0 /opt/toolchains/n64/mips64-elf/mips64-elf/lib/libc.a(lib_a-malloc.o)
 *fill*         0x00000000803fc504        0x4 00
 .bss           0x00000000803fc508       0x28 /opt/toolchains/n64/mips64-elf/mips64-elf/lib/libc.a(lib_a-mallocr.o)
                0x00000000803fc508                __malloc_current_mallinfo
 .bss           0x00000000803fc530        0x0 /opt/toolchains/n64/mips64-elf/mips64-elf/lib/libc.a(lib_a-memcpy.o)
 .bss           0x00000000803fc530        0x0 /opt/toolchains/n64/mips64-elf/mips64-elf/lib/libc.a(lib_a-memset.o)
 .bss           0x00000000803fc530        0x0 /opt/toolchains/n64/mips64-elf/mips64-elf/lib/libc.a(lib_a-mlock.o)
 .bss           0x00000000803fc530        0x0 /opt/toolchains/n64/mips64-elf/mips64-elf/lib/libc.a(lib_a-openr.o)
 .bss           0x00000000803fc530        0x0 /opt/toolchains/n64/mips64-elf/mips64-elf/lib/libc.a(lib_a-realloc.o)
 .bss           0x00000000803fc530        0x0 /opt/toolchains/n64/mips64-elf/mips64-elf/lib/libc.a(lib_a-reallocr.o)
 .bss           0x00000000803fc530        0x0 /opt/toolchains/n64/mips64-elf/mips64-elf/lib/libc.a(lib_a-reent.o)
 .bss           0x00000000803fc530        0x0 /opt/toolchains/n64/mips64-elf/mips64-elf/lib/libc.a(lib_a-refill.o)
 .bss           0x00000000803fc530        0x0 /opt/toolchains/n64/mips64-elf/mips64-elf/lib/libc.a(lib_a-sbrkr.o)
 .bss           0x00000000803fc530        0x0 /opt/toolchains/n64/mips64-elf/mips64-elf/lib/libc.a(lib_a-sprintf.o)
 .bss           0x00000000803fc530        0x0 /opt/toolchains/n64/mips64-elf/mips64-elf/lib/libc.a(lib_a-stdio.o)
 .bss           0x00000000803fc530        0x0 /opt/toolchains/n64/mips64-elf/mips64-elf/lib/libc.a(lib_a-strcmp.o)
 .bss           0x00000000803fc530        0x0 /opt/toolchains/n64/mips64-elf/mips64-elf/lib/libc.a(lib_a-strcpy.o)
 .bss           0x00000000803fc530        0x0 /opt/toolchains/n64/mips64-elf/mips64-elf/lib/libc.a(lib_a-strlen.o)
 .bss           0x00000000803fc530        0x0 /opt/toolchains/n64/mips64-elf/mips64-elf/lib/libc.a(lib_a-svfprintf.o)
 .bss           0x00000000803fc530        0x0 /opt/toolchains/n64/mips64-elf/mips64-elf/lib/libc.a(lib_a-vfiprintf.o)
 .bss           0x00000000803fc530        0x0 /opt/toolchains/n64/mips64-elf/mips64-elf/lib/libc.a(lib_a-writer.o)
 .bss           0x00000000803fc530        0x0 /opt/toolchains/n64/mips64-elf/mips64-elf/lib/libc.a(lib_a-wsetup.o)
 .bss           0x00000000803fc530        0x0 /opt/toolchains/n64/mips64-elf/mips64-elf/lib/libc.a(lib_a-abort.o)
 .bss           0x00000000803fc530        0x0 /opt/toolchains/n64/mips64-elf/mips64-elf/lib/libc.a(lib_a-closer.o)
 .bss           0x00000000803fc530        0x0 /opt/toolchains/n64/mips64-elf/mips64-elf/lib/libc.a(lib_a-dtoa.o)
 .bss           0x00000000803fc530        0x0 /opt/toolchains/n64/mips64-elf/mips64-elf/lib/libc.a(lib_a-flags.o)
 .bss           0x00000000803fc530        0x0 /opt/toolchains/n64/mips64-elf/mips64-elf/lib/libc.a(lib_a-fputwc.o)
 .bss           0x00000000803fc530        0x0 /opt/toolchains/n64/mips64-elf/mips64-elf/lib/libc.a(lib_a-fvwrite.o)
 .bss           0x00000000803fc530        0x0 /opt/toolchains/n64/mips64-elf/mips64-elf/lib/libc.a(lib_a-isattyr.o)
 .bss           0x00000000803fc530        0x0 /opt/toolchains/n64/mips64-elf/mips64-elf/lib/libc.a(lib_a-locale.o)
 .bss           0x00000000803fc530        0x0 /opt/toolchains/n64/mips64-elf/mips64-elf/lib/libc.a(lib_a-lseekr.o)
 .bss           0x00000000803fc530        0x0 /opt/toolchains/n64/mips64-elf/mips64-elf/lib/libc.a(lib_a-memchr.o)
 .bss           0x00000000803fc530        0x0 /opt/toolchains/n64/mips64-elf/mips64-elf/lib/libc.a(lib_a-memmove.o)
 .bss           0x00000000803fc530        0x0 /opt/toolchains/n64/mips64-elf/mips64-elf/lib/libc.a(lib_a-mprec.o)
 .bss           0x00000000803fc530        0x0 /opt/toolchains/n64/mips64-elf/mips64-elf/lib/libc.a(lib_a-readr.o)
 .bss           0x00000000803fc530        0x0 /opt/toolchains/n64/mips64-elf/mips64-elf/lib/libc.a(lib_a-signal.o)
 .bss           0x00000000803fc530        0x0 /opt/toolchains/n64/mips64-elf/mips64-elf/lib/libc.a(lib_a-signalr.o)
 .bss           0x00000000803fc530        0x0 /opt/toolchains/n64/mips64-elf/mips64-elf/lib/libc.a(lib_a-svfiprintf.o)
 .bss           0x00000000803fc530        0x0 /opt/toolchains/n64/mips64-elf/mips64-elf/lib/libc.a(lib_a-wbuf.o)
 .bss           0x00000000803fc530        0x0 /opt/toolchains/n64/mips64-elf/mips64-elf/lib/libc.a(lib_a-wcrtomb.o)
 .bss           0x00000000803fc530        0x0 /opt/toolchains/n64/mips64-elf/mips64-elf/lib/libc.a(lib_a-wctomb_r.o)
 .bss           0x00000000803fc530        0x0 /opt/toolchains/n64/mips64-elf/mips64-elf/lib/libc.a(lib_a-callocr.o)
 .bss           0x00000000803fc530      0x520 /opt/toolchains/n64/mips64-elf/lib/libdragonsys.a(system.o)
                0x00000000803fc530                __env
 .bss           0x00000000803fca50        0x0 /opt/toolchains/n64/mips64-elf/mips64-elf/lib/libnosys.a(_exit.o)
 *(.bss.*)
 *(.gnu.linkonce.b.*)
 *(COMMON)
 COMMON         0x00000000803fca50    0x84b20 main.o
                0x00000000803fca50                yeti
                0x0000000080471450                gKeys
                0x00000000804714f0                yetiMap
 COMMON         0x0000000080481570    0x12000 ../y3d/y3d_fixed.o
                0x0000000080481570                sintable
                0x0000000080483570                reciprocal
 COMMON         0x0000000080493570        0xc /opt/toolchains/n64/mips64-elf/lib/libdragon.a(display.o)
                0x0000000080493570                __safe_buffer
                0x000000008049357c                end = .
                0x0000000080493580                _end = ALIGN (0x10)
                0x0000000080493580                __end = _end
                0x000000008049357c                __bss_end = .
LOAD /opt/toolchains/n64/mips64-elf/mips64-elf/lib/libm.a
LOAD /opt/toolchains/n64/mips64-elf/lib/libdragon.a
LOAD /opt/toolchains/n64/mips64-elf/mips64-elf/lib/libc.a
LOAD /opt/toolchains/n64/mips64-elf/lib/libdragonsys.a
LOAD /opt/toolchains/n64/mips64-elf/mips64-elf/lib/libnosys.a
OUTPUT(Yeti3D_Pro.elf elf32-bigmips)

.reginfo        0x0000000000000000       0x18
 .reginfo       0x0000000000000000       0x18 main.o

.pdr            0x0000000000000000     0x4be0
 .pdr           0x0000000000000000      0x2a0 main.o
 .pdr           0x00000000000002a0      0x740 stb_image.o
 .pdr           0x00000000000009e0       0x60 ../game/ai/boost.o
 .pdr           0x0000000000000a40       0xa0 ../game/ai/bullet.o
 .pdr           0x0000000000000ae0       0x40 ../game/ai/death.o
 .pdr           0x0000000000000b20       0x80 ../game/ai/explode.o
 .pdr           0x0000000000000ba0       0x20 ../game/ai/pickup.o
 .pdr           0x0000000000000bc0       0x60 ../game/ai/quad.o
 .pdr           0x0000000000000c20       0x40 ../game/ai/sheba.o
 .pdr           0x0000000000000c60        0x0 ../game/ai/static_model.o
 .pdr           0x0000000000000c60        0x0 ../game/ai/static_sprite.o
 .pdr           0x0000000000000c60       0x40 ../game/ai/teleporter.o
 .pdr           0x0000000000000ca0       0x80 ../game/ai/torch.o
 .pdr           0x0000000000000d20        0x0 ../game/data.o
 .pdr           0x0000000000000d20      0x180 ../game/entities.o
 .pdr           0x0000000000000ea0      0x420 ../game/game.o
 .pdr           0x00000000000012c0        0x0 ../game/maps.o
 .pdr           0x00000000000012c0        0x0 ../game/models.o
 .pdr           0x00000000000012c0      0x220 ../game/screens.o
 .pdr           0x00000000000014e0        0x0 ../game/sprites.o
 .pdr           0x00000000000014e0       0xa0 ../y3d/y3d_animation.o
 .pdr           0x0000000000001580       0x80 ../y3d/y3d_ansic.o
 .pdr           0x0000000000001600       0x40 ../y3d/y3d_cell.o
 .pdr           0x0000000000001640      0x180 ../y3d/y3d_draw.o
 .pdr           0x00000000000017c0      0x120 ../y3d/y3d_engine.o
 .pdr           0x00000000000018e0      0x220 ../y3d/y3d_entity.o
 .pdr           0x0000000000001b00       0x20 ../y3d/y3d_file.o
 .pdr           0x0000000000001b20       0x40 ../y3d/y3d_fixed.o
 .pdr           0x0000000000001b60       0x40 ../y3d/y3d_fruity.o
 .pdr           0x0000000000001ba0       0x60 ../y3d/y3d_image.o
 .pdr           0x0000000000001c00       0x40 ../y3d/y3d_keyboard.o
 .pdr           0x0000000000001c40      0x1e0 ../y3d/y3d_map.o
 .pdr           0x0000000000001e20       0x60 ../y3d/y3d_matrix.o
 .pdr           0x0000000000001e80      0x100 ../y3d/y3d_pixel.o
 .pdr           0x0000000000001f80       0xe0 ../y3d/y3d_record.o
 .pdr           0x0000000000002060        0x0 ../y3d/y3d_sound.o
 .pdr           0x0000000000002060       0x80 ../y3d/y3d_spanner.o
 .pdr           0x00000000000020e0       0x40 ../y3d/y3d_surface.o
 .pdr           0x0000000000002120       0x20 ../y3d/y3d_vertex.o
 .pdr           0x0000000000002140      0x160 ../y3d/y3d_yeti.o
 .pdr           0x00000000000022a0       0x20 /opt/toolchains/n64/mips64-elf/mips64-elf/lib/libm.a(lib_a-s_sin.o)
 .pdr           0x00000000000022c0       0x20 /opt/toolchains/n64/mips64-elf/mips64-elf/lib/libm.a(lib_a-w_pow.o)
 .pdr           0x00000000000022e0       0x20 /opt/toolchains/n64/mips64-elf/mips64-elf/lib/libm.a(lib_a-e_pow.o)
 .pdr           0x0000000000002300       0x20 /opt/toolchains/n64/mips64-elf/mips64-elf/lib/libm.a(lib_a-e_rem_pio2.o)
 .pdr           0x0000000000002320       0x20 /opt/toolchains/n64/mips64-elf/mips64-elf/lib/libm.a(lib_a-e_sqrt.o)
 .pdr           0x0000000000002340       0x20 /opt/toolchains/n64/mips64-elf/mips64-elf/lib/libm.a(lib_a-k_cos.o)
 .pdr           0x0000000000002360       0x20 /opt/toolchains/n64/mips64-elf/mips64-elf/lib/libm.a(lib_a-k_rem_pio2.o)
 .pdr           0x0000000000002380       0x20 /opt/toolchains/n64/mips64-elf/mips64-elf/lib/libm.a(lib_a-k_sin.o)
 .pdr           0x00000000000023a0       0x20 /opt/toolchains/n64/mips64-elf/mips64-elf/lib/libm.a(lib_a-s_fabs.o)
 .pdr           0x00000000000023c0       0x20 /opt/toolchains/n64/mips64-elf/mips64-elf/lib/libm.a(lib_a-s_finite.o)
 .pdr           0x00000000000023e0       0x20 /opt/toolchains/n64/mips64-elf/mips64-elf/lib/libm.a(lib_a-s_floor.o)
 .pdr           0x0000000000002400       0x20 /opt/toolchains/n64/mips64-elf/mips64-elf/lib/libm.a(lib_a-s_fpclassify.o)
 .pdr           0x0000000000002420        0x0 /opt/toolchains/n64/mips64-elf/mips64-elf/lib/libm.a(lib_a-s_lib_ver.o)
 .pdr           0x0000000000002420       0x20 /opt/toolchains/n64/mips64-elf/mips64-elf/lib/libm.a(lib_a-s_matherr.o)
 .pdr           0x0000000000002440       0x20 /opt/toolchains/n64/mips64-elf/mips64-elf/lib/libm.a(lib_a-s_nan.o)
 .pdr           0x0000000000002460       0x20 /opt/toolchains/n64/mips64-elf/mips64-elf/lib/libm.a(lib_a-s_rint.o)
 .pdr           0x0000000000002480       0x20 /opt/toolchains/n64/mips64-elf/mips64-elf/lib/libm.a(lib_a-s_scalbn.o)
 .pdr           0x00000000000024a0       0x20 /opt/toolchains/n64/mips64-elf/mips64-elf/lib/libm.a(lib_a-s_copysign.o)
 .pdr           0x00000000000024c0      0x1a0 /opt/toolchains/n64/mips64-elf/lib/libdragon.a(n64sys.o)
 .pdr           0x0000000000002660      0x380 /opt/toolchains/n64/mips64-elf/lib/libdragon.a(interrupt.o)
 .pdr           0x00000000000029e0        0x0 /opt/toolchains/n64/mips64-elf/lib/libdragon.a(entrypoint.o)
 .pdr           0x00000000000029e0      0x2a0 /opt/toolchains/n64/mips64-elf/lib/libdragon.a(dragonfs.o)
 .pdr           0x0000000000002c80      0x100 /opt/toolchains/n64/mips64-elf/lib/libdragon.a(audio.o)
 .pdr           0x0000000000002d80       0xa0 /opt/toolchains/n64/mips64-elf/lib/libdragon.a(display.o)
 .pdr           0x0000000000002e20      0x2a0 /opt/toolchains/n64/mips64-elf/lib/libdragon.a(controller.o)
 .pdr           0x00000000000030c0      0x200 /opt/toolchains/n64/mips64-elf/lib/libdragon.a(graphics.o)
 .pdr           0x00000000000032c0      0x2c0 /opt/toolchains/n64/mips64-elf/lib/libdragon.a(rdp.o)
 .pdr           0x0000000000003580       0xa0 /opt/toolchains/n64/mips64-elf/lib/libdragon.a(dma.o)
 .pdr           0x0000000000003620      0x100 /opt/toolchains/n64/mips64-elf/lib/libdragon.a(timer.o)
 .pdr           0x0000000000003720        0x0 /opt/toolchains/n64/mips64-elf/lib/libdragon.a(inthandler.o)
 .pdr           0x0000000000003720       0x60 /opt/toolchains/n64/mips64-elf/lib/libdragon.a(exception.o)
 .pdr           0x0000000000003780       0x40 /opt/toolchains/n64/mips64-elf/mips64-elf/lib/libc.a(lib_a-assert.o)
 .pdr           0x00000000000037c0       0x20 /opt/toolchains/n64/mips64-elf/mips64-elf/lib/libc.a(lib_a-errno.o)
 .pdr           0x00000000000037e0       0x40 /opt/toolchains/n64/mips64-elf/mips64-elf/lib/libc.a(lib_a-fclose.o)
 .pdr           0x0000000000003820       0x60 /opt/toolchains/n64/mips64-elf/mips64-elf/lib/libc.a(lib_a-fflush.o)
 .pdr           0x0000000000003880      0x1c0 /opt/toolchains/n64/mips64-elf/mips64-elf/lib/libc.a(lib_a-findfp.o)
 .pdr           0x0000000000003a40       0x40 /opt/toolchains/n64/mips64-elf/mips64-elf/lib/libc.a(lib_a-fiprintf.o)
 .pdr           0x0000000000003a80       0x40 /opt/toolchains/n64/mips64-elf/mips64-elf/lib/libc.a(lib_a-fopen.o)
 .pdr           0x0000000000003ac0       0x40 /opt/toolchains/n64/mips64-elf/mips64-elf/lib/libc.a(lib_a-fread.o)
 .pdr           0x0000000000003b00       0x40 /opt/toolchains/n64/mips64-elf/mips64-elf/lib/libc.a(lib_a-freer.o)
 .pdr           0x0000000000003b40       0x40 /opt/toolchains/n64/mips64-elf/mips64-elf/lib/libc.a(lib_a-fseek.o)
 .pdr           0x0000000000003b80       0x20 /opt/toolchains/n64/mips64-elf/mips64-elf/lib/libc.a(lib_a-fstatr.o)
 .pdr           0x0000000000003ba0       0x40 /opt/toolchains/n64/mips64-elf/mips64-elf/lib/libc.a(lib_a-ftell.o)
 .pdr           0x0000000000003be0       0x40 /opt/toolchains/n64/mips64-elf/mips64-elf/lib/libc.a(lib_a-fwalk.o)
 .pdr           0x0000000000003c20       0x40 /opt/toolchains/n64/mips64-elf/mips64-elf/lib/libc.a(lib_a-fwrite.o)
 .pdr           0x0000000000003c60        0x0 /opt/toolchains/n64/mips64-elf/mips64-elf/lib/libc.a(lib_a-impure.o)
 .pdr           0x0000000000003c60       0x20 /opt/toolchains/n64/mips64-elf/mips64-elf/lib/libc.a(lib_a-makebuf.o)
 .pdr           0x0000000000003c80       0x40 /opt/toolchains/n64/mips64-elf/mips64-elf/lib/libc.a(lib_a-malloc.o)
 .pdr           0x0000000000003cc0       0x20 /opt/toolchains/n64/mips64-elf/mips64-elf/lib/libc.a(lib_a-mallocr.o)
 .pdr           0x0000000000003ce0       0x20 /opt/toolchains/n64/mips64-elf/mips64-elf/lib/libc.a(lib_a-memcpy.o)
 .pdr           0x0000000000003d00       0x20 /opt/toolchains/n64/mips64-elf/mips64-elf/lib/libc.a(lib_a-memset.o)
 .pdr           0x0000000000003d20       0x40 /opt/toolchains/n64/mips64-elf/mips64-elf/lib/libc.a(lib_a-mlock.o)
 .pdr           0x0000000000003d60       0x20 /opt/toolchains/n64/mips64-elf/mips64-elf/lib/libc.a(lib_a-openr.o)
 .pdr           0x0000000000003d80       0x20 /opt/toolchains/n64/mips64-elf/mips64-elf/lib/libc.a(lib_a-realloc.o)
 .pdr           0x0000000000003da0       0x20 /opt/toolchains/n64/mips64-elf/mips64-elf/lib/libc.a(lib_a-reallocr.o)
 .pdr           0x0000000000003dc0       0x60 /opt/toolchains/n64/mips64-elf/mips64-elf/lib/libc.a(lib_a-reent.o)
 .pdr           0x0000000000003e20       0x40 /opt/toolchains/n64/mips64-elf/mips64-elf/lib/libc.a(lib_a-refill.o)
 .pdr           0x0000000000003e60       0x20 /opt/toolchains/n64/mips64-elf/mips64-elf/lib/libc.a(lib_a-sbrkr.o)
 .pdr           0x0000000000003e80       0x40 /opt/toolchains/n64/mips64-elf/mips64-elf/lib/libc.a(lib_a-sprintf.o)
 .pdr           0x0000000000003ec0       0xa0 /opt/toolchains/n64/mips64-elf/mips64-elf/lib/libc.a(lib_a-stdio.o)
 .pdr           0x0000000000003f60       0x20 /opt/toolchains/n64/mips64-elf/mips64-elf/lib/libc.a(lib_a-strcmp.o)
 .pdr           0x0000000000003f80       0x20 /opt/toolchains/n64/mips64-elf/mips64-elf/lib/libc.a(lib_a-strcpy.o)
 .pdr           0x0000000000003fa0       0x20 /opt/toolchains/n64/mips64-elf/mips64-elf/lib/libc.a(lib_a-strlen.o)
 .pdr           0x0000000000003fc0       0x20 /opt/toolchains/n64/mips64-elf/mips64-elf/lib/libc.a(lib_a-svfprintf.o)
 .pdr           0x0000000000003fe0       0x60 /opt/toolchains/n64/mips64-elf/mips64-elf/lib/libc.a(lib_a-vfiprintf.o)
 .pdr           0x0000000000004040       0x20 /opt/toolchains/n64/mips64-elf/mips64-elf/lib/libc.a(lib_a-writer.o)
 .pdr           0x0000000000004060       0x20 /opt/toolchains/n64/mips64-elf/mips64-elf/lib/libc.a(lib_a-wsetup.o)
 .pdr           0x0000000000004080       0x20 /opt/toolchains/n64/mips64-elf/mips64-elf/lib/libc.a(lib_a-abort.o)
 .pdr           0x00000000000040a0       0x20 /opt/toolchains/n64/mips64-elf/mips64-elf/lib/libc.a(lib_a-closer.o)
 .pdr           0x00000000000040c0       0x40 /opt/toolchains/n64/mips64-elf/mips64-elf/lib/libc.a(lib_a-dtoa.o)
 .pdr           0x0000000000004100       0x20 /opt/toolchains/n64/mips64-elf/mips64-elf/lib/libc.a(lib_a-flags.o)
 .pdr           0x0000000000004120       0x40 /opt/toolchains/n64/mips64-elf/mips64-elf/lib/libc.a(lib_a-fputwc.o)
 .pdr           0x0000000000004160       0x20 /opt/toolchains/n64/mips64-elf/mips64-elf/lib/libc.a(lib_a-fvwrite.o)
 .pdr           0x0000000000004180       0x20 /opt/toolchains/n64/mips64-elf/mips64-elf/lib/libc.a(lib_a-isattyr.o)
 .pdr           0x00000000000041a0      0x100 /opt/toolchains/n64/mips64-elf/mips64-elf/lib/libc.a(lib_a-locale.o)
 .pdr           0x00000000000042a0       0x20 /opt/toolchains/n64/mips64-elf/mips64-elf/lib/libc.a(lib_a-lseekr.o)
 .pdr           0x00000000000042c0       0x20 /opt/toolchains/n64/mips64-elf/mips64-elf/lib/libc.a(lib_a-memchr.o)
 .pdr           0x00000000000042e0       0x20 /opt/toolchains/n64/mips64-elf/mips64-elf/lib/libc.a(lib_a-memmove.o)
 .pdr           0x0000000000004300      0x260 /opt/toolchains/n64/mips64-elf/mips64-elf/lib/libc.a(lib_a-mprec.o)
 .pdr           0x0000000000004560       0x20 /opt/toolchains/n64/mips64-elf/mips64-elf/lib/libc.a(lib_a-readr.o)
 .pdr           0x0000000000004580      0x100 /opt/toolchains/n64/mips64-elf/mips64-elf/lib/libc.a(lib_a-signal.o)
 .pdr           0x0000000000004680       0x40 /opt/toolchains/n64/mips64-elf/mips64-elf/lib/libc.a(lib_a-signalr.o)
 .pdr           0x00000000000046c0       0x40 /opt/toolchains/n64/mips64-elf/mips64-elf/lib/libc.a(lib_a-svfiprintf.o)
 .pdr           0x0000000000004700       0x40 /opt/toolchains/n64/mips64-elf/mips64-elf/lib/libc.a(lib_a-wbuf.o)
 .pdr           0x0000000000004740       0x40 /opt/toolchains/n64/mips64-elf/mips64-elf/lib/libc.a(lib_a-wcrtomb.o)
 .pdr           0x0000000000004780       0x40 /opt/toolchains/n64/mips64-elf/mips64-elf/lib/libc.a(lib_a-wctomb_r.o)
 .pdr           0x00000000000047c0       0x20 /opt/toolchains/n64/mips64-elf/mips64-elf/lib/libc.a(lib_a-callocr.o)
 .pdr           0x00000000000047e0      0x3e0 /opt/toolchains/n64/mips64-elf/lib/libdragonsys.a(system.o)
 .pdr           0x0000000000004bc0       0x20 /opt/toolchains/n64/mips64-elf/mips64-elf/lib/libnosys.a(_exit.o)

.mdebug.abiO64  0x0000000000000000        0x0
 .mdebug.abiO64
                0x0000000000000000        0x0 main.o
 .mdebug.abiO64
                0x0000000000000000        0x0 stb_image.o
 .mdebug.abiO64
                0x0000000000000000        0x0 ../game/ai/boost.o
 .mdebug.abiO64
                0x0000000000000000        0x0 ../game/ai/bullet.o
 .mdebug.abiO64
                0x0000000000000000        0x0 ../game/ai/death.o
 .mdebug.abiO64
                0x0000000000000000        0x0 ../game/ai/explode.o
 .mdebug.abiO64
                0x0000000000000000        0x0 ../game/ai/pickup.o
 .mdebug.abiO64
                0x0000000000000000        0x0 ../game/ai/quad.o
 .mdebug.abiO64
                0x0000000000000000        0x0 ../game/ai/sheba.o
 .mdebug.abiO64
                0x0000000000000000        0x0 ../game/ai/static_model.o
 .mdebug.abiO64
                0x0000000000000000        0x0 ../game/ai/static_sprite.o
 .mdebug.abiO64
                0x0000000000000000        0x0 ../game/ai/teleporter.o
 .mdebug.abiO64
                0x0000000000000000        0x0 ../game/ai/torch.o
 .mdebug.abiO64
                0x0000000000000000        0x0 ../game/data.o
 .mdebug.abiO64
                0x0000000000000000        0x0 ../game/entities.o
 .mdebug.abiO64
                0x0000000000000000        0x0 ../game/game.o
 .mdebug.abiO64
                0x0000000000000000        0x0 ../game/maps.o
 .mdebug.abiO64
                0x0000000000000000        0x0 ../game/models.o
 .mdebug.abiO64
                0x0000000000000000        0x0 ../game/screens.o
 .mdebug.abiO64
                0x0000000000000000        0x0 ../game/sprites.o
 .mdebug.abiO64
                0x0000000000000000        0x0 ../y3d/y3d_animation.o
 .mdebug.abiO64
                0x0000000000000000        0x0 ../y3d/y3d_ansic.o
 .mdebug.abiO64
                0x0000000000000000        0x0 ../y3d/y3d_cell.o
 .mdebug.abiO64
                0x0000000000000000        0x0 ../y3d/y3d_draw.o
 .mdebug.abiO64
                0x0000000000000000        0x0 ../y3d/y3d_engine.o
 .mdebug.abiO64
                0x0000000000000000        0x0 ../y3d/y3d_entity.o
 .mdebug.abiO64
                0x0000000000000000        0x0 ../y3d/y3d_file.o
 .mdebug.abiO64
                0x0000000000000000        0x0 ../y3d/y3d_fixed.o
 .mdebug.abiO64
                0x0000000000000000        0x0 ../y3d/y3d_fruity.o
 .mdebug.abiO64
                0x0000000000000000        0x0 ../y3d/y3d_image.o
 .mdebug.abiO64
                0x0000000000000000        0x0 ../y3d/y3d_keyboard.o
 .mdebug.abiO64
                0x0000000000000000        0x0 ../y3d/y3d_map.o
 .mdebug.abiO64
                0x0000000000000000        0x0 ../y3d/y3d_matrix.o
 .mdebug.abiO64
                0x0000000000000000        0x0 ../y3d/y3d_pixel.o
 .mdebug.abiO64
                0x0000000000000000        0x0 ../y3d/y3d_record.o
 .mdebug.abiO64
                0x0000000000000000        0x0 ../y3d/y3d_sound.o
 .mdebug.abiO64
                0x0000000000000000        0x0 ../y3d/y3d_spanner.o
 .mdebug.abiO64
                0x0000000000000000        0x0 ../y3d/y3d_surface.o
 .mdebug.abiO64
                0x0000000000000000        0x0 ../y3d/y3d_vertex.o
 .mdebug.abiO64
                0x0000000000000000        0x0 ../y3d/y3d_yeti.o
 .mdebug.abiO64
                0x0000000000000000        0x0 /opt/toolchains/n64/mips64-elf/mips64-elf/lib/libm.a(lib_a-s_sin.o)
 .mdebug.abiO64
                0x0000000000000000        0x0 /opt/toolchains/n64/mips64-elf/mips64-elf/lib/libm.a(lib_a-w_pow.o)
 .mdebug.abiO64
                0x0000000000000000        0x0 /opt/toolchains/n64/mips64-elf/mips64-elf/lib/libm.a(lib_a-e_pow.o)
 .mdebug.abiO64
                0x0000000000000000        0x0 /opt/toolchains/n64/mips64-elf/mips64-elf/lib/libm.a(lib_a-e_rem_pio2.o)
 .mdebug.abiO64
                0x0000000000000000        0x0 /opt/toolchains/n64/mips64-elf/mips64-elf/lib/libm.a(lib_a-e_sqrt.o)
 .mdebug.abiO64
                0x0000000000000000        0x0 /opt/toolchains/n64/mips64-elf/mips64-elf/lib/libm.a(lib_a-k_cos.o)
 .mdebug.abiO64
                0x0000000000000000        0x0 /opt/toolchains/n64/mips64-elf/mips64-elf/lib/libm.a(lib_a-k_rem_pio2.o)
 .mdebug.abiO64
                0x0000000000000000        0x0 /opt/toolchains/n64/mips64-elf/mips64-elf/lib/libm.a(lib_a-k_sin.o)
 .mdebug.abiO64
                0x0000000000000000        0x0 /opt/toolchains/n64/mips64-elf/mips64-elf/lib/libm.a(lib_a-s_fabs.o)
 .mdebug.abiO64
                0x0000000000000000        0x0 /opt/toolchains/n64/mips64-elf/mips64-elf/lib/libm.a(lib_a-s_finite.o)
 .mdebug.abiO64
                0x0000000000000000        0x0 /opt/toolchains/n64/mips64-elf/mips64-elf/lib/libm.a(lib_a-s_floor.o)
 .mdebug.abiO64
                0x0000000000000000        0x0 /opt/toolchains/n64/mips64-elf/mips64-elf/lib/libm.a(lib_a-s_fpclassify.o)
 .mdebug.abiO64
                0x0000000000000000        0x0 /opt/toolchains/n64/mips64-elf/mips64-elf/lib/libm.a(lib_a-s_lib_ver.o)
 .mdebug.abiO64
                0x0000000000000000        0x0 /opt/toolchains/n64/mips64-elf/mips64-elf/lib/libm.a(lib_a-s_matherr.o)
 .mdebug.abiO64
                0x0000000000000000        0x0 /opt/toolchains/n64/mips64-elf/mips64-elf/lib/libm.a(lib_a-s_nan.o)
 .mdebug.abiO64
                0x0000000000000000        0x0 /opt/toolchains/n64/mips64-elf/mips64-elf/lib/libm.a(lib_a-s_rint.o)
 .mdebug.abiO64
                0x0000000000000000        0x0 /opt/toolchains/n64/mips64-elf/mips64-elf/lib/libm.a(lib_a-s_scalbn.o)
 .mdebug.abiO64
                0x0000000000000000        0x0 /opt/toolchains/n64/mips64-elf/mips64-elf/lib/libm.a(lib_a-s_copysign.o)
 .mdebug.abiO64
                0x0000000000000000        0x0 /opt/toolchains/n64/mips64-elf/lib/libdragon.a(n64sys.o)
 .mdebug.abiO64
                0x0000000000000000        0x0 /opt/toolchains/n64/mips64-elf/lib/libdragon.a(interrupt.o)
 .mdebug.abiO64
                0x0000000000000000        0x0 /opt/toolchains/n64/mips64-elf/lib/libdragon.a(dragonfs.o)
 .mdebug.abiO64
                0x0000000000000000        0x0 /opt/toolchains/n64/mips64-elf/lib/libdragon.a(audio.o)
 .mdebug.abiO64
                0x0000000000000000        0x0 /opt/toolchains/n64/mips64-elf/lib/libdragon.a(display.o)
 .mdebug.abiO64
                0x0000000000000000        0x0 /opt/toolchains/n64/mips64-elf/lib/libdragon.a(controller.o)
 .mdebug.abiO64
                0x0000000000000000        0x0 /opt/toolchains/n64/mips64-elf/lib/libdragon.a(graphics.o)
 .mdebug.abiO64
                0x0000000000000000        0x0 /opt/toolchains/n64/mips64-elf/lib/libdragon.a(rdp.o)
 .mdebug.abiO64
                0x0000000000000000        0x0 /opt/toolchains/n64/mips64-elf/lib/libdragon.a(dma.o)
 .mdebug.abiO64
                0x0000000000000000        0x0 /opt/toolchains/n64/mips64-elf/lib/libdragon.a(timer.o)
 .mdebug.abiO64
                0x0000000000000000        0x0 /opt/toolchains/n64/mips64-elf/lib/libdragon.a(exception.o)
 .mdebug.abiO64
                0x0000000000000000        0x0 /opt/toolchains/n64/mips64-elf/mips64-elf/lib/libc.a(lib_a-assert.o)
 .mdebug.abiO64
                0x0000000000000000        0x0 /opt/toolchains/n64/mips64-elf/mips64-elf/lib/libc.a(lib_a-errno.o)
 .mdebug.abiO64
                0x0000000000000000        0x0 /opt/toolchains/n64/mips64-elf/mips64-elf/lib/libc.a(lib_a-fclose.o)
 .mdebug.abiO64
                0x0000000000000000        0x0 /opt/toolchains/n64/mips64-elf/mips64-elf/lib/libc.a(lib_a-fflush.o)
 .mdebug.abiO64
                0x0000000000000000        0x0 /opt/toolchains/n64/mips64-elf/mips64-elf/lib/libc.a(lib_a-findfp.o)
 .mdebug.abiO64
                0x0000000000000000        0x0 /opt/toolchains/n64/mips64-elf/mips64-elf/lib/libc.a(lib_a-fiprintf.o)
 .mdebug.abiO64
                0x0000000000000000        0x0 /opt/toolchains/n64/mips64-elf/mips64-elf/lib/libc.a(lib_a-fopen.o)
 .mdebug.abiO64
                0x0000000000000000        0x0 /opt/toolchains/n64/mips64-elf/mips64-elf/lib/libc.a(lib_a-fread.o)
 .mdebug.abiO64
                0x0000000000000000        0x0 /opt/toolchains/n64/mips64-elf/mips64-elf/lib/libc.a(lib_a-freer.o)
 .mdebug.abiO64
                0x0000000000000000        0x0 /opt/toolchains/n64/mips64-elf/mips64-elf/lib/libc.a(lib_a-fseek.o)
 .mdebug.abiO64
                0x0000000000000000        0x0 /opt/toolchains/n64/mips64-elf/mips64-elf/lib/libc.a(lib_a-fstatr.o)
 .mdebug.abiO64
                0x0000000000000000        0x0 /opt/toolchains/n64/mips64-elf/mips64-elf/lib/libc.a(lib_a-ftell.o)
 .mdebug.abiO64
                0x0000000000000000        0x0 /opt/toolchains/n64/mips64-elf/mips64-elf/lib/libc.a(lib_a-fwalk.o)
 .mdebug.abiO64
                0x0000000000000000        0x0 /opt/toolchains/n64/mips64-elf/mips64-elf/lib/libc.a(lib_a-fwrite.o)
 .mdebug.abiO64
                0x0000000000000000        0x0 /opt/toolchains/n64/mips64-elf/mips64-elf/lib/libc.a(lib_a-impure.o)
 .mdebug.abiO64
                0x0000000000000000        0x0 /opt/toolchains/n64/mips64-elf/mips64-elf/lib/libc.a(lib_a-makebuf.o)
 .mdebug.abiO64
                0x0000000000000000        0x0 /opt/toolchains/n64/mips64-elf/mips64-elf/lib/libc.a(lib_a-malloc.o)
 .mdebug.abiO64
                0x0000000000000000        0x0 /opt/toolchains/n64/mips64-elf/mips64-elf/lib/libc.a(lib_a-mallocr.o)
 .mdebug.abiO64
                0x0000000000000000        0x0 /opt/toolchains/n64/mips64-elf/mips64-elf/lib/libc.a(lib_a-memcpy.o)
 .mdebug.abiO64
                0x0000000000000000        0x0 /opt/toolchains/n64/mips64-elf/mips64-elf/lib/libc.a(lib_a-memset.o)
 .mdebug.abiO64
                0x0000000000000000        0x0 /opt/toolchains/n64/mips64-elf/mips64-elf/lib/libc.a(lib_a-mlock.o)
 .mdebug.abiO64
                0x0000000000000000        0x0 /opt/toolchains/n64/mips64-elf/mips64-elf/lib/libc.a(lib_a-openr.o)
 .mdebug.abiO64
                0x0000000000000000        0x0 /opt/toolchains/n64/mips64-elf/mips64-elf/lib/libc.a(lib_a-realloc.o)
 .mdebug.abiO64
                0x0000000000000000        0x0 /opt/toolchains/n64/mips64-elf/mips64-elf/lib/libc.a(lib_a-reallocr.o)
 .mdebug.abiO64
                0x0000000000000000        0x0 /opt/toolchains/n64/mips64-elf/mips64-elf/lib/libc.a(lib_a-reent.o)
 .mdebug.abiO64
                0x0000000000000000        0x0 /opt/toolchains/n64/mips64-elf/mips64-elf/lib/libc.a(lib_a-refill.o)
 .mdebug.abiO64
                0x0000000000000000        0x0 /opt/toolchains/n64/mips64-elf/mips64-elf/lib/libc.a(lib_a-sbrkr.o)
 .mdebug.abiO64
                0x0000000000000000        0x0 /opt/toolchains/n64/mips64-elf/mips64-elf/lib/libc.a(lib_a-sprintf.o)
 .mdebug.abiO64
                0x0000000000000000        0x0 /opt/toolchains/n64/mips64-elf/mips64-elf/lib/libc.a(lib_a-stdio.o)
 .mdebug.abiO64
                0x0000000000000000        0x0 /opt/toolchains/n64/mips64-elf/mips64-elf/lib/libc.a(lib_a-strcmp.o)
 .mdebug.abiO64
                0x0000000000000000        0x0 /opt/toolchains/n64/mips64-elf/mips64-elf/lib/libc.a(lib_a-strcpy.o)
 .mdebug.abiO64
                0x0000000000000000        0x0 /opt/toolchains/n64/mips64-elf/mips64-elf/lib/libc.a(lib_a-strlen.o)
 .mdebug.abiO64
                0x0000000000000000        0x0 /opt/toolchains/n64/mips64-elf/mips64-elf/lib/libc.a(lib_a-svfprintf.o)
 .mdebug.abiO64
                0x0000000000000000        0x0 /opt/toolchains/n64/mips64-elf/mips64-elf/lib/libc.a(lib_a-vfiprintf.o)
 .mdebug.abiO64
                0x0000000000000000        0x0 /opt/toolchains/n64/mips64-elf/mips64-elf/lib/libc.a(lib_a-writer.o)
 .mdebug.abiO64
                0x0000000000000000        0x0 /opt/toolchains/n64/mips64-elf/mips64-elf/lib/libc.a(lib_a-wsetup.o)
 .mdebug.abiO64
                0x0000000000000000        0x0 /opt/toolchains/n64/mips64-elf/mips64-elf/lib/libc.a(lib_a-abort.o)
 .mdebug.abiO64
                0x0000000000000000        0x0 /opt/toolchains/n64/mips64-elf/mips64-elf/lib/libc.a(lib_a-closer.o)
 .mdebug.abiO64
                0x0000000000000000        0x0 /opt/toolchains/n64/mips64-elf/mips64-elf/lib/libc.a(lib_a-dtoa.o)
 .mdebug.abiO64
                0x0000000000000000        0x0 /opt/toolchains/n64/mips64-elf/mips64-elf/lib/libc.a(lib_a-flags.o)
 .mdebug.abiO64
                0x0000000000000000        0x0 /opt/toolchains/n64/mips64-elf/mips64-elf/lib/libc.a(lib_a-fputwc.o)
 .mdebug.abiO64
                0x0000000000000000        0x0 /opt/toolchains/n64/mips64-elf/mips64-elf/lib/libc.a(lib_a-fvwrite.o)
 .mdebug.abiO64
                0x0000000000000000        0x0 /opt/toolchains/n64/mips64-elf/mips64-elf/lib/libc.a(lib_a-isattyr.o)
 .mdebug.abiO64
                0x0000000000000000        0x0 /opt/toolchains/n64/mips64-elf/mips64-elf/lib/libc.a(lib_a-locale.o)
 .mdebug.abiO64
                0x0000000000000000        0x0 /opt/toolchains/n64/mips64-elf/mips64-elf/lib/libc.a(lib_a-lseekr.o)
 .mdebug.abiO64
                0x0000000000000000        0x0 /opt/toolchains/n64/mips64-elf/mips64-elf/lib/libc.a(lib_a-memchr.o)
 .mdebug.abiO64
                0x0000000000000000        0x0 /opt/toolchains/n64/mips64-elf/mips64-elf/lib/libc.a(lib_a-memmove.o)
 .mdebug.abiO64
                0x0000000000000000        0x0 /opt/toolchains/n64/mips64-elf/mips64-elf/lib/libc.a(lib_a-mprec.o)
 .mdebug.abiO64
                0x0000000000000000        0x0 /opt/toolchains/n64/mips64-elf/mips64-elf/lib/libc.a(lib_a-readr.o)
 .mdebug.abiO64
                0x0000000000000000        0x0 /opt/toolchains/n64/mips64-elf/mips64-elf/lib/libc.a(lib_a-signal.o)
 .mdebug.abiO64
                0x0000000000000000        0x0 /opt/toolchains/n64/mips64-elf/mips64-elf/lib/libc.a(lib_a-signalr.o)
 .mdebug.abiO64
                0x0000000000000000        0x0 /opt/toolchains/n64/mips64-elf/mips64-elf/lib/libc.a(lib_a-svfiprintf.o)
 .mdebug.abiO64
                0x0000000000000000        0x0 /opt/toolchains/n64/mips64-elf/mips64-elf/lib/libc.a(lib_a-wbuf.o)
 .mdebug.abiO64
                0x0000000000000000        0x0 /opt/toolchains/n64/mips64-elf/mips64-elf/lib/libc.a(lib_a-wcrtomb.o)
 .mdebug.abiO64
                0x0000000000000000        0x0 /opt/toolchains/n64/mips64-elf/mips64-elf/lib/libc.a(lib_a-wctomb_r.o)
 .mdebug.abiO64
                0x0000000000000000        0x0 /opt/toolchains/n64/mips64-elf/mips64-elf/lib/libc.a(lib_a-callocr.o)
 .mdebug.abiO64
                0x0000000000000000        0x0 /opt/toolchains/n64/mips64-elf/lib/libdragonsys.a(system.o)
 .mdebug.abiO64
                0x0000000000000000        0x0 /opt/toolchains/n64/mips64-elf/mips64-elf/lib/libnosys.a(_exit.o)

.gcc_compiled_long32
                0x0000000000000000        0x0
 .gcc_compiled_long32
                0x0000000000000000        0x0 main.o
 .gcc_compiled_long32
                0x0000000000000000        0x0 stb_image.o
 .gcc_compiled_long32
                0x0000000000000000        0x0 ../game/ai/boost.o
 .gcc_compiled_long32
                0x0000000000000000        0x0 ../game/ai/bullet.o
 .gcc_compiled_long32
                0x0000000000000000        0x0 ../game/ai/death.o
 .gcc_compiled_long32
                0x0000000000000000        0x0 ../game/ai/explode.o
 .gcc_compiled_long32
                0x0000000000000000        0x0 ../game/ai/pickup.o
 .gcc_compiled_long32
                0x0000000000000000        0x0 ../game/ai/quad.o
 .gcc_compiled_long32
                0x0000000000000000        0x0 ../game/ai/sheba.o
 .gcc_compiled_long32
                0x0000000000000000        0x0 ../game/ai/static_model.o
 .gcc_compiled_long32
                0x0000000000000000        0x0 ../game/ai/static_sprite.o
 .gcc_compiled_long32
                0x0000000000000000        0x0 ../game/ai/teleporter.o
 .gcc_compiled_long32
                0x0000000000000000        0x0 ../game/ai/torch.o
 .gcc_compiled_long32
                0x0000000000000000        0x0 ../game/data.o
 .gcc_compiled_long32
                0x0000000000000000        0x0 ../game/entities.o
 .gcc_compiled_long32
                0x0000000000000000        0x0 ../game/game.o
 .gcc_compiled_long32
                0x0000000000000000        0x0 ../game/maps.o
 .gcc_compiled_long32
                0x0000000000000000        0x0 ../game/models.o
 .gcc_compiled_long32
                0x0000000000000000        0x0 ../game/screens.o
 .gcc_compiled_long32
                0x0000000000000000        0x0 ../game/sprites.o
 .gcc_compiled_long32
                0x0000000000000000        0x0 ../y3d/y3d_animation.o
 .gcc_compiled_long32
                0x0000000000000000        0x0 ../y3d/y3d_ansic.o
 .gcc_compiled_long32
                0x0000000000000000        0x0 ../y3d/y3d_cell.o
 .gcc_compiled_long32
                0x0000000000000000        0x0 ../y3d/y3d_draw.o
 .gcc_compiled_long32
                0x0000000000000000        0x0 ../y3d/y3d_engine.o
 .gcc_compiled_long32
                0x0000000000000000        0x0 ../y3d/y3d_entity.o
 .gcc_compiled_long32
                0x0000000000000000        0x0 ../y3d/y3d_file.o
 .gcc_compiled_long32
                0x0000000000000000        0x0 ../y3d/y3d_fixed.o
 .gcc_compiled_long32
                0x0000000000000000        0x0 ../y3d/y3d_fruity.o
 .gcc_compiled_long32
                0x0000000000000000        0x0 ../y3d/y3d_image.o
 .gcc_compiled_long32
                0x0000000000000000        0x0 ../y3d/y3d_keyboard.o
 .gcc_compiled_long32
                0x0000000000000000        0x0 ../y3d/y3d_map.o
 .gcc_compiled_long32
                0x0000000000000000        0x0 ../y3d/y3d_matrix.o
 .gcc_compiled_long32
                0x0000000000000000        0x0 ../y3d/y3d_pixel.o
 .gcc_compiled_long32
                0x0000000000000000        0x0 ../y3d/y3d_record.o
 .gcc_compiled_long32
                0x0000000000000000        0x0 ../y3d/y3d_sound.o
 .gcc_compiled_long32
                0x0000000000000000        0x0 ../y3d/y3d_spanner.o
 .gcc_compiled_long32
                0x0000000000000000        0x0 ../y3d/y3d_surface.o
 .gcc_compiled_long32
                0x0000000000000000        0x0 ../y3d/y3d_vertex.o
 .gcc_compiled_long32
                0x0000000000000000        0x0 ../y3d/y3d_yeti.o
 .gcc_compiled_long32
                0x0000000000000000        0x0 /opt/toolchains/n64/mips64-elf/mips64-elf/lib/libm.a(lib_a-s_sin.o)
 .gcc_compiled_long32
                0x0000000000000000        0x0 /opt/toolchains/n64/mips64-elf/mips64-elf/lib/libm.a(lib_a-w_pow.o)
 .gcc_compiled_long32
                0x0000000000000000        0x0 /opt/toolchains/n64/mips64-elf/mips64-elf/lib/libm.a(lib_a-e_pow.o)
 .gcc_compiled_long32
                0x0000000000000000        0x0 /opt/toolchains/n64/mips64-elf/mips64-elf/lib/libm.a(lib_a-e_rem_pio2.o)
 .gcc_compiled_long32
                0x0000000000000000        0x0 /opt/toolchains/n64/mips64-elf/mips64-elf/lib/libm.a(lib_a-e_sqrt.o)
 .gcc_compiled_long32
                0x0000000000000000        0x0 /opt/toolchains/n64/mips64-elf/mips64-elf/lib/libm.a(lib_a-k_cos.o)
 .gcc_compiled_long32
                0x0000000000000000        0x0 /opt/toolchains/n64/mips64-elf/mips64-elf/lib/libm.a(lib_a-k_rem_pio2.o)
 .gcc_compiled_long32
                0x0000000000000000        0x0 /opt/toolchains/n64/mips64-elf/mips64-elf/lib/libm.a(lib_a-k_sin.o)
 .gcc_compiled_long32
                0x0000000000000000        0x0 /opt/toolchains/n64/mips64-elf/mips64-elf/lib/libm.a(lib_a-s_fabs.o)
 .gcc_compiled_long32
                0x0000000000000000        0x0 /opt/toolchains/n64/mips64-elf/mips64-elf/lib/libm.a(lib_a-s_finite.o)
 .gcc_compiled_long32
                0x0000000000000000        0x0 /opt/toolchains/n64/mips64-elf/mips64-elf/lib/libm.a(lib_a-s_floor.o)
 .gcc_compiled_long32
                0x0000000000000000        0x0 /opt/toolchains/n64/mips64-elf/mips64-elf/lib/libm.a(lib_a-s_fpclassify.o)
 .gcc_compiled_long32
                0x0000000000000000        0x0 /opt/toolchains/n64/mips64-elf/mips64-elf/lib/libm.a(lib_a-s_lib_ver.o)
 .gcc_compiled_long32
                0x0000000000000000        0x0 /opt/toolchains/n64/mips64-elf/mips64-elf/lib/libm.a(lib_a-s_matherr.o)
 .gcc_compiled_long32
                0x0000000000000000        0x0 /opt/toolchains/n64/mips64-elf/mips64-elf/lib/libm.a(lib_a-s_nan.o)
 .gcc_compiled_long32
                0x0000000000000000        0x0 /opt/toolchains/n64/mips64-elf/mips64-elf/lib/libm.a(lib_a-s_rint.o)
 .gcc_compiled_long32
                0x0000000000000000        0x0 /opt/toolchains/n64/mips64-elf/mips64-elf/lib/libm.a(lib_a-s_scalbn.o)
 .gcc_compiled_long32
                0x0000000000000000        0x0 /opt/toolchains/n64/mips64-elf/mips64-elf/lib/libm.a(lib_a-s_copysign.o)
 .gcc_compiled_long32
                0x0000000000000000        0x0 /opt/toolchains/n64/mips64-elf/lib/libdragon.a(n64sys.o)
 .gcc_compiled_long32
                0x0000000000000000        0x0 /opt/toolchains/n64/mips64-elf/lib/libdragon.a(interrupt.o)
 .gcc_compiled_long32
                0x0000000000000000        0x0 /opt/toolchains/n64/mips64-elf/lib/libdragon.a(dragonfs.o)
 .gcc_compiled_long32
                0x0000000000000000        0x0 /opt/toolchains/n64/mips64-elf/lib/libdragon.a(audio.o)
 .gcc_compiled_long32
                0x0000000000000000        0x0 /opt/toolchains/n64/mips64-elf/lib/libdragon.a(display.o)
 .gcc_compiled_long32
                0x0000000000000000        0x0 /opt/toolchains/n64/mips64-elf/lib/libdragon.a(controller.o)
 .gcc_compiled_long32
                0x0000000000000000        0x0 /opt/toolchains/n64/mips64-elf/lib/libdragon.a(graphics.o)
 .gcc_compiled_long32
                0x0000000000000000        0x0 /opt/toolchains/n64/mips64-elf/lib/libdragon.a(rdp.o)
 .gcc_compiled_long32
                0x0000000000000000        0x0 /opt/toolchains/n64/mips64-elf/lib/libdragon.a(dma.o)
 .gcc_compiled_long32
                0x0000000000000000        0x0 /opt/toolchains/n64/mips64-elf/lib/libdragon.a(timer.o)
 .gcc_compiled_long32
                0x0000000000000000        0x0 /opt/toolchains/n64/mips64-elf/lib/libdragon.a(exception.o)
 .gcc_compiled_long32
                0x0000000000000000        0x0 /opt/toolchains/n64/mips64-elf/mips64-elf/lib/libc.a(lib_a-assert.o)
 .gcc_compiled_long32
                0x0000000000000000        0x0 /opt/toolchains/n64/mips64-elf/mips64-elf/lib/libc.a(lib_a-errno.o)
 .gcc_compiled_long32
                0x0000000000000000        0x0 /opt/toolchains/n64/mips64-elf/mips64-elf/lib/libc.a(lib_a-fclose.o)
 .gcc_compiled_long32
                0x0000000000000000        0x0 /opt/toolchains/n64/mips64-elf/mips64-elf/lib/libc.a(lib_a-fflush.o)
 .gcc_compiled_long32
                0x0000000000000000        0x0 /opt/toolchains/n64/mips64-elf/mips64-elf/lib/libc.a(lib_a-findfp.o)
 .gcc_compiled_long32
                0x0000000000000000        0x0 /opt/toolchains/n64/mips64-elf/mips64-elf/lib/libc.a(lib_a-fiprintf.o)
 .gcc_compiled_long32
                0x0000000000000000        0x0 /opt/toolchains/n64/mips64-elf/mips64-elf/lib/libc.a(lib_a-fopen.o)
 .gcc_compiled_long32
                0x0000000000000000        0x0 /opt/toolchains/n64/mips64-elf/mips64-elf/lib/libc.a(lib_a-fread.o)
 .gcc_compiled_long32
                0x0000000000000000        0x0 /opt/toolchains/n64/mips64-elf/mips64-elf/lib/libc.a(lib_a-freer.o)
 .gcc_compiled_long32
                0x0000000000000000        0x0 /opt/toolchains/n64/mips64-elf/mips64-elf/lib/libc.a(lib_a-fseek.o)
 .gcc_compiled_long32
                0x0000000000000000        0x0 /opt/toolchains/n64/mips64-elf/mips64-elf/lib/libc.a(lib_a-fstatr.o)
 .gcc_compiled_long32
                0x0000000000000000        0x0 /opt/toolchains/n64/mips64-elf/mips64-elf/lib/libc.a(lib_a-ftell.o)
 .gcc_compiled_long32
                0x0000000000000000        0x0 /opt/toolchains/n64/mips64-elf/mips64-elf/lib/libc.a(lib_a-fwalk.o)
 .gcc_compiled_long32
                0x0000000000000000        0x0 /opt/toolchains/n64/mips64-elf/mips64-elf/lib/libc.a(lib_a-fwrite.o)
 .gcc_compiled_long32
                0x0000000000000000        0x0 /opt/toolchains/n64/mips64-elf/mips64-elf/lib/libc.a(lib_a-impure.o)
 .gcc_compiled_long32
                0x0000000000000000        0x0 /opt/toolchains/n64/mips64-elf/mips64-elf/lib/libc.a(lib_a-makebuf.o)
 .gcc_compiled_long32
                0x0000000000000000        0x0 /opt/toolchains/n64/mips64-elf/mips64-elf/lib/libc.a(lib_a-malloc.o)
 .gcc_compiled_long32
                0x0000000000000000        0x0 /opt/toolchains/n64/mips64-elf/mips64-elf/lib/libc.a(lib_a-mallocr.o)
 .gcc_compiled_long32
                0x0000000000000000        0x0 /opt/toolchains/n64/mips64-elf/mips64-elf/lib/libc.a(lib_a-memcpy.o)
 .gcc_compiled_long32
                0x0000000000000000        0x0 /opt/toolchains/n64/mips64-elf/mips64-elf/lib/libc.a(lib_a-memset.o)
 .gcc_compiled_long32
                0x0000000000000000        0x0 /opt/toolchains/n64/mips64-elf/mips64-elf/lib/libc.a(lib_a-mlock.o)
 .gcc_compiled_long32
                0x0000000000000000        0x0 /opt/toolchains/n64/mips64-elf/mips64-elf/lib/libc.a(lib_a-openr.o)
 .gcc_compiled_long32
                0x0000000000000000        0x0 /opt/toolchains/n64/mips64-elf/mips64-elf/lib/libc.a(lib_a-realloc.o)
 .gcc_compiled_long32
                0x0000000000000000        0x0 /opt/toolchains/n64/mips64-elf/mips64-elf/lib/libc.a(lib_a-reallocr.o)
 .gcc_compiled_long32
                0x0000000000000000        0x0 /opt/toolchains/n64/mips64-elf/mips64-elf/lib/libc.a(lib_a-reent.o)
 .gcc_compiled_long32
                0x0000000000000000        0x0 /opt/toolchains/n64/mips64-elf/mips64-elf/lib/libc.a(lib_a-refill.o)
 .gcc_compiled_long32
                0x0000000000000000        0x0 /opt/toolchains/n64/mips64-elf/mips64-elf/lib/libc.a(lib_a-sbrkr.o)
 .gcc_compiled_long32
                0x0000000000000000        0x0 /opt/toolchains/n64/mips64-elf/mips64-elf/lib/libc.a(lib_a-sprintf.o)
 .gcc_compiled_long32
                0x0000000000000000        0x0 /opt/toolchains/n64/mips64-elf/mips64-elf/lib/libc.a(lib_a-stdio.o)
 .gcc_compiled_long32
                0x0000000000000000        0x0 /opt/toolchains/n64/mips64-elf/mips64-elf/lib/libc.a(lib_a-strcmp.o)
 .gcc_compiled_long32
                0x0000000000000000        0x0 /opt/toolchains/n64/mips64-elf/mips64-elf/lib/libc.a(lib_a-strcpy.o)
 .gcc_compiled_long32
                0x0000000000000000        0x0 /opt/toolchains/n64/mips64-elf/mips64-elf/lib/libc.a(lib_a-strlen.o)
 .gcc_compiled_long32
                0x0000000000000000        0x0 /opt/toolchains/n64/mips64-elf/mips64-elf/lib/libc.a(lib_a-svfprintf.o)
 .gcc_compiled_long32
                0x0000000000000000        0x0 /opt/toolchains/n64/mips64-elf/mips64-elf/lib/libc.a(lib_a-vfiprintf.o)
 .gcc_compiled_long32
                0x0000000000000000        0x0 /opt/toolchains/n64/mips64-elf/mips64-elf/lib/libc.a(lib_a-writer.o)
 .gcc_compiled_long32
                0x0000000000000000        0x0 /opt/toolchains/n64/mips64-elf/mips64-elf/lib/libc.a(lib_a-wsetup.o)
 .gcc_compiled_long32
                0x0000000000000000        0x0 /opt/toolchains/n64/mips64-elf/mips64-elf/lib/libc.a(lib_a-abort.o)
 .gcc_compiled_long32
                0x0000000000000000        0x0 /opt/toolchains/n64/mips64-elf/mips64-elf/lib/libc.a(lib_a-closer.o)
 .gcc_compiled_long32
                0x0000000000000000        0x0 /opt/toolchains/n64/mips64-elf/mips64-elf/lib/libc.a(lib_a-dtoa.o)
 .gcc_compiled_long32
                0x0000000000000000        0x0 /opt/toolchains/n64/mips64-elf/mips64-elf/lib/libc.a(lib_a-flags.o)
 .gcc_compiled_long32
                0x0000000000000000        0x0 /opt/toolchains/n64/mips64-elf/mips64-elf/lib/libc.a(lib_a-fputwc.o)
 .gcc_compiled_long32
                0x0000000000000000        0x0 /opt/toolchains/n64/mips64-elf/mips64-elf/lib/libc.a(lib_a-fvwrite.o)
 .gcc_compiled_long32
                0x0000000000000000        0x0 /opt/toolchains/n64/mips64-elf/mips64-elf/lib/libc.a(lib_a-isattyr.o)
 .gcc_compiled_long32
                0x0000000000000000        0x0 /opt/toolchains/n64/mips64-elf/mips64-elf/lib/libc.a(lib_a-locale.o)
 .gcc_compiled_long32
                0x0000000000000000        0x0 /opt/toolchains/n64/mips64-elf/mips64-elf/lib/libc.a(lib_a-lseekr.o)
 .gcc_compiled_long32
                0x0000000000000000        0x0 /opt/toolchains/n64/mips64-elf/mips64-elf/lib/libc.a(lib_a-memchr.o)
 .gcc_compiled_long32
                0x0000000000000000        0x0 /opt/toolchains/n64/mips64-elf/mips64-elf/lib/libc.a(lib_a-memmove.o)
 .gcc_compiled_long32
                0x0000000000000000        0x0 /opt/toolchains/n64/mips64-elf/mips64-elf/lib/libc.a(lib_a-mprec.o)
 .gcc_compiled_long32
                0x0000000000000000        0x0 /opt/toolchains/n64/mips64-elf/mips64-elf/lib/libc.a(lib_a-readr.o)
 .gcc_compiled_long32
                0x0000000000000000        0x0 /opt/toolchains/n64/mips64-elf/mips64-elf/lib/libc.a(lib_a-signal.o)
 .gcc_compiled_long32
                0x0000000000000000        0x0 /opt/toolchains/n64/mips64-elf/mips64-elf/lib/libc.a(lib_a-signalr.o)
 .gcc_compiled_long32
                0x0000000000000000        0x0 /opt/toolchains/n64/mips64-elf/mips64-elf/lib/libc.a(lib_a-svfiprintf.o)
 .gcc_compiled_long32
                0x0000000000000000        0x0 /opt/toolchains/n64/mips64-elf/mips64-elf/lib/libc.a(lib_a-wbuf.o)
 .gcc_compiled_long32
                0x0000000000000000        0x0 /opt/toolchains/n64/mips64-elf/mips64-elf/lib/libc.a(lib_a-wcrtomb.o)
 .gcc_compiled_long32
                0x0000000000000000        0x0 /opt/toolchains/n64/mips64-elf/mips64-elf/lib/libc.a(lib_a-wctomb_r.o)
 .gcc_compiled_long32
                0x0000000000000000        0x0 /opt/toolchains/n64/mips64-elf/mips64-elf/lib/libc.a(lib_a-callocr.o)
 .gcc_compiled_long32
                0x0000000000000000        0x0 /opt/toolchains/n64/mips64-elf/lib/libdragonsys.a(system.o)
 .gcc_compiled_long32
                0x0000000000000000        0x0 /opt/toolchains/n64/mips64-elf/mips64-elf/lib/libnosys.a(_exit.o)

.comment        0x0000000000000000       0x11
 .comment       0x0000000000000000       0x11 main.o
                                         0x12 (size before relaxing)
 .comment       0x0000000000000000       0x12 stb_image.o
 .comment       0x0000000000000000       0x12 ../game/ai/boost.o
 .comment       0x0000000000000000       0x12 ../game/ai/bullet.o
 .comment       0x0000000000000000       0x12 ../game/ai/death.o
 .comment       0x0000000000000000       0x12 ../game/ai/explode.o
 .comment       0x0000000000000000       0x12 ../game/ai/pickup.o
 .comment       0x0000000000000000       0x12 ../game/ai/quad.o
 .comment       0x0000000000000000       0x12 ../game/ai/sheba.o
 .comment       0x0000000000000000       0x12 ../game/ai/static_model.o
 .comment       0x0000000000000000       0x12 ../game/ai/static_sprite.o
 .comment       0x0000000000000000       0x12 ../game/ai/teleporter.o
 .comment       0x0000000000000000       0x12 ../game/ai/torch.o
 .comment       0x0000000000000000       0x12 ../game/data.o
 .comment       0x0000000000000000       0x12 ../game/entities.o
 .comment       0x0000000000000000       0x12 ../game/game.o
 .comment       0x0000000000000000       0x12 ../game/maps.o
 .comment       0x0000000000000000       0x12 ../game/models.o
 .comment       0x0000000000000000       0x12 ../game/screens.o
 .comment       0x0000000000000000       0x12 ../game/sprites.o
 .comment       0x0000000000000000       0x12 ../y3d/y3d_animation.o
 .comment       0x0000000000000000       0x12 ../y3d/y3d_ansic.o
 .comment       0x0000000000000000       0x12 ../y3d/y3d_cell.o
 .comment       0x0000000000000000       0x12 ../y3d/y3d_draw.o
 .comment       0x0000000000000000       0x12 ../y3d/y3d_engine.o
 .comment       0x0000000000000000       0x12 ../y3d/y3d_entity.o
 .comment       0x0000000000000000       0x12 ../y3d/y3d_file.o
 .comment       0x0000000000000000       0x12 ../y3d/y3d_fixed.o
 .comment       0x0000000000000000       0x12 ../y3d/y3d_fruity.o
 .comment       0x0000000000000000       0x12 ../y3d/y3d_image.o
 .comment       0x0000000000000000       0x12 ../y3d/y3d_keyboard.o
 .comment       0x0000000000000000       0x12 ../y3d/y3d_map.o
 .comment       0x0000000000000000       0x12 ../y3d/y3d_matrix.o
 .comment       0x0000000000000000       0x12 ../y3d/y3d_pixel.o
 .comment       0x0000000000000000       0x12 ../y3d/y3d_record.o
 .comment       0x0000000000000000       0x12 ../y3d/y3d_sound.o
 .comment       0x0000000000000000       0x12 ../y3d/y3d_spanner.o
 .comment       0x0000000000000000       0x12 ../y3d/y3d_surface.o
 .comment       0x0000000000000000       0x12 ../y3d/y3d_vertex.o
 .comment       0x0000000000000000       0x12 ../y3d/y3d_yeti.o
 .comment       0x0000000000000000       0x12 /opt/toolchains/n64/mips64-elf/mips64-elf/lib/libm.a(lib_a-s_sin.o)
 .comment       0x0000000000000000       0x12 /opt/toolchains/n64/mips64-elf/mips64-elf/lib/libm.a(lib_a-w_pow.o)
 .comment       0x0000000000000000       0x12 /opt/toolchains/n64/mips64-elf/mips64-elf/lib/libm.a(lib_a-e_pow.o)
 .comment       0x0000000000000000       0x12 /opt/toolchains/n64/mips64-elf/mips64-elf/lib/libm.a(lib_a-e_rem_pio2.o)
 .comment       0x0000000000000000       0x12 /opt/toolchains/n64/mips64-elf/mips64-elf/lib/libm.a(lib_a-e_sqrt.o)
 .comment       0x0000000000000000       0x12 /opt/toolchains/n64/mips64-elf/mips64-elf/lib/libm.a(lib_a-k_cos.o)
 .comment       0x0000000000000000       0x12 /opt/toolchains/n64/mips64-elf/mips64-elf/lib/libm.a(lib_a-k_rem_pio2.o)
 .comment       0x0000000000000000       0x12 /opt/toolchains/n64/mips64-elf/mips64-elf/lib/libm.a(lib_a-k_sin.o)
 .comment       0x0000000000000000       0x12 /opt/toolchains/n64/mips64-elf/mips64-elf/lib/libm.a(lib_a-s_fabs.o)
 .comment       0x0000000000000000       0x12 /opt/toolchains/n64/mips64-elf/mips64-elf/lib/libm.a(lib_a-s_finite.o)
 .comment       0x0000000000000000       0x12 /opt/toolchains/n64/mips64-elf/mips64-elf/lib/libm.a(lib_a-s_floor.o)
 .comment       0x0000000000000000       0x12 /opt/toolchains/n64/mips64-elf/mips64-elf/lib/libm.a(lib_a-s_fpclassify.o)
 .comment       0x0000000000000000       0x12 /opt/toolchains/n64/mips64-elf/mips64-elf/lib/libm.a(lib_a-s_lib_ver.o)
 .comment       0x0000000000000000       0x12 /opt/toolchains/n64/mips64-elf/mips64-elf/lib/libm.a(lib_a-s_matherr.o)
 .comment       0x0000000000000000       0x12 /opt/toolchains/n64/mips64-elf/mips64-elf/lib/libm.a(lib_a-s_nan.o)
 .comment       0x0000000000000000       0x12 /opt/toolchains/n64/mips64-elf/mips64-elf/lib/libm.a(lib_a-s_rint.o)
 .comment       0x0000000000000000       0x12 /opt/toolchains/n64/mips64-elf/mips64-elf/lib/libm.a(lib_a-s_scalbn.o)
 .comment       0x0000000000000000       0x12 /opt/toolchains/n64/mips64-elf/mips64-elf/lib/libm.a(lib_a-s_copysign.o)
 .comment       0x0000000000000000       0x12 /opt/toolchains/n64/mips64-elf/lib/libdragon.a(n64sys.o)
 .comment       0x0000000000000000       0x12 /opt/toolchains/n64/mips64-elf/lib/libdragon.a(interrupt.o)
 .comment       0x0000000000000000       0x12 /opt/toolchains/n64/mips64-elf/lib/libdragon.a(dragonfs.o)
 .comment       0x0000000000000000       0x12 /opt/toolchains/n64/mips64-elf/lib/libdragon.a(audio.o)
 .comment       0x0000000000000000       0x12 /opt/toolchains/n64/mips64-elf/lib/libdragon.a(display.o)
 .comment       0x0000000000000000       0x12 /opt/toolchains/n64/mips64-elf/lib/libdragon.a(controller.o)
 .comment       0x0000000000000000       0x12 /opt/toolchains/n64/mips64-elf/lib/libdragon.a(graphics.o)
 .comment       0x0000000000000000       0x12 /opt/toolchains/n64/mips64-elf/lib/libdragon.a(rdp.o)
 .comment       0x0000000000000000       0x12 /opt/toolchains/n64/mips64-elf/lib/libdragon.a(dma.o)
 .comment       0x0000000000000000       0x12 /opt/toolchains/n64/mips64-elf/lib/libdragon.a(timer.o)
 .comment       0x0000000000000000       0x12 /opt/toolchains/n64/mips64-elf/lib/libdragon.a(exception.o)
 .comment       0x0000000000000000       0x12 /opt/toolchains/n64/mips64-elf/mips64-elf/lib/libc.a(lib_a-assert.o)
 .comment       0x0000000000000000       0x12 /opt/toolchains/n64/mips64-elf/mips64-elf/lib/libc.a(lib_a-errno.o)
 .comment       0x0000000000000000       0x12 /opt/toolchains/n64/mips64-elf/mips64-elf/lib/libc.a(lib_a-fclose.o)
 .comment       0x0000000000000000       0x12 /opt/toolchains/n64/mips64-elf/mips64-elf/lib/libc.a(lib_a-fflush.o)
 .comment       0x0000000000000000       0x12 /opt/toolchains/n64/mips64-elf/mips64-elf/lib/libc.a(lib_a-findfp.o)
 .comment       0x0000000000000000       0x12 /opt/toolchains/n64/mips64-elf/mips64-elf/lib/libc.a(lib_a-fiprintf.o)
 .comment       0x0000000000000000       0x12 /opt/toolchains/n64/mips64-elf/mips64-elf/lib/libc.a(lib_a-fopen.o)
 .comment       0x0000000000000000       0x12 /opt/toolchains/n64/mips64-elf/mips64-elf/lib/libc.a(lib_a-fread.o)
 .comment       0x0000000000000000       0x12 /opt/toolchains/n64/mips64-elf/mips64-elf/lib/libc.a(lib_a-freer.o)
 .comment       0x0000000000000000       0x12 /opt/toolchains/n64/mips64-elf/mips64-elf/lib/libc.a(lib_a-fseek.o)
 .comment       0x0000000000000000       0x12 /opt/toolchains/n64/mips64-elf/mips64-elf/lib/libc.a(lib_a-fstatr.o)
 .comment       0x0000000000000000       0x12 /opt/toolchains/n64/mips64-elf/mips64-elf/lib/libc.a(lib_a-ftell.o)
 .comment       0x0000000000000000       0x12 /opt/toolchains/n64/mips64-elf/mips64-elf/lib/libc.a(lib_a-fwalk.o)
 .comment       0x0000000000000000       0x12 /opt/toolchains/n64/mips64-elf/mips64-elf/lib/libc.a(lib_a-fwrite.o)
 .comment       0x0000000000000000       0x12 /opt/toolchains/n64/mips64-elf/mips64-elf/lib/libc.a(lib_a-impure.o)
 .comment       0x0000000000000000       0x12 /opt/toolchains/n64/mips64-elf/mips64-elf/lib/libc.a(lib_a-makebuf.o)
 .comment       0x0000000000000000       0x12 /opt/toolchains/n64/mips64-elf/mips64-elf/lib/libc.a(lib_a-malloc.o)
 .comment       0x0000000000000000       0x12 /opt/toolchains/n64/mips64-elf/mips64-elf/lib/libc.a(lib_a-mallocr.o)
 .comment       0x0000000000000000       0x12 /opt/toolchains/n64/mips64-elf/mips64-elf/lib/libc.a(lib_a-memcpy.o)
 .comment       0x0000000000000000       0x12 /opt/toolchains/n64/mips64-elf/mips64-elf/lib/libc.a(lib_a-memset.o)
 .comment       0x0000000000000000       0x12 /opt/toolchains/n64/mips64-elf/mips64-elf/lib/libc.a(lib_a-mlock.o)
 .comment       0x0000000000000000       0x12 /opt/toolchains/n64/mips64-elf/mips64-elf/lib/libc.a(lib_a-openr.o)
 .comment       0x0000000000000000       0x12 /opt/toolchains/n64/mips64-elf/mips64-elf/lib/libc.a(lib_a-realloc.o)
 .comment       0x0000000000000000       0x12 /opt/toolchains/n64/mips64-elf/mips64-elf/lib/libc.a(lib_a-reallocr.o)
 .comment       0x0000000000000000       0x12 /opt/toolchains/n64/mips64-elf/mips64-elf/lib/libc.a(lib_a-reent.o)
 .comment       0x0000000000000000       0x12 /opt/toolchains/n64/mips64-elf/mips64-elf/lib/libc.a(lib_a-refill.o)
 .comment       0x0000000000000000       0x12 /opt/toolchains/n64/mips64-elf/mips64-elf/lib/libc.a(lib_a-sbrkr.o)
 .comment       0x0000000000000000       0x12 /opt/toolchains/n64/mips64-elf/mips64-elf/lib/libc.a(lib_a-sprintf.o)
 .comment       0x0000000000000000       0x12 /opt/toolchains/n64/mips64-elf/mips64-elf/lib/libc.a(lib_a-stdio.o)
 .comment       0x0000000000000000       0x12 /opt/toolchains/n64/mips64-elf/mips64-elf/lib/libc.a(lib_a-strcmp.o)
 .comment       0x0000000000000000       0x12 /opt/toolchains/n64/mips64-elf/mips64-elf/lib/libc.a(lib_a-strcpy.o)
 .comment       0x0000000000000000       0x12 /opt/toolchains/n64/mips64-elf/mips64-elf/lib/libc.a(lib_a-strlen.o)
 .comment       0x0000000000000000       0x12 /opt/toolchains/n64/mips64-elf/mips64-elf/lib/libc.a(lib_a-svfprintf.o)
 .comment       0x0000000000000000       0x12 /opt/toolchains/n64/mips64-elf/mips64-elf/lib/libc.a(lib_a-vfiprintf.o)
 .comment       0x0000000000000000       0x12 /opt/toolchains/n64/mips64-elf/mips64-elf/lib/libc.a(lib_a-writer.o)
 .comment       0x0000000000000000       0x12 /opt/toolchains/n64/mips64-elf/mips64-elf/lib/libc.a(lib_a-wsetup.o)
 .comment       0x0000000000000000       0x12 /opt/toolchains/n64/mips64-elf/mips64-elf/lib/libc.a(lib_a-abort.o)
 .comment       0x0000000000000000       0x12 /opt/toolchains/n64/mips64-elf/mips64-elf/lib/libc.a(lib_a-closer.o)
 .comment       0x0000000000000000       0x12 /opt/toolchains/n64/mips64-elf/mips64-elf/lib/libc.a(lib_a-dtoa.o)
 .comment       0x0000000000000000       0x12 /opt/toolchains/n64/mips64-elf/mips64-elf/lib/libc.a(lib_a-flags.o)
 .comment       0x0000000000000000       0x12 /opt/toolchains/n64/mips64-elf/mips64-elf/lib/libc.a(lib_a-fputwc.o)
 .comment       0x0000000000000000       0x12 /opt/toolchains/n64/mips64-elf/mips64-elf/lib/libc.a(lib_a-fvwrite.o)
 .comment       0x0000000000000000       0x12 /opt/toolchains/n64/mips64-elf/mips64-elf/lib/libc.a(lib_a-isattyr.o)
 .comment       0x0000000000000000       0x12 /opt/toolchains/n64/mips64-elf/mips64-elf/lib/libc.a(lib_a-locale.o)
 .comment       0x0000000000000000       0x12 /opt/toolchains/n64/mips64-elf/mips64-elf/lib/libc.a(lib_a-lseekr.o)
 .comment       0x0000000000000000       0x12 /opt/toolchains/n64/mips64-elf/mips64-elf/lib/libc.a(lib_a-memchr.o)
 .comment       0x0000000000000000       0x12 /opt/toolchains/n64/mips64-elf/mips64-elf/lib/libc.a(lib_a-memmove.o)
 .comment       0x0000000000000000       0x12 /opt/toolchains/n64/mips64-elf/mips64-elf/lib/libc.a(lib_a-mprec.o)
 .comment       0x0000000000000000       0x12 /opt/toolchains/n64/mips64-elf/mips64-elf/lib/libc.a(lib_a-readr.o)
 .comment       0x0000000000000000       0x12 /opt/toolchains/n64/mips64-elf/mips64-elf/lib/libc.a(lib_a-signal.o)
 .comment       0x0000000000000000       0x12 /opt/toolchains/n64/mips64-elf/mips64-elf/lib/libc.a(lib_a-signalr.o)
 .comment       0x0000000000000000       0x12 /opt/toolchains/n64/mips64-elf/mips64-elf/lib/libc.a(lib_a-svfiprintf.o)
 .comment       0x0000000000000000       0x12 /opt/toolchains/n64/mips64-elf/mips64-elf/lib/libc.a(lib_a-wbuf.o)
 .comment       0x0000000000000000       0x12 /opt/toolchains/n64/mips64-elf/mips64-elf/lib/libc.a(lib_a-wcrtomb.o)
 .comment       0x0000000000000000       0x12 /opt/toolchains/n64/mips64-elf/mips64-elf/lib/libc.a(lib_a-wctomb_r.o)
 .comment       0x0000000000000000       0x12 /opt/toolchains/n64/mips64-elf/mips64-elf/lib/libc.a(lib_a-callocr.o)
 .comment       0x0000000000000000       0x12 /opt/toolchains/n64/mips64-elf/lib/libdragonsys.a(system.o)
 .comment       0x0000000000000000       0x12 /opt/toolchains/n64/mips64-elf/mips64-elf/lib/libnosys.a(_exit.o)

.gnu.attributes
                0x0000000000000000       0x10
 .gnu.attributes
                0x0000000000000000       0x10 main.o
 .gnu.attributes
                0x0000000000000010       0x10 stb_image.o
 .gnu.attributes
                0x0000000000000020       0x10 ../game/ai/boost.o
 .gnu.attributes
                0x0000000000000030       0x10 ../game/ai/bullet.o
 .gnu.attributes
                0x0000000000000040       0x10 ../game/ai/death.o
 .gnu.attributes
                0x0000000000000050       0x10 ../game/ai/explode.o
 .gnu.attributes
                0x0000000000000060       0x10 ../game/ai/pickup.o
 .gnu.attributes
                0x0000000000000070       0x10 ../game/ai/quad.o
 .gnu.attributes
                0x0000000000000080       0x10 ../game/ai/sheba.o
 .gnu.attributes
                0x0000000000000090       0x10 ../game/ai/static_model.o
 .gnu.attributes
                0x00000000000000a0       0x10 ../game/ai/static_sprite.o
 .gnu.attributes
                0x00000000000000b0       0x10 ../game/ai/teleporter.o
 .gnu.attributes
                0x00000000000000c0       0x10 ../game/ai/torch.o
 .gnu.attributes
                0x00000000000000d0       0x10 ../game/data.o
 .gnu.attributes
                0x00000000000000e0       0x10 ../game/entities.o
 .gnu.attributes
                0x00000000000000f0       0x10 ../game/game.o
 .gnu.attributes
                0x0000000000000100       0x10 ../game/maps.o
 .gnu.attributes
                0x0000000000000110       0x10 ../game/models.o
 .gnu.attributes
                0x0000000000000120       0x10 ../game/screens.o
 .gnu.attributes
                0x0000000000000130       0x10 ../game/sprites.o
 .gnu.attributes
                0x0000000000000140       0x10 ../y3d/y3d_animation.o
 .gnu.attributes
                0x0000000000000150       0x10 ../y3d/y3d_ansic.o
 .gnu.attributes
                0x0000000000000160       0x10 ../y3d/y3d_cell.o
 .gnu.attributes
                0x0000000000000170       0x10 ../y3d/y3d_draw.o
 .gnu.attributes
                0x0000000000000180       0x10 ../y3d/y3d_engine.o
 .gnu.attributes
                0x0000000000000190       0x10 ../y3d/y3d_entity.o
 .gnu.attributes
                0x00000000000001a0       0x10 ../y3d/y3d_file.o
 .gnu.attributes
                0x00000000000001b0       0x10 ../y3d/y3d_fixed.o
 .gnu.attributes
                0x00000000000001c0       0x10 ../y3d/y3d_fruity.o
 .gnu.attributes
                0x00000000000001d0       0x10 ../y3d/y3d_image.o
 .gnu.attributes
                0x00000000000001e0       0x10 ../y3d/y3d_keyboard.o
 .gnu.attributes
                0x00000000000001f0       0x10 ../y3d/y3d_map.o
 .gnu.attributes
                0x0000000000000200       0x10 ../y3d/y3d_matrix.o
 .gnu.attributes
                0x0000000000000210       0x10 ../y3d/y3d_pixel.o
 .gnu.attributes
                0x0000000000000220       0x10 ../y3d/y3d_record.o
 .gnu.attributes
                0x0000000000000230       0x10 ../y3d/y3d_sound.o
 .gnu.attributes
                0x0000000000000240       0x10 ../y3d/y3d_spanner.o
 .gnu.attributes
                0x0000000000000250       0x10 ../y3d/y3d_surface.o
 .gnu.attributes
                0x0000000000000260       0x10 ../y3d/y3d_vertex.o
 .gnu.attributes
                0x0000000000000270       0x10 ../y3d/y3d_yeti.o
 .gnu.attributes
                0x0000000000000280       0x10 /opt/toolchains/n64/mips64-elf/mips64-elf/lib/libm.a(lib_a-s_sin.o)
 .gnu.attributes
                0x0000000000000290       0x10 /opt/toolchains/n64/mips64-elf/mips64-elf/lib/libm.a(lib_a-w_pow.o)
 .gnu.attributes
                0x00000000000002a0       0x10 /opt/toolchains/n64/mips64-elf/mips64-elf/lib/libm.a(lib_a-e_pow.o)
 .gnu.attributes
                0x00000000000002b0       0x10 /opt/toolchains/n64/mips64-elf/mips64-elf/lib/libm.a(lib_a-e_rem_pio2.o)
 .gnu.attributes
                0x00000000000002c0       0x10 /opt/toolchains/n64/mips64-elf/mips64-elf/lib/libm.a(lib_a-e_sqrt.o)
 .gnu.attributes
                0x00000000000002d0       0x10 /opt/toolchains/n64/mips64-elf/mips64-elf/lib/libm.a(lib_a-k_cos.o)
 .gnu.attributes
                0x00000000000002e0       0x10 /opt/toolchains/n64/mips64-elf/mips64-elf/lib/libm.a(lib_a-k_rem_pio2.o)
 .gnu.attributes
                0x00000000000002f0       0x10 /opt/toolchains/n64/mips64-elf/mips64-elf/lib/libm.a(lib_a-k_sin.o)
 .gnu.attributes
                0x0000000000000300       0x10 /opt/toolchains/n64/mips64-elf/mips64-elf/lib/libm.a(lib_a-s_fabs.o)
 .gnu.attributes
                0x0000000000000310       0x10 /opt/toolchains/n64/mips64-elf/mips64-elf/lib/libm.a(lib_a-s_finite.o)
 .gnu.attributes
                0x0000000000000320       0x10 /opt/toolchains/n64/mips64-elf/mips64-elf/lib/libm.a(lib_a-s_floor.o)
 .gnu.attributes
                0x0000000000000330       0x10 /opt/toolchains/n64/mips64-elf/mips64-elf/lib/libm.a(lib_a-s_fpclassify.o)
 .gnu.attributes
                0x0000000000000340       0x10 /opt/toolchains/n64/mips64-elf/mips64-elf/lib/libm.a(lib_a-s_lib_ver.o)
 .gnu.attributes
                0x0000000000000350       0x10 /opt/toolchains/n64/mips64-elf/mips64-elf/lib/libm.a(lib_a-s_matherr.o)
 .gnu.attributes
                0x0000000000000360       0x10 /opt/toolchains/n64/mips64-elf/mips64-elf/lib/libm.a(lib_a-s_nan.o)
 .gnu.attributes
                0x0000000000000370       0x10 /opt/toolchains/n64/mips64-elf/mips64-elf/lib/libm.a(lib_a-s_rint.o)
 .gnu.attributes
                0x0000000000000380       0x10 /opt/toolchains/n64/mips64-elf/mips64-elf/lib/libm.a(lib_a-s_scalbn.o)
 .gnu.attributes
                0x0000000000000390       0x10 /opt/toolchains/n64/mips64-elf/mips64-elf/lib/libm.a(lib_a-s_copysign.o)
 .gnu.attributes
                0x00000000000003a0       0x10 /opt/toolchains/n64/mips64-elf/lib/libdragon.a(n64sys.o)
 .gnu.attributes
                0x00000000000003b0       0x10 /opt/toolchains/n64/mips64-elf/lib/libdragon.a(interrupt.o)
 .gnu.attributes
                0x00000000000003c0       0x10 /opt/toolchains/n64/mips64-elf/lib/libdragon.a(dragonfs.o)
 .gnu.attributes
                0x00000000000003d0       0x10 /opt/toolchains/n64/mips64-elf/lib/libdragon.a(audio.o)
 .gnu.attributes
                0x00000000000003e0       0x10 /opt/toolchains/n64/mips64-elf/lib/libdragon.a(display.o)
 .gnu.attributes
                0x00000000000003f0       0x10 /opt/toolchains/n64/mips64-elf/lib/libdragon.a(controller.o)
 .gnu.attributes
                0x0000000000000400       0x10 /opt/toolchains/n64/mips64-elf/lib/libdragon.a(graphics.o)
 .gnu.attributes
                0x0000000000000410       0x10 /opt/toolchains/n64/mips64-elf/lib/libdragon.a(rdp.o)
 .gnu.attributes
                0x0000000000000420       0x10 /opt/toolchains/n64/mips64-elf/lib/libdragon.a(dma.o)
 .gnu.attributes
                0x0000000000000430       0x10 /opt/toolchains/n64/mips64-elf/lib/libdragon.a(timer.o)
 .gnu.attributes
                0x0000000000000440       0x10 /opt/toolchains/n64/mips64-elf/lib/libdragon.a(exception.o)
 .gnu.attributes
                0x0000000000000450       0x10 /opt/toolchains/n64/mips64-elf/mips64-elf/lib/libc.a(lib_a-assert.o)
 .gnu.attributes
                0x0000000000000460       0x10 /opt/toolchains/n64/mips64-elf/mips64-elf/lib/libc.a(lib_a-errno.o)
 .gnu.attributes
                0x0000000000000470       0x10 /opt/toolchains/n64/mips64-elf/mips64-elf/lib/libc.a(lib_a-fclose.o)
 .gnu.attributes
                0x0000000000000480       0x10 /opt/toolchains/n64/mips64-elf/mips64-elf/lib/libc.a(lib_a-fflush.o)
 .gnu.attributes
                0x0000000000000490       0x10 /opt/toolchains/n64/mips64-elf/mips64-elf/lib/libc.a(lib_a-findfp.o)
 .gnu.attributes
                0x00000000000004a0       0x10 /opt/toolchains/n64/mips64-elf/mips64-elf/lib/libc.a(lib_a-fiprintf.o)
 .gnu.attributes
                0x00000000000004b0       0x10 /opt/toolchains/n64/mips64-elf/mips64-elf/lib/libc.a(lib_a-fopen.o)
 .gnu.attributes
                0x00000000000004c0       0x10 /opt/toolchains/n64/mips64-elf/mips64-elf/lib/libc.a(lib_a-fread.o)
 .gnu.attributes
                0x00000000000004d0       0x10 /opt/toolchains/n64/mips64-elf/mips64-elf/lib/libc.a(lib_a-freer.o)
 .gnu.attributes
                0x00000000000004e0       0x10 /opt/toolchains/n64/mips64-elf/mips64-elf/lib/libc.a(lib_a-fseek.o)
 .gnu.attributes
                0x00000000000004f0       0x10 /opt/toolchains/n64/mips64-elf/mips64-elf/lib/libc.a(lib_a-fstatr.o)
 .gnu.attributes
                0x0000000000000500       0x10 /opt/toolchains/n64/mips64-elf/mips64-elf/lib/libc.a(lib_a-ftell.o)
 .gnu.attributes
                0x0000000000000510       0x10 /opt/toolchains/n64/mips64-elf/mips64-elf/lib/libc.a(lib_a-fwalk.o)
 .gnu.attributes
                0x0000000000000520       0x10 /opt/toolchains/n64/mips64-elf/mips64-elf/lib/libc.a(lib_a-fwrite.o)
 .gnu.attributes
                0x0000000000000530       0x10 /opt/toolchains/n64/mips64-elf/mips64-elf/lib/libc.a(lib_a-impure.o)
 .gnu.attributes
                0x0000000000000540       0x10 /opt/toolchains/n64/mips64-elf/mips64-elf/lib/libc.a(lib_a-makebuf.o)
 .gnu.attributes
                0x0000000000000550       0x10 /opt/toolchains/n64/mips64-elf/mips64-elf/lib/libc.a(lib_a-malloc.o)
 .gnu.attributes
                0x0000000000000560       0x10 /opt/toolchains/n64/mips64-elf/mips64-elf/lib/libc.a(lib_a-mallocr.o)
 .gnu.attributes
                0x0000000000000570       0x10 /opt/toolchains/n64/mips64-elf/mips64-elf/lib/libc.a(lib_a-memcpy.o)
 .gnu.attributes
                0x0000000000000580       0x10 /opt/toolchains/n64/mips64-elf/mips64-elf/lib/libc.a(lib_a-memset.o)
 .gnu.attributes
                0x0000000000000590       0x10 /opt/toolchains/n64/mips64-elf/mips64-elf/lib/libc.a(lib_a-mlock.o)
 .gnu.attributes
                0x00000000000005a0       0x10 /opt/toolchains/n64/mips64-elf/mips64-elf/lib/libc.a(lib_a-openr.o)
 .gnu.attributes
                0x00000000000005b0       0x10 /opt/toolchains/n64/mips64-elf/mips64-elf/lib/libc.a(lib_a-realloc.o)
 .gnu.attributes
                0x00000000000005c0       0x10 /opt/toolchains/n64/mips64-elf/mips64-elf/lib/libc.a(lib_a-reallocr.o)
 .gnu.attributes
                0x00000000000005d0       0x10 /opt/toolchains/n64/mips64-elf/mips64-elf/lib/libc.a(lib_a-reent.o)
 .gnu.attributes
                0x00000000000005e0       0x10 /opt/toolchains/n64/mips64-elf/mips64-elf/lib/libc.a(lib_a-refill.o)
 .gnu.attributes
                0x00000000000005f0       0x10 /opt/toolchains/n64/mips64-elf/mips64-elf/lib/libc.a(lib_a-sbrkr.o)
 .gnu.attributes
                0x0000000000000600       0x10 /opt/toolchains/n64/mips64-elf/mips64-elf/lib/libc.a(lib_a-sprintf.o)
 .gnu.attributes
                0x0000000000000610       0x10 /opt/toolchains/n64/mips64-elf/mips64-elf/lib/libc.a(lib_a-stdio.o)
 .gnu.attributes
                0x0000000000000620       0x10 /opt/toolchains/n64/mips64-elf/mips64-elf/lib/libc.a(lib_a-strcmp.o)
 .gnu.attributes
                0x0000000000000630       0x10 /opt/toolchains/n64/mips64-elf/mips64-elf/lib/libc.a(lib_a-strcpy.o)
 .gnu.attributes
                0x0000000000000640       0x10 /opt/toolchains/n64/mips64-elf/mips64-elf/lib/libc.a(lib_a-strlen.o)
 .gnu.attributes
                0x0000000000000650       0x10 /opt/toolchains/n64/mips64-elf/mips64-elf/lib/libc.a(lib_a-svfprintf.o)
 .gnu.attributes
                0x0000000000000660       0x10 /opt/toolchains/n64/mips64-elf/mips64-elf/lib/libc.a(lib_a-vfiprintf.o)
 .gnu.attributes
                0x0000000000000670       0x10 /opt/toolchains/n64/mips64-elf/mips64-elf/lib/libc.a(lib_a-writer.o)
 .gnu.attributes
                0x0000000000000680       0x10 /opt/toolchains/n64/mips64-elf/mips64-elf/lib/libc.a(lib_a-wsetup.o)
 .gnu.attributes
                0x0000000000000690       0x10 /opt/toolchains/n64/mips64-elf/mips64-elf/lib/libc.a(lib_a-abort.o)
 .gnu.attributes
                0x00000000000006a0       0x10 /opt/toolchains/n64/mips64-elf/mips64-elf/lib/libc.a(lib_a-closer.o)
 .gnu.attributes
                0x00000000000006b0       0x10 /opt/toolchains/n64/mips64-elf/mips64-elf/lib/libc.a(lib_a-dtoa.o)
 .gnu.attributes
                0x00000000000006c0       0x10 /opt/toolchains/n64/mips64-elf/mips64-elf/lib/libc.a(lib_a-flags.o)
 .gnu.attributes
                0x00000000000006d0       0x10 /opt/toolchains/n64/mips64-elf/mips64-elf/lib/libc.a(lib_a-fputwc.o)
 .gnu.attributes
                0x00000000000006e0       0x10 /opt/toolchains/n64/mips64-elf/mips64-elf/lib/libc.a(lib_a-fvwrite.o)
 .gnu.attributes
                0x00000000000006f0       0x10 /opt/toolchains/n64/mips64-elf/mips64-elf/lib/libc.a(lib_a-isattyr.o)
 .gnu.attributes
                0x0000000000000700       0x10 /opt/toolchains/n64/mips64-elf/mips64-elf/lib/libc.a(lib_a-locale.o)
 .gnu.attributes
                0x0000000000000710       0x10 /opt/toolchains/n64/mips64-elf/mips64-elf/lib/libc.a(lib_a-lseekr.o)
 .gnu.attributes
                0x0000000000000720       0x10 /opt/toolchains/n64/mips64-elf/mips64-elf/lib/libc.a(lib_a-memchr.o)
 .gnu.attributes
                0x0000000000000730       0x10 /opt/toolchains/n64/mips64-elf/mips64-elf/lib/libc.a(lib_a-memmove.o)
 .gnu.attributes
                0x0000000000000740       0x10 /opt/toolchains/n64/mips64-elf/mips64-elf/lib/libc.a(lib_a-mprec.o)
 .gnu.attributes
                0x0000000000000750       0x10 /opt/toolchains/n64/mips64-elf/mips64-elf/lib/libc.a(lib_a-readr.o)
 .gnu.attributes
                0x0000000000000760       0x10 /opt/toolchains/n64/mips64-elf/mips64-elf/lib/libc.a(lib_a-signal.o)
 .gnu.attributes
                0x0000000000000770       0x10 /opt/toolchains/n64/mips64-elf/mips64-elf/lib/libc.a(lib_a-signalr.o)
 .gnu.attributes
                0x0000000000000780       0x10 /opt/toolchains/n64/mips64-elf/mips64-elf/lib/libc.a(lib_a-svfiprintf.o)
 .gnu.attributes
                0x0000000000000790       0x10 /opt/toolchains/n64/mips64-elf/mips64-elf/lib/libc.a(lib_a-wbuf.o)
 .gnu.attributes
                0x00000000000007a0       0x10 /opt/toolchains/n64/mips64-elf/mips64-elf/lib/libc.a(lib_a-wcrtomb.o)
 .gnu.attributes
                0x00000000000007b0       0x10 /opt/toolchains/n64/mips64-elf/mips64-elf/lib/libc.a(lib_a-wctomb_r.o)
 .gnu.attributes
                0x00000000000007c0       0x10 /opt/toolchains/n64/mips64-elf/mips64-elf/lib/libc.a(lib_a-callocr.o)
 .gnu.attributes
                0x00000000000007d0       0x10 /opt/toolchains/n64/mips64-elf/lib/libdragonsys.a(system.o)
 .gnu.attributes
                0x00000000000007e0       0x10 /opt/toolchains/n64/mips64-elf/mips64-elf/lib/libnosys.a(_exit.o)

.code           0x0000000000000000        0x0
 .code          0x0000000000000000        0x0 /opt/toolchains/n64/mips64-elf/lib/libdragon.a(entrypoint.o)

.debug_info     0x0000000000000000    0x23dbb
 .debug_info    0x0000000000000000      0x17c /opt/toolchains/n64/mips64-elf/mips64-elf/lib/libm.a(lib_a-s_sin.o)
 .debug_info    0x000000000000017c      0x18c /opt/toolchains/n64/mips64-elf/mips64-elf/lib/libm.a(lib_a-w_pow.o)
 .debug_info    0x0000000000000308      0x6f1 /opt/toolchains/n64/mips64-elf/mips64-elf/lib/libm.a(lib_a-e_pow.o)
 .debug_info    0x00000000000009f9      0x36f /opt/toolchains/n64/mips64-elf/mips64-elf/lib/libm.a(lib_a-e_rem_pio2.o)
 .debug_info    0x0000000000000d68      0x230 /opt/toolchains/n64/mips64-elf/mips64-elf/lib/libm.a(lib_a-e_sqrt.o)
 .debug_info    0x0000000000000f98      0x233 /opt/toolchains/n64/mips64-elf/mips64-elf/lib/libm.a(lib_a-k_cos.o)
 .debug_info    0x00000000000011cb      0x2e3 /opt/toolchains/n64/mips64-elf/mips64-elf/lib/libm.a(lib_a-k_rem_pio2.o)
 .debug_info    0x00000000000014ae      0x20b /opt/toolchains/n64/mips64-elf/mips64-elf/lib/libm.a(lib_a-k_sin.o)
 .debug_info    0x00000000000016b9      0x14f /opt/toolchains/n64/mips64-elf/mips64-elf/lib/libm.a(lib_a-s_fabs.o)
 .debug_info    0x0000000000001808      0x13b /opt/toolchains/n64/mips64-elf/mips64-elf/lib/libm.a(lib_a-s_finite.o)
 .debug_info    0x0000000000001943      0x1ac /opt/toolchains/n64/mips64-elf/mips64-elf/lib/libm.a(lib_a-s_floor.o)
 .debug_info    0x0000000000001aef      0x141 /opt/toolchains/n64/mips64-elf/mips64-elf/lib/libm.a(lib_a-s_fpclassify.o)
 .debug_info    0x0000000000001c30       0xc1 /opt/toolchains/n64/mips64-elf/mips64-elf/lib/libm.a(lib_a-s_lib_ver.o)
 .debug_info    0x0000000000001cf1      0x12f /opt/toolchains/n64/mips64-elf/mips64-elf/lib/libm.a(lib_a-s_matherr.o)
 .debug_info    0x0000000000001e20      0x13b /opt/toolchains/n64/mips64-elf/mips64-elf/lib/libm.a(lib_a-s_nan.o)
 .debug_info    0x0000000000001f5b      0x221 /opt/toolchains/n64/mips64-elf/mips64-elf/lib/libm.a(lib_a-s_rint.o)
 .debug_info    0x000000000000217c      0x1fc /opt/toolchains/n64/mips64-elf/mips64-elf/lib/libm.a(lib_a-s_scalbn.o)
 .debug_info    0x0000000000002378      0x17d /opt/toolchains/n64/mips64-elf/mips64-elf/lib/libm.a(lib_a-s_copysign.o)
 .debug_info    0x00000000000024f5      0x9e3 /opt/toolchains/n64/mips64-elf/mips64-elf/lib/libc.a(lib_a-assert.o)
 .debug_info    0x0000000000002ed8      0x964 /opt/toolchains/n64/mips64-elf/mips64-elf/lib/libc.a(lib_a-errno.o)
 .debug_info    0x000000000000383c      0x9cb /opt/toolchains/n64/mips64-elf/mips64-elf/lib/libc.a(lib_a-fclose.o)
 .debug_info    0x0000000000004207      0xa85 /opt/toolchains/n64/mips64-elf/mips64-elf/lib/libc.a(lib_a-fflush.o)
 .debug_info    0x0000000000004c8c      0xbf6 /opt/toolchains/n64/mips64-elf/mips64-elf/lib/libc.a(lib_a-findfp.o)
 .debug_info    0x0000000000005882      0xa2f /opt/toolchains/n64/mips64-elf/mips64-elf/lib/libc.a(lib_a-fiprintf.o)
 .debug_info    0x00000000000062b1      0xa16 /opt/toolchains/n64/mips64-elf/mips64-elf/lib/libc.a(lib_a-fopen.o)
 .debug_info    0x0000000000006cc7      0xab5 /opt/toolchains/n64/mips64-elf/mips64-elf/lib/libc.a(lib_a-fread.o)
 .debug_info    0x000000000000777c      0xc40 /opt/toolchains/n64/mips64-elf/mips64-elf/lib/libc.a(lib_a-freer.o)
 .debug_info    0x00000000000083bc      0xc12 /opt/toolchains/n64/mips64-elf/mips64-elf/lib/libc.a(lib_a-fseek.o)
 .debug_info    0x0000000000008fce      0xb30 /opt/toolchains/n64/mips64-elf/mips64-elf/lib/libc.a(lib_a-fstatr.o)
 .debug_info    0x0000000000009afe      0x9cd /opt/toolchains/n64/mips64-elf/mips64-elf/lib/libc.a(lib_a-ftell.o)
 .debug_info    0x000000000000a4cb      0xa52 /opt/toolchains/n64/mips64-elf/mips64-elf/lib/libc.a(lib_a-fwalk.o)
 .debug_info    0x000000000000af1d      0xaba /opt/toolchains/n64/mips64-elf/mips64-elf/lib/libc.a(lib_a-fwrite.o)
 .debug_info    0x000000000000b9d7      0x966 /opt/toolchains/n64/mips64-elf/mips64-elf/lib/libc.a(lib_a-impure.o)
 .debug_info    0x000000000000c33d      0xb45 /opt/toolchains/n64/mips64-elf/mips64-elf/lib/libc.a(lib_a-makebuf.o)
 .debug_info    0x000000000000ce82      0x9a5 /opt/toolchains/n64/mips64-elf/mips64-elf/lib/libc.a(lib_a-malloc.o)
 .debug_info    0x000000000000d827      0xd6b /opt/toolchains/n64/mips64-elf/mips64-elf/lib/libc.a(lib_a-mallocr.o)
 .debug_info    0x000000000000e592      0x19d /opt/toolchains/n64/mips64-elf/mips64-elf/lib/libc.a(lib_a-memcpy.o)
 .debug_info    0x000000000000e72f      0x139 /opt/toolchains/n64/mips64-elf/mips64-elf/lib/libc.a(lib_a-memset.o)
 .debug_info    0x000000000000e868      0x980 /opt/toolchains/n64/mips64-elf/mips64-elf/lib/libc.a(lib_a-mlock.o)
 .debug_info    0x000000000000f1e8      0x9ab /opt/toolchains/n64/mips64-elf/mips64-elf/lib/libc.a(lib_a-openr.o)
 .debug_info    0x000000000000fb93      0x98b /opt/toolchains/n64/mips64-elf/mips64-elf/lib/libc.a(lib_a-realloc.o)
 .debug_info    0x000000000001051e      0xc00 /opt/toolchains/n64/mips64-elf/mips64-elf/lib/libc.a(lib_a-reallocr.o)
 .debug_info    0x000000000001111e      0xa64 /opt/toolchains/n64/mips64-elf/mips64-elf/lib/libc.a(lib_a-reent.o)
 .debug_info    0x0000000000011b82      0x9da /opt/toolchains/n64/mips64-elf/mips64-elf/lib/libc.a(lib_a-refill.o)
 .debug_info    0x000000000001255c      0x9ac /opt/toolchains/n64/mips64-elf/mips64-elf/lib/libc.a(lib_a-sbrkr.o)
 .debug_info    0x0000000000012f08      0xa52 /opt/toolchains/n64/mips64-elf/mips64-elf/lib/libc.a(lib_a-sprintf.o)
 .debug_info    0x000000000001395a      0xb2b /opt/toolchains/n64/mips64-elf/mips64-elf/lib/libc.a(lib_a-stdio.o)
 .debug_info    0x0000000000014485      0x123 /opt/toolchains/n64/mips64-elf/mips64-elf/lib/libc.a(lib_a-strcmp.o)
 .debug_info    0x00000000000145a8      0x10c /opt/toolchains/n64/mips64-elf/mips64-elf/lib/libc.a(lib_a-strcpy.o)
 .debug_info    0x00000000000146b4       0x73 /opt/toolchains/n64/mips64-elf/mips64-elf/lib/libc.a(lib_a-strlen.o)
 .debug_info    0x0000000000014727     0x1008 /opt/toolchains/n64/mips64-elf/mips64-elf/lib/libc.a(lib_a-svfprintf.o)
 .debug_info    0x000000000001572f      0xf41 /opt/toolchains/n64/mips64-elf/mips64-elf/lib/libc.a(lib_a-vfiprintf.o)
 .debug_info    0x0000000000016670      0x9c7 /opt/toolchains/n64/mips64-elf/mips64-elf/lib/libc.a(lib_a-writer.o)
 .debug_info    0x0000000000017037      0x992 /opt/toolchains/n64/mips64-elf/mips64-elf/lib/libc.a(lib_a-wsetup.o)
 .debug_info    0x00000000000179c9       0x88 /opt/toolchains/n64/mips64-elf/mips64-elf/lib/libc.a(lib_a-abort.o)
 .debug_info    0x0000000000017a51      0x98c /opt/toolchains/n64/mips64-elf/mips64-elf/lib/libc.a(lib_a-closer.o)
 .debug_info    0x00000000000183dd      0xdcc /opt/toolchains/n64/mips64-elf/mips64-elf/lib/libc.a(lib_a-dtoa.o)
 .debug_info    0x00000000000191a9      0x99f /opt/toolchains/n64/mips64-elf/mips64-elf/lib/libc.a(lib_a-flags.o)
 .debug_info    0x0000000000019b48      0xaa8 /opt/toolchains/n64/mips64-elf/mips64-elf/lib/libc.a(lib_a-fputwc.o)
 .debug_info    0x000000000001a5f0      0xab3 /opt/toolchains/n64/mips64-elf/mips64-elf/lib/libc.a(lib_a-fvwrite.o)
 .debug_info    0x000000000001b0a3      0x98c /opt/toolchains/n64/mips64-elf/mips64-elf/lib/libc.a(lib_a-isattyr.o)
 .debug_info    0x000000000001ba2f      0xc94 /opt/toolchains/n64/mips64-elf/mips64-elf/lib/libc.a(lib_a-locale.o)
 .debug_info    0x000000000001c6c3      0x9b5 /opt/toolchains/n64/mips64-elf/mips64-elf/lib/libc.a(lib_a-lseekr.o)
 .debug_info    0x000000000001d078      0x125 /opt/toolchains/n64/mips64-elf/mips64-elf/lib/libc.a(lib_a-memchr.o)
 .debug_info    0x000000000001d19d      0x12f /opt/toolchains/n64/mips64-elf/mips64-elf/lib/libc.a(lib_a-memmove.o)
 .debug_info    0x000000000001d2cc     0x14f1 /opt/toolchains/n64/mips64-elf/mips64-elf/lib/libc.a(lib_a-mprec.o)
 .debug_info    0x000000000001e7bd      0x9c0 /opt/toolchains/n64/mips64-elf/mips64-elf/lib/libc.a(lib_a-readr.o)
 .debug_info    0x000000000001f17d      0xb57 /opt/toolchains/n64/mips64-elf/mips64-elf/lib/libc.a(lib_a-signal.o)
 .debug_info    0x000000000001fcd4      0x9e2 /opt/toolchains/n64/mips64-elf/mips64-elf/lib/libc.a(lib_a-signalr.o)
 .debug_info    0x00000000000206b6      0xd85 /opt/toolchains/n64/mips64-elf/mips64-elf/lib/libc.a(lib_a-svfiprintf.o)
 .debug_info    0x000000000002143b      0x9e5 /opt/toolchains/n64/mips64-elf/mips64-elf/lib/libc.a(lib_a-wbuf.o)
 .debug_info    0x0000000000021e20      0xa99 /opt/toolchains/n64/mips64-elf/mips64-elf/lib/libc.a(lib_a-wcrtomb.o)
 .debug_info    0x00000000000228b9      0xa59 /opt/toolchains/n64/mips64-elf/mips64-elf/lib/libc.a(lib_a-wctomb_r.o)
 .debug_info    0x0000000000023312      0xa4e /opt/toolchains/n64/mips64-elf/mips64-elf/lib/libc.a(lib_a-callocr.o)
 .debug_info    0x0000000000023d60       0x5b /opt/toolchains/n64/mips64-elf/mips64-elf/lib/libnosys.a(_exit.o)

.debug_abbrev   0x0000000000000000     0x6dc0
 .debug_abbrev  0x0000000000000000       0xf7 /opt/toolchains/n64/mips64-elf/mips64-elf/lib/libm.a(lib_a-s_sin.o)
 .debug_abbrev  0x00000000000000f7       0xcf /opt/toolchains/n64/mips64-elf/mips64-elf/lib/libm.a(lib_a-w_pow.o)
 .debug_abbrev  0x00000000000001c6      0x162 /opt/toolchains/n64/mips64-elf/mips64-elf/lib/libm.a(lib_a-e_pow.o)
 .debug_abbrev  0x0000000000000328      0x12c /opt/toolchains/n64/mips64-elf/mips64-elf/lib/libm.a(lib_a-e_rem_pio2.o)
 .debug_abbrev  0x0000000000000454      0x115 /opt/toolchains/n64/mips64-elf/mips64-elf/lib/libm.a(lib_a-e_sqrt.o)
 .debug_abbrev  0x0000000000000569      0x104 /opt/toolchains/n64/mips64-elf/mips64-elf/lib/libm.a(lib_a-k_cos.o)
 .debug_abbrev  0x000000000000066d       0xf7 /opt/toolchains/n64/mips64-elf/mips64-elf/lib/libm.a(lib_a-k_rem_pio2.o)
 .debug_abbrev  0x0000000000000764      0x10a /opt/toolchains/n64/mips64-elf/mips64-elf/lib/libm.a(lib_a-k_sin.o)
 .debug_abbrev  0x000000000000086e       0xd0 /opt/toolchains/n64/mips64-elf/mips64-elf/lib/libm.a(lib_a-s_fabs.o)
 .debug_abbrev  0x000000000000093e       0xc5 /opt/toolchains/n64/mips64-elf/mips64-elf/lib/libm.a(lib_a-s_finite.o)
 .debug_abbrev  0x0000000000000a03       0xf7 /opt/toolchains/n64/mips64-elf/mips64-elf/lib/libm.a(lib_a-s_floor.o)
 .debug_abbrev  0x0000000000000afa       0xc7 /opt/toolchains/n64/mips64-elf/mips64-elf/lib/libm.a(lib_a-s_fpclassify.o)
 .debug_abbrev  0x0000000000000bc1       0x53 /opt/toolchains/n64/mips64-elf/mips64-elf/lib/libm.a(lib_a-s_lib_ver.o)
 .debug_abbrev  0x0000000000000c14       0x97 /opt/toolchains/n64/mips64-elf/mips64-elf/lib/libm.a(lib_a-s_matherr.o)
 .debug_abbrev  0x0000000000000cab       0xd5 /opt/toolchains/n64/mips64-elf/mips64-elf/lib/libm.a(lib_a-s_nan.o)
 .debug_abbrev  0x0000000000000d80      0x10e /opt/toolchains/n64/mips64-elf/mips64-elf/lib/libm.a(lib_a-s_rint.o)
 .debug_abbrev  0x0000000000000e8e       0xea /opt/toolchains/n64/mips64-elf/mips64-elf/lib/libm.a(lib_a-s_scalbn.o)
 .debug_abbrev  0x0000000000000f78       0xf5 /opt/toolchains/n64/mips64-elf/mips64-elf/lib/libm.a(lib_a-s_copysign.o)
 .debug_abbrev  0x000000000000106d      0x17d /opt/toolchains/n64/mips64-elf/mips64-elf/lib/libc.a(lib_a-assert.o)
 .debug_abbrev  0x00000000000011ea      0x16e /opt/toolchains/n64/mips64-elf/mips64-elf/lib/libc.a(lib_a-errno.o)
 .debug_abbrev  0x0000000000001358      0x1b6 /opt/toolchains/n64/mips64-elf/mips64-elf/lib/libc.a(lib_a-fclose.o)
 .debug_abbrev  0x000000000000150e      0x1e3 /opt/toolchains/n64/mips64-elf/mips64-elf/lib/libc.a(lib_a-fflush.o)
 .debug_abbrev  0x00000000000016f1      0x289 /opt/toolchains/n64/mips64-elf/mips64-elf/lib/libc.a(lib_a-findfp.o)
 .debug_abbrev  0x000000000000197a      0x1b5 /opt/toolchains/n64/mips64-elf/mips64-elf/lib/libc.a(lib_a-fiprintf.o)
 .debug_abbrev  0x0000000000001b2f      0x1d4 /opt/toolchains/n64/mips64-elf/mips64-elf/lib/libc.a(lib_a-fopen.o)
 .debug_abbrev  0x0000000000001d03      0x1e4 /opt/toolchains/n64/mips64-elf/mips64-elf/lib/libc.a(lib_a-fread.o)
 .debug_abbrev  0x0000000000001ee7      0x1ea /opt/toolchains/n64/mips64-elf/mips64-elf/lib/libc.a(lib_a-freer.o)
 .debug_abbrev  0x00000000000020d1      0x217 /opt/toolchains/n64/mips64-elf/mips64-elf/lib/libc.a(lib_a-fseek.o)
 .debug_abbrev  0x00000000000022e8      0x19d /opt/toolchains/n64/mips64-elf/mips64-elf/lib/libc.a(lib_a-fstatr.o)
 .debug_abbrev  0x0000000000002485      0x1a7 /opt/toolchains/n64/mips64-elf/mips64-elf/lib/libc.a(lib_a-ftell.o)
 .debug_abbrev  0x000000000000262c      0x18c /opt/toolchains/n64/mips64-elf/mips64-elf/lib/libc.a(lib_a-fwalk.o)
 .debug_abbrev  0x00000000000027b8      0x1d9 /opt/toolchains/n64/mips64-elf/mips64-elf/lib/libc.a(lib_a-fwrite.o)
 .debug_abbrev  0x0000000000002991      0x166 /opt/toolchains/n64/mips64-elf/mips64-elf/lib/libc.a(lib_a-impure.o)
 .debug_abbrev  0x0000000000002af7      0x199 /opt/toolchains/n64/mips64-elf/mips64-elf/lib/libc.a(lib_a-makebuf.o)
 .debug_abbrev  0x0000000000002c90      0x196 /opt/toolchains/n64/mips64-elf/mips64-elf/lib/libc.a(lib_a-malloc.o)
 .debug_abbrev  0x0000000000002e26      0x233 /opt/toolchains/n64/mips64-elf/mips64-elf/lib/libc.a(lib_a-mallocr.o)
 .debug_abbrev  0x0000000000003059       0xba /opt/toolchains/n64/mips64-elf/mips64-elf/lib/libc.a(lib_a-memcpy.o)
 .debug_abbrev  0x0000000000003113       0xae /opt/toolchains/n64/mips64-elf/mips64-elf/lib/libc.a(lib_a-memset.o)
 .debug_abbrev  0x00000000000031c1      0x179 /opt/toolchains/n64/mips64-elf/mips64-elf/lib/libc.a(lib_a-mlock.o)
 .debug_abbrev  0x000000000000333a      0x19d /opt/toolchains/n64/mips64-elf/mips64-elf/lib/libc.a(lib_a-openr.o)
 .debug_abbrev  0x00000000000034d7      0x18e /opt/toolchains/n64/mips64-elf/mips64-elf/lib/libc.a(lib_a-realloc.o)
 .debug_abbrev  0x0000000000003665      0x1df /opt/toolchains/n64/mips64-elf/mips64-elf/lib/libc.a(lib_a-reallocr.o)
 .debug_abbrev  0x0000000000003844      0x1e6 /opt/toolchains/n64/mips64-elf/mips64-elf/lib/libc.a(lib_a-reent.o)
 .debug_abbrev  0x0000000000003a2a      0x1ae /opt/toolchains/n64/mips64-elf/mips64-elf/lib/libc.a(lib_a-refill.o)
 .debug_abbrev  0x0000000000003bd8      0x1b0 /opt/toolchains/n64/mips64-elf/mips64-elf/lib/libc.a(lib_a-sbrkr.o)
 .debug_abbrev  0x0000000000003d88      0x1b5 /opt/toolchains/n64/mips64-elf/mips64-elf/lib/libc.a(lib_a-sprintf.o)
 .debug_abbrev  0x0000000000003f3d      0x203 /opt/toolchains/n64/mips64-elf/mips64-elf/lib/libc.a(lib_a-stdio.o)
 .debug_abbrev  0x0000000000004140       0x8d /opt/toolchains/n64/mips64-elf/mips64-elf/lib/libc.a(lib_a-strcmp.o)
 .debug_abbrev  0x00000000000041cd       0x80 /opt/toolchains/n64/mips64-elf/mips64-elf/lib/libc.a(lib_a-strcpy.o)
 .debug_abbrev  0x000000000000424d       0x2a /opt/toolchains/n64/mips64-elf/mips64-elf/lib/libc.a(lib_a-strlen.o)
 .debug_abbrev  0x0000000000004277      0x2df /opt/toolchains/n64/mips64-elf/mips64-elf/lib/libc.a(lib_a-svfprintf.o)
 .debug_abbrev  0x0000000000004556      0x32a /opt/toolchains/n64/mips64-elf/mips64-elf/lib/libc.a(lib_a-vfiprintf.o)
 .debug_abbrev  0x0000000000004880      0x193 /opt/toolchains/n64/mips64-elf/mips64-elf/lib/libc.a(lib_a-writer.o)
 .debug_abbrev  0x0000000000004a13      0x17f /opt/toolchains/n64/mips64-elf/mips64-elf/lib/libc.a(lib_a-wsetup.o)
 .debug_abbrev  0x0000000000004b92       0x3f /opt/toolchains/n64/mips64-elf/mips64-elf/lib/libc.a(lib_a-abort.o)
 .debug_abbrev  0x0000000000004bd1      0x18e /opt/toolchains/n64/mips64-elf/mips64-elf/lib/libc.a(lib_a-closer.o)
 .debug_abbrev  0x0000000000004d5f      0x229 /opt/toolchains/n64/mips64-elf/mips64-elf/lib/libc.a(lib_a-dtoa.o)
 .debug_abbrev  0x0000000000004f88      0x18c /opt/toolchains/n64/mips64-elf/mips64-elf/lib/libc.a(lib_a-flags.o)
 .debug_abbrev  0x0000000000005114      0x1ec /opt/toolchains/n64/mips64-elf/mips64-elf/lib/libc.a(lib_a-fputwc.o)
 .debug_abbrev  0x0000000000005300      0x1a5 /opt/toolchains/n64/mips64-elf/mips64-elf/lib/libc.a(lib_a-fvwrite.o)
 .debug_abbrev  0x00000000000054a5      0x18e /opt/toolchains/n64/mips64-elf/mips64-elf/lib/libc.a(lib_a-isattyr.o)
 .debug_abbrev  0x0000000000005633      0x25e /opt/toolchains/n64/mips64-elf/mips64-elf/lib/libc.a(lib_a-locale.o)
 .debug_abbrev  0x0000000000005891      0x19d /opt/toolchains/n64/mips64-elf/mips64-elf/lib/libc.a(lib_a-lseekr.o)
 .debug_abbrev  0x0000000000005a2e       0xb7 /opt/toolchains/n64/mips64-elf/mips64-elf/lib/libc.a(lib_a-memchr.o)
 .debug_abbrev  0x0000000000005ae5       0x99 /opt/toolchains/n64/mips64-elf/mips64-elf/lib/libc.a(lib_a-memmove.o)
 .debug_abbrev  0x0000000000005b7e      0x30e /opt/toolchains/n64/mips64-elf/mips64-elf/lib/libc.a(lib_a-mprec.o)
 .debug_abbrev  0x0000000000005e8c      0x18e /opt/toolchains/n64/mips64-elf/mips64-elf/lib/libc.a(lib_a-readr.o)
 .debug_abbrev  0x000000000000601a      0x238 /opt/toolchains/n64/mips64-elf/mips64-elf/lib/libc.a(lib_a-signal.o)
 .debug_abbrev  0x0000000000006252      0x1ca /opt/toolchains/n64/mips64-elf/mips64-elf/lib/libc.a(lib_a-signalr.o)
 .debug_abbrev  0x000000000000641c      0x25e /opt/toolchains/n64/mips64-elf/mips64-elf/lib/libc.a(lib_a-svfiprintf.o)
 .debug_abbrev  0x000000000000667a      0x1a7 /opt/toolchains/n64/mips64-elf/mips64-elf/lib/libc.a(lib_a-wbuf.o)
 .debug_abbrev  0x0000000000006821      0x1ae /opt/toolchains/n64/mips64-elf/mips64-elf/lib/libc.a(lib_a-wcrtomb.o)
 .debug_abbrev  0x00000000000069cf      0x1e5 /opt/toolchains/n64/mips64-elf/mips64-elf/lib/libc.a(lib_a-wctomb_r.o)
 .debug_abbrev  0x0000000000006bb4      0x1ba /opt/toolchains/n64/mips64-elf/mips64-elf/lib/libc.a(lib_a-callocr.o)
 .debug_abbrev  0x0000000000006d6e       0x52 /opt/toolchains/n64/mips64-elf/mips64-elf/lib/libnosys.a(_exit.o)

.debug_loc      0x0000000000000000     0xf6c1
 .debug_loc     0x0000000000000000       0x90 /opt/toolchains/n64/mips64-elf/mips64-elf/lib/libm.a(lib_a-s_sin.o)
 .debug_loc     0x0000000000000090       0xbd /opt/toolchains/n64/mips64-elf/mips64-elf/lib/libm.a(lib_a-w_pow.o)
 .debug_loc     0x000000000000014d      0xd9d /opt/toolchains/n64/mips64-elf/mips64-elf/lib/libm.a(lib_a-e_pow.o)
 .debug_loc     0x0000000000000eea      0x367 /opt/toolchains/n64/mips64-elf/mips64-elf/lib/libm.a(lib_a-e_rem_pio2.o)
 .debug_loc     0x0000000000001251      0x432 /opt/toolchains/n64/mips64-elf/mips64-elf/lib/libm.a(lib_a-e_sqrt.o)
 .debug_loc     0x0000000000001683      0x12e /opt/toolchains/n64/mips64-elf/mips64-elf/lib/libm.a(lib_a-k_cos.o)
 .debug_loc     0x00000000000017b1      0x573 /opt/toolchains/n64/mips64-elf/mips64-elf/lib/libm.a(lib_a-k_rem_pio2.o)
 .debug_loc     0x0000000000001d24       0xbf /opt/toolchains/n64/mips64-elf/mips64-elf/lib/libm.a(lib_a-k_sin.o)
 .debug_loc     0x0000000000001de3       0x3a /opt/toolchains/n64/mips64-elf/mips64-elf/lib/libm.a(lib_a-s_fabs.o)
 .debug_loc     0x0000000000001e1d       0x13 /opt/toolchains/n64/mips64-elf/mips64-elf/lib/libm.a(lib_a-s_finite.o)
 .debug_loc     0x0000000000001e30      0x1d1 /opt/toolchains/n64/mips64-elf/mips64-elf/lib/libm.a(lib_a-s_floor.o)
 .debug_loc     0x0000000000002001       0x33 /opt/toolchains/n64/mips64-elf/mips64-elf/lib/libm.a(lib_a-s_fpclassify.o)
 .debug_loc     0x0000000000002034       0x1c /opt/toolchains/n64/mips64-elf/mips64-elf/lib/libm.a(lib_a-s_nan.o)
 .debug_loc     0x0000000000002050      0x283 /opt/toolchains/n64/mips64-elf/mips64-elf/lib/libm.a(lib_a-s_rint.o)
 .debug_loc     0x00000000000022d3      0x200 /opt/toolchains/n64/mips64-elf/mips64-elf/lib/libm.a(lib_a-s_scalbn.o)
 .debug_loc     0x00000000000024d3       0x60 /opt/toolchains/n64/mips64-elf/mips64-elf/lib/libm.a(lib_a-s_copysign.o)
 .debug_loc     0x0000000000002533      0x129 /opt/toolchains/n64/mips64-elf/mips64-elf/lib/libc.a(lib_a-assert.o)
 .debug_loc     0x000000000000265c       0xf1 /opt/toolchains/n64/mips64-elf/mips64-elf/lib/libc.a(lib_a-fclose.o)
 .debug_loc     0x000000000000274d      0x28b /opt/toolchains/n64/mips64-elf/mips64-elf/lib/libc.a(lib_a-fflush.o)
 .debug_loc     0x00000000000029d8      0x216 /opt/toolchains/n64/mips64-elf/mips64-elf/lib/libc.a(lib_a-findfp.o)
 .debug_loc     0x0000000000002bee       0xb5 /opt/toolchains/n64/mips64-elf/mips64-elf/lib/libc.a(lib_a-fiprintf.o)
 .debug_loc     0x0000000000002ca3      0x169 /opt/toolchains/n64/mips64-elf/mips64-elf/lib/libc.a(lib_a-fopen.o)
 .debug_loc     0x0000000000002e0c      0x3b6 /opt/toolchains/n64/mips64-elf/mips64-elf/lib/libc.a(lib_a-fread.o)
 .debug_loc     0x00000000000031c2      0x3b8 /opt/toolchains/n64/mips64-elf/mips64-elf/lib/libc.a(lib_a-freer.o)
 .debug_loc     0x000000000000357a      0x371 /opt/toolchains/n64/mips64-elf/mips64-elf/lib/libc.a(lib_a-fseek.o)
 .debug_loc     0x00000000000038eb       0x7a /opt/toolchains/n64/mips64-elf/mips64-elf/lib/libc.a(lib_a-fstatr.o)
 .debug_loc     0x0000000000003965       0xcf /opt/toolchains/n64/mips64-elf/mips64-elf/lib/libc.a(lib_a-ftell.o)
 .debug_loc     0x0000000000003a34      0x18f /opt/toolchains/n64/mips64-elf/mips64-elf/lib/libc.a(lib_a-fwalk.o)
 .debug_loc     0x0000000000003bc3      0x188 /opt/toolchains/n64/mips64-elf/mips64-elf/lib/libc.a(lib_a-fwrite.o)
 .debug_loc     0x0000000000003d4b      0x159 /opt/toolchains/n64/mips64-elf/mips64-elf/lib/libc.a(lib_a-makebuf.o)
 .debug_loc     0x0000000000003ea4       0x3c /opt/toolchains/n64/mips64-elf/mips64-elf/lib/libc.a(lib_a-malloc.o)
 .debug_loc     0x0000000000003ee0      0x9d5 /opt/toolchains/n64/mips64-elf/mips64-elf/lib/libc.a(lib_a-mallocr.o)
 .debug_loc     0x00000000000048b5      0x31e /opt/toolchains/n64/mips64-elf/mips64-elf/lib/libc.a(lib_a-memcpy.o)
 .debug_loc     0x0000000000004bd3      0x166 /opt/toolchains/n64/mips64-elf/mips64-elf/lib/libc.a(lib_a-memset.o)
 .debug_loc     0x0000000000004d39       0x98 /opt/toolchains/n64/mips64-elf/mips64-elf/lib/libc.a(lib_a-openr.o)
 .debug_loc     0x0000000000004dd1       0x3c /opt/toolchains/n64/mips64-elf/mips64-elf/lib/libc.a(lib_a-realloc.o)
 .debug_loc     0x0000000000004e0d      0xd57 /opt/toolchains/n64/mips64-elf/mips64-elf/lib/libc.a(lib_a-reallocr.o)
 .debug_loc     0x0000000000005b64      0x1e5 /opt/toolchains/n64/mips64-elf/mips64-elf/lib/libc.a(lib_a-reent.o)
 .debug_loc     0x0000000000005d49       0xc5 /opt/toolchains/n64/mips64-elf/mips64-elf/lib/libc.a(lib_a-refill.o)
 .debug_loc     0x0000000000005e0e       0x5c /opt/toolchains/n64/mips64-elf/mips64-elf/lib/libc.a(lib_a-sbrkr.o)
 .debug_loc     0x0000000000005e6a       0xcd /opt/toolchains/n64/mips64-elf/mips64-elf/lib/libc.a(lib_a-sprintf.o)
 .debug_loc     0x0000000000005f37      0x241 /opt/toolchains/n64/mips64-elf/mips64-elf/lib/libc.a(lib_a-stdio.o)
 .debug_loc     0x0000000000006178       0x8e /opt/toolchains/n64/mips64-elf/mips64-elf/lib/libc.a(lib_a-strcmp.o)
 .debug_loc     0x0000000000006206      0x12c /opt/toolchains/n64/mips64-elf/mips64-elf/lib/libc.a(lib_a-strcpy.o)
 .debug_loc     0x0000000000006332     0x21be /opt/toolchains/n64/mips64-elf/mips64-elf/lib/libc.a(lib_a-svfprintf.o)
 .debug_loc     0x00000000000084f0     0x1317 /opt/toolchains/n64/mips64-elf/mips64-elf/lib/libc.a(lib_a-vfiprintf.o)
 .debug_loc     0x0000000000009807       0x98 /opt/toolchains/n64/mips64-elf/mips64-elf/lib/libc.a(lib_a-writer.o)
 .debug_loc     0x000000000000989f       0x72 /opt/toolchains/n64/mips64-elf/mips64-elf/lib/libc.a(lib_a-wsetup.o)
 .debug_loc     0x0000000000009911       0x20 /opt/toolchains/n64/mips64-elf/mips64-elf/lib/libc.a(lib_a-abort.o)
 .debug_loc     0x0000000000009931       0x5c /opt/toolchains/n64/mips64-elf/mips64-elf/lib/libc.a(lib_a-closer.o)
 .debug_loc     0x000000000000998d     0x1d17 /opt/toolchains/n64/mips64-elf/mips64-elf/lib/libc.a(lib_a-dtoa.o)
 .debug_loc     0x000000000000b6a4       0xb6 /opt/toolchains/n64/mips64-elf/mips64-elf/lib/libc.a(lib_a-flags.o)
 .debug_loc     0x000000000000b75a      0x26d /opt/toolchains/n64/mips64-elf/mips64-elf/lib/libc.a(lib_a-fputwc.o)
 .debug_loc     0x000000000000b9c7      0x4f6 /opt/toolchains/n64/mips64-elf/mips64-elf/lib/libc.a(lib_a-fvwrite.o)
 .debug_loc     0x000000000000bebd       0x5c /opt/toolchains/n64/mips64-elf/mips64-elf/lib/libc.a(lib_a-isattyr.o)
 .debug_loc     0x000000000000bf19       0x95 /opt/toolchains/n64/mips64-elf/mips64-elf/lib/libc.a(lib_a-locale.o)
 .debug_loc     0x000000000000bfae       0x98 /opt/toolchains/n64/mips64-elf/mips64-elf/lib/libc.a(lib_a-lseekr.o)
 .debug_loc     0x000000000000c046      0x141 /opt/toolchains/n64/mips64-elf/mips64-elf/lib/libc.a(lib_a-memchr.o)
 .debug_loc     0x000000000000c187      0x21f /opt/toolchains/n64/mips64-elf/mips64-elf/lib/libc.a(lib_a-memmove.o)
 .debug_loc     0x000000000000c3a6     0x1712 /opt/toolchains/n64/mips64-elf/mips64-elf/lib/libc.a(lib_a-mprec.o)
 .debug_loc     0x000000000000dab8       0x98 /opt/toolchains/n64/mips64-elf/mips64-elf/lib/libc.a(lib_a-readr.o)
 .debug_loc     0x000000000000db50      0x2b2 /opt/toolchains/n64/mips64-elf/mips64-elf/lib/libc.a(lib_a-signal.o)
 .debug_loc     0x000000000000de02       0x8d /opt/toolchains/n64/mips64-elf/mips64-elf/lib/libc.a(lib_a-signalr.o)
 .debug_loc     0x000000000000de8f     0x129d /opt/toolchains/n64/mips64-elf/mips64-elf/lib/libc.a(lib_a-svfiprintf.o)
 .debug_loc     0x000000000000f12c      0x13d /opt/toolchains/n64/mips64-elf/mips64-elf/lib/libc.a(lib_a-wbuf.o)
 .debug_loc     0x000000000000f269      0x1e3 /opt/toolchains/n64/mips64-elf/mips64-elf/lib/libc.a(lib_a-wcrtomb.o)
 .debug_loc     0x000000000000f44c       0x78 /opt/toolchains/n64/mips64-elf/mips64-elf/lib/libc.a(lib_a-wctomb_r.o)
 .debug_loc     0x000000000000f4c4      0x1fd /opt/toolchains/n64/mips64-elf/mips64-elf/lib/libc.a(lib_a-callocr.o)

.debug_aranges  0x0000000000000000      0x900
 .debug_aranges
                0x0000000000000000       0x20 /opt/toolchains/n64/mips64-elf/mips64-elf/lib/libm.a(lib_a-s_sin.o)
 .debug_aranges
                0x0000000000000020       0x20 /opt/toolchains/n64/mips64-elf/mips64-elf/lib/libm.a(lib_a-w_pow.o)
 .debug_aranges
                0x0000000000000040       0x20 /opt/toolchains/n64/mips64-elf/mips64-elf/lib/libm.a(lib_a-e_pow.o)
 .debug_aranges
                0x0000000000000060       0x20 /opt/toolchains/n64/mips64-elf/mips64-elf/lib/libm.a(lib_a-e_rem_pio2.o)
 .debug_aranges
                0x0000000000000080       0x20 /opt/toolchains/n64/mips64-elf/mips64-elf/lib/libm.a(lib_a-e_sqrt.o)
 .debug_aranges
                0x00000000000000a0       0x20 /opt/toolchains/n64/mips64-elf/mips64-elf/lib/libm.a(lib_a-k_cos.o)
 .debug_aranges
                0x00000000000000c0       0x20 /opt/toolchains/n64/mips64-elf/mips64-elf/lib/libm.a(lib_a-k_rem_pio2.o)
 .debug_aranges
                0x00000000000000e0       0x20 /opt/toolchains/n64/mips64-elf/mips64-elf/lib/libm.a(lib_a-k_sin.o)
 .debug_aranges
                0x0000000000000100       0x20 /opt/toolchains/n64/mips64-elf/mips64-elf/lib/libm.a(lib_a-s_fabs.o)
 .debug_aranges
                0x0000000000000120       0x20 /opt/toolchains/n64/mips64-elf/mips64-elf/lib/libm.a(lib_a-s_finite.o)
 .debug_aranges
                0x0000000000000140       0x20 /opt/toolchains/n64/mips64-elf/mips64-elf/lib/libm.a(lib_a-s_floor.o)
 .debug_aranges
                0x0000000000000160       0x20 /opt/toolchains/n64/mips64-elf/mips64-elf/lib/libm.a(lib_a-s_fpclassify.o)
 .debug_aranges
                0x0000000000000180       0x20 /opt/toolchains/n64/mips64-elf/mips64-elf/lib/libm.a(lib_a-s_matherr.o)
 .debug_aranges
                0x00000000000001a0       0x20 /opt/toolchains/n64/mips64-elf/mips64-elf/lib/libm.a(lib_a-s_nan.o)
 .debug_aranges
                0x00000000000001c0       0x20 /opt/toolchains/n64/mips64-elf/mips64-elf/lib/libm.a(lib_a-s_rint.o)
 .debug_aranges
                0x00000000000001e0       0x20 /opt/toolchains/n64/mips64-elf/mips64-elf/lib/libm.a(lib_a-s_scalbn.o)
 .debug_aranges
                0x0000000000000200       0x20 /opt/toolchains/n64/mips64-elf/mips64-elf/lib/libm.a(lib_a-s_copysign.o)
 .debug_aranges
                0x0000000000000220       0x20 /opt/toolchains/n64/mips64-elf/mips64-elf/lib/libc.a(lib_a-assert.o)
 .debug_aranges
                0x0000000000000240       0x20 /opt/toolchains/n64/mips64-elf/mips64-elf/lib/libc.a(lib_a-errno.o)
 .debug_aranges
                0x0000000000000260       0x20 /opt/toolchains/n64/mips64-elf/mips64-elf/lib/libc.a(lib_a-fclose.o)
 .debug_aranges
                0x0000000000000280       0x20 /opt/toolchains/n64/mips64-elf/mips64-elf/lib/libc.a(lib_a-fflush.o)
 .debug_aranges
                0x00000000000002a0       0x20 /opt/toolchains/n64/mips64-elf/mips64-elf/lib/libc.a(lib_a-findfp.o)
 .debug_aranges
                0x00000000000002c0       0x20 /opt/toolchains/n64/mips64-elf/mips64-elf/lib/libc.a(lib_a-fiprintf.o)
 .debug_aranges
                0x00000000000002e0       0x20 /opt/toolchains/n64/mips64-elf/mips64-elf/lib/libc.a(lib_a-fopen.o)
 .debug_aranges
                0x0000000000000300       0x20 /opt/toolchains/n64/mips64-elf/mips64-elf/lib/libc.a(lib_a-fread.o)
 .debug_aranges
                0x0000000000000320       0x20 /opt/toolchains/n64/mips64-elf/mips64-elf/lib/libc.a(lib_a-freer.o)
 .debug_aranges
                0x0000000000000340       0x20 /opt/toolchains/n64/mips64-elf/mips64-elf/lib/libc.a(lib_a-fseek.o)
 .debug_aranges
                0x0000000000000360       0x20 /opt/toolchains/n64/mips64-elf/mips64-elf/lib/libc.a(lib_a-fstatr.o)
 .debug_aranges
                0x0000000000000380       0x20 /opt/toolchains/n64/mips64-elf/mips64-elf/lib/libc.a(lib_a-ftell.o)
 .debug_aranges
                0x00000000000003a0       0x20 /opt/toolchains/n64/mips64-elf/mips64-elf/lib/libc.a(lib_a-fwalk.o)
 .debug_aranges
                0x00000000000003c0       0x20 /opt/toolchains/n64/mips64-elf/mips64-elf/lib/libc.a(lib_a-fwrite.o)
 .debug_aranges
                0x00000000000003e0       0x20 /opt/toolchains/n64/mips64-elf/mips64-elf/lib/libc.a(lib_a-makebuf.o)
 .debug_aranges
                0x0000000000000400       0x20 /opt/toolchains/n64/mips64-elf/mips64-elf/lib/libc.a(lib_a-malloc.o)
 .debug_aranges
                0x0000000000000420       0x20 /opt/toolchains/n64/mips64-elf/mips64-elf/lib/libc.a(lib_a-mallocr.o)
 .debug_aranges
                0x0000000000000440       0x20 /opt/toolchains/n64/mips64-elf/mips64-elf/lib/libc.a(lib_a-memcpy.o)
 .debug_aranges
                0x0000000000000460       0x20 /opt/toolchains/n64/mips64-elf/mips64-elf/lib/libc.a(lib_a-memset.o)
 .debug_aranges
                0x0000000000000480       0x20 /opt/toolchains/n64/mips64-elf/mips64-elf/lib/libc.a(lib_a-mlock.o)
 .debug_aranges
                0x00000000000004a0       0x20 /opt/toolchains/n64/mips64-elf/mips64-elf/lib/libc.a(lib_a-openr.o)
 .debug_aranges
                0x00000000000004c0       0x20 /opt/toolchains/n64/mips64-elf/mips64-elf/lib/libc.a(lib_a-realloc.o)
 .debug_aranges
                0x00000000000004e0       0x20 /opt/toolchains/n64/mips64-elf/mips64-elf/lib/libc.a(lib_a-reallocr.o)
 .debug_aranges
                0x0000000000000500       0x20 /opt/toolchains/n64/mips64-elf/mips64-elf/lib/libc.a(lib_a-reent.o)
 .debug_aranges
                0x0000000000000520       0x20 /opt/toolchains/n64/mips64-elf/mips64-elf/lib/libc.a(lib_a-refill.o)
 .debug_aranges
                0x0000000000000540       0x20 /opt/toolchains/n64/mips64-elf/mips64-elf/lib/libc.a(lib_a-sbrkr.o)
 .debug_aranges
                0x0000000000000560       0x20 /opt/toolchains/n64/mips64-elf/mips64-elf/lib/libc.a(lib_a-sprintf.o)
 .debug_aranges
                0x0000000000000580       0x20 /opt/toolchains/n64/mips64-elf/mips64-elf/lib/libc.a(lib_a-stdio.o)
 .debug_aranges
                0x00000000000005a0       0x20 /opt/toolchains/n64/mips64-elf/mips64-elf/lib/libc.a(lib_a-strcmp.o)
 .debug_aranges
                0x00000000000005c0       0x20 /opt/toolchains/n64/mips64-elf/mips64-elf/lib/libc.a(lib_a-strcpy.o)
 .debug_aranges
                0x00000000000005e0       0x20 /opt/toolchains/n64/mips64-elf/mips64-elf/lib/libc.a(lib_a-svfprintf.o)
 .debug_aranges
                0x0000000000000600       0x20 /opt/toolchains/n64/mips64-elf/mips64-elf/lib/libc.a(lib_a-vfiprintf.o)
 .debug_aranges
                0x0000000000000620       0x20 /opt/toolchains/n64/mips64-elf/mips64-elf/lib/libc.a(lib_a-writer.o)
 .debug_aranges
                0x0000000000000640       0x20 /opt/toolchains/n64/mips64-elf/mips64-elf/lib/libc.a(lib_a-wsetup.o)
 .debug_aranges
                0x0000000000000660       0x20 /opt/toolchains/n64/mips64-elf/mips64-elf/lib/libc.a(lib_a-abort.o)
 .debug_aranges
                0x0000000000000680       0x20 /opt/toolchains/n64/mips64-elf/mips64-elf/lib/libc.a(lib_a-closer.o)
 .debug_aranges
                0x00000000000006a0       0x20 /opt/toolchains/n64/mips64-elf/mips64-elf/lib/libc.a(lib_a-dtoa.o)
 .debug_aranges
                0x00000000000006c0       0x20 /opt/toolchains/n64/mips64-elf/mips64-elf/lib/libc.a(lib_a-flags.o)
 .debug_aranges
                0x00000000000006e0       0x20 /opt/toolchains/n64/mips64-elf/mips64-elf/lib/libc.a(lib_a-fputwc.o)
 .debug_aranges
                0x0000000000000700       0x20 /opt/toolchains/n64/mips64-elf/mips64-elf/lib/libc.a(lib_a-fvwrite.o)
 .debug_aranges
                0x0000000000000720       0x20 /opt/toolchains/n64/mips64-elf/mips64-elf/lib/libc.a(lib_a-isattyr.o)
 .debug_aranges
                0x0000000000000740       0x20 /opt/toolchains/n64/mips64-elf/mips64-elf/lib/libc.a(lib_a-locale.o)
 .debug_aranges
                0x0000000000000760       0x20 /opt/toolchains/n64/mips64-elf/mips64-elf/lib/libc.a(lib_a-lseekr.o)
 .debug_aranges
                0x0000000000000780       0x20 /opt/toolchains/n64/mips64-elf/mips64-elf/lib/libc.a(lib_a-memchr.o)
 .debug_aranges
                0x00000000000007a0       0x20 /opt/toolchains/n64/mips64-elf/mips64-elf/lib/libc.a(lib_a-memmove.o)
 .debug_aranges
                0x00000000000007c0       0x20 /opt/toolchains/n64/mips64-elf/mips64-elf/lib/libc.a(lib_a-mprec.o)
 .debug_aranges
                0x00000000000007e0       0x20 /opt/toolchains/n64/mips64-elf/mips64-elf/lib/libc.a(lib_a-readr.o)
 .debug_aranges
                0x0000000000000800       0x20 /opt/toolchains/n64/mips64-elf/mips64-elf/lib/libc.a(lib_a-signal.o)
 .debug_aranges
                0x0000000000000820       0x20 /opt/toolchains/n64/mips64-elf/mips64-elf/lib/libc.a(lib_a-signalr.o)
 .debug_aranges
                0x0000000000000840       0x20 /opt/toolchains/n64/mips64-elf/mips64-elf/lib/libc.a(lib_a-svfiprintf.o)
 .debug_aranges
                0x0000000000000860       0x20 /opt/toolchains/n64/mips64-elf/mips64-elf/lib/libc.a(lib_a-wbuf.o)
 .debug_aranges
                0x0000000000000880       0x20 /opt/toolchains/n64/mips64-elf/mips64-elf/lib/libc.a(lib_a-wcrtomb.o)
 .debug_aranges
                0x00000000000008a0       0x20 /opt/toolchains/n64/mips64-elf/mips64-elf/lib/libc.a(lib_a-wctomb_r.o)
 .debug_aranges
                0x00000000000008c0       0x20 /opt/toolchains/n64/mips64-elf/mips64-elf/lib/libc.a(lib_a-callocr.o)
 .debug_aranges
                0x00000000000008e0       0x20 /opt/toolchains/n64/mips64-elf/mips64-elf/lib/libnosys.a(_exit.o)

.debug_line     0x0000000000000000     0x926d
 .debug_line    0x0000000000000000      0x18c /opt/toolchains/n64/mips64-elf/mips64-elf/lib/libm.a(lib_a-s_sin.o)
 .debug_line    0x000000000000018c      0x182 /opt/toolchains/n64/mips64-elf/mips64-elf/lib/libm.a(lib_a-w_pow.o)
 .debug_line    0x000000000000030e      0x2f2 /opt/toolchains/n64/mips64-elf/mips64-elf/lib/libm.a(lib_a-e_pow.o)
 .debug_line    0x0000000000000600      0x1c6 /opt/toolchains/n64/mips64-elf/mips64-elf/lib/libm.a(lib_a-e_rem_pio2.o)
 .debug_line    0x00000000000007c6      0x1a4 /opt/toolchains/n64/mips64-elf/mips64-elf/lib/libm.a(lib_a-e_sqrt.o)
 .debug_line    0x000000000000096a      0x135 /opt/toolchains/n64/mips64-elf/mips64-elf/lib/libm.a(lib_a-k_cos.o)
 .debug_line    0x0000000000000a9f      0x39b /opt/toolchains/n64/mips64-elf/mips64-elf/lib/libm.a(lib_a-k_rem_pio2.o)
 .debug_line    0x0000000000000e3a      0x120 /opt/toolchains/n64/mips64-elf/mips64-elf/lib/libm.a(lib_a-k_sin.o)
 .debug_line    0x0000000000000f5a      0x160 /opt/toolchains/n64/mips64-elf/mips64-elf/lib/libm.a(lib_a-s_fabs.o)
 .debug_line    0x00000000000010ba      0x129 /opt/toolchains/n64/mips64-elf/mips64-elf/lib/libm.a(lib_a-s_finite.o)
 .debug_line    0x00000000000011e3      0x199 /opt/toolchains/n64/mips64-elf/mips64-elf/lib/libm.a(lib_a-s_floor.o)
 .debug_line    0x000000000000137c      0x15d /opt/toolchains/n64/mips64-elf/mips64-elf/lib/libm.a(lib_a-s_fpclassify.o)
 .debug_line    0x00000000000014d9       0x6c /opt/toolchains/n64/mips64-elf/mips64-elf/lib/libm.a(lib_a-s_lib_ver.o)
 .debug_line    0x0000000000001545       0xbc /opt/toolchains/n64/mips64-elf/mips64-elf/lib/libm.a(lib_a-s_matherr.o)
 .debug_line    0x0000000000001601      0x126 /opt/toolchains/n64/mips64-elf/mips64-elf/lib/libm.a(lib_a-s_nan.o)
 .debug_line    0x0000000000001727      0x16a /opt/toolchains/n64/mips64-elf/mips64-elf/lib/libm.a(lib_a-s_rint.o)
 .debug_line    0x0000000000001891      0x197 /opt/toolchains/n64/mips64-elf/mips64-elf/lib/libm.a(lib_a-s_scalbn.o)
 .debug_line    0x0000000000001a28      0x131 /opt/toolchains/n64/mips64-elf/mips64-elf/lib/libm.a(lib_a-s_copysign.o)
 .debug_line    0x0000000000001b59      0x187 /opt/toolchains/n64/mips64-elf/mips64-elf/lib/libc.a(lib_a-assert.o)
 .debug_line    0x0000000000001ce0      0x128 /opt/toolchains/n64/mips64-elf/mips64-elf/lib/libc.a(lib_a-errno.o)
 .debug_line    0x0000000000001e08      0x1b4 /opt/toolchains/n64/mips64-elf/mips64-elf/lib/libc.a(lib_a-fclose.o)
 .debug_line    0x0000000000001fbc      0x24e /opt/toolchains/n64/mips64-elf/mips64-elf/lib/libc.a(lib_a-fflush.o)
 .debug_line    0x000000000000220a      0x220 /opt/toolchains/n64/mips64-elf/mips64-elf/lib/libc.a(lib_a-findfp.o)
 .debug_line    0x000000000000242a      0x18a /opt/toolchains/n64/mips64-elf/mips64-elf/lib/libc.a(lib_a-fiprintf.o)
 .debug_line    0x00000000000025b4      0x19d /opt/toolchains/n64/mips64-elf/mips64-elf/lib/libc.a(lib_a-fopen.o)
 .debug_line    0x0000000000002751      0x22f /opt/toolchains/n64/mips64-elf/mips64-elf/lib/libc.a(lib_a-fread.o)
 .debug_line    0x0000000000002980      0x22c /opt/toolchains/n64/mips64-elf/mips64-elf/lib/libc.a(lib_a-freer.o)
 .debug_line    0x0000000000002bac      0x2a5 /opt/toolchains/n64/mips64-elf/mips64-elf/lib/libc.a(lib_a-fseek.o)
 .debug_line    0x0000000000002e51      0x18f /opt/toolchains/n64/mips64-elf/mips64-elf/lib/libc.a(lib_a-fstatr.o)
 .debug_line    0x0000000000002fe0      0x1b0 /opt/toolchains/n64/mips64-elf/mips64-elf/lib/libc.a(lib_a-ftell.o)
 .debug_line    0x0000000000003190      0x1af /opt/toolchains/n64/mips64-elf/mips64-elf/lib/libc.a(lib_a-fwalk.o)
 .debug_line    0x000000000000333f      0x1b3 /opt/toolchains/n64/mips64-elf/mips64-elf/lib/libc.a(lib_a-fwrite.o)
 .debug_line    0x00000000000034f2      0x10e /opt/toolchains/n64/mips64-elf/mips64-elf/lib/libc.a(lib_a-impure.o)
 .debug_line    0x0000000000003600      0x1f7 /opt/toolchains/n64/mips64-elf/mips64-elf/lib/libc.a(lib_a-makebuf.o)
 .debug_line    0x00000000000037f7      0x175 /opt/toolchains/n64/mips64-elf/mips64-elf/lib/libc.a(lib_a-malloc.o)
 .debug_line    0x000000000000396c      0x361 /opt/toolchains/n64/mips64-elf/mips64-elf/lib/libc.a(lib_a-mallocr.o)
 .debug_line    0x0000000000003ccd      0x111 /opt/toolchains/n64/mips64-elf/mips64-elf/lib/libc.a(lib_a-memcpy.o)
 .debug_line    0x0000000000003dde      0x171 /opt/toolchains/n64/mips64-elf/mips64-elf/lib/libc.a(lib_a-memset.o)
 .debug_line    0x0000000000003f4f      0x120 /opt/toolchains/n64/mips64-elf/mips64-elf/lib/libc.a(lib_a-mlock.o)
 .debug_line    0x000000000000406f      0x178 /opt/toolchains/n64/mips64-elf/mips64-elf/lib/libc.a(lib_a-openr.o)
 .debug_line    0x00000000000041e7      0x174 /opt/toolchains/n64/mips64-elf/mips64-elf/lib/libc.a(lib_a-realloc.o)
 .debug_line    0x000000000000435b      0x2c7 /opt/toolchains/n64/mips64-elf/mips64-elf/lib/libc.a(lib_a-reallocr.o)
 .debug_line    0x0000000000004622      0x172 /opt/toolchains/n64/mips64-elf/mips64-elf/lib/libc.a(lib_a-reent.o)
 .debug_line    0x0000000000004794      0x1ff /opt/toolchains/n64/mips64-elf/mips64-elf/lib/libc.a(lib_a-refill.o)
 .debug_line    0x0000000000004993      0x178 /opt/toolchains/n64/mips64-elf/mips64-elf/lib/libc.a(lib_a-sbrkr.o)
 .debug_line    0x0000000000004b0b      0x1b5 /opt/toolchains/n64/mips64-elf/mips64-elf/lib/libc.a(lib_a-sprintf.o)
 .debug_line    0x0000000000004cc0      0x1aa /opt/toolchains/n64/mips64-elf/mips64-elf/lib/libc.a(lib_a-stdio.o)
 .debug_line    0x0000000000004e6a       0xe3 /opt/toolchains/n64/mips64-elf/mips64-elf/lib/libc.a(lib_a-strcmp.o)
 .debug_line    0x0000000000004f4d       0xd7 /opt/toolchains/n64/mips64-elf/mips64-elf/lib/libc.a(lib_a-strcpy.o)
 .debug_line    0x0000000000005024       0x1d /opt/toolchains/n64/mips64-elf/mips64-elf/lib/libc.a(lib_a-strlen.o)
 .debug_line    0x0000000000005041      0x8fc /opt/toolchains/n64/mips64-elf/mips64-elf/lib/libc.a(lib_a-svfprintf.o)
 .debug_line    0x000000000000593d      0x673 /opt/toolchains/n64/mips64-elf/mips64-elf/lib/libc.a(lib_a-vfiprintf.o)
 .debug_line    0x0000000000005fb0      0x179 /opt/toolchains/n64/mips64-elf/mips64-elf/lib/libc.a(lib_a-writer.o)
 .debug_line    0x0000000000006129      0x1d1 /opt/toolchains/n64/mips64-elf/mips64-elf/lib/libc.a(lib_a-wsetup.o)
 .debug_line    0x00000000000062fa       0xba /opt/toolchains/n64/mips64-elf/mips64-elf/lib/libc.a(lib_a-abort.o)
 .debug_line    0x00000000000063b4      0x179 /opt/toolchains/n64/mips64-elf/mips64-elf/lib/libc.a(lib_a-closer.o)
 .debug_line    0x000000000000652d      0x71a /opt/toolchains/n64/mips64-elf/mips64-elf/lib/libc.a(lib_a-dtoa.o)
 .debug_line    0x0000000000006c47      0x147 /opt/toolchains/n64/mips64-elf/mips64-elf/lib/libc.a(lib_a-flags.o)
 .debug_line    0x0000000000006d8e      0x1e0 /opt/toolchains/n64/mips64-elf/mips64-elf/lib/libc.a(lib_a-fputwc.o)
 .debug_line    0x0000000000006f6e      0x2b0 /opt/toolchains/n64/mips64-elf/mips64-elf/lib/libc.a(lib_a-fvwrite.o)
 .debug_line    0x000000000000721e      0x17a /opt/toolchains/n64/mips64-elf/mips64-elf/lib/libc.a(lib_a-isattyr.o)
 .debug_line    0x0000000000007398      0x1b6 /opt/toolchains/n64/mips64-elf/mips64-elf/lib/libc.a(lib_a-locale.o)
 .debug_line    0x000000000000754e      0x179 /opt/toolchains/n64/mips64-elf/mips64-elf/lib/libc.a(lib_a-lseekr.o)
 .debug_line    0x00000000000076c7      0x140 /opt/toolchains/n64/mips64-elf/mips64-elf/lib/libc.a(lib_a-memchr.o)
 .debug_line    0x0000000000007807      0x181 /opt/toolchains/n64/mips64-elf/mips64-elf/lib/libc.a(lib_a-memmove.o)
 .debug_line    0x0000000000007988      0x67c /opt/toolchains/n64/mips64-elf/mips64-elf/lib/libc.a(lib_a-mprec.o)
 .debug_line    0x0000000000008004      0x178 /opt/toolchains/n64/mips64-elf/mips64-elf/lib/libc.a(lib_a-readr.o)
 .debug_line    0x000000000000817c      0x200 /opt/toolchains/n64/mips64-elf/mips64-elf/lib/libc.a(lib_a-signal.o)
 .debug_line    0x000000000000837c      0x17f /opt/toolchains/n64/mips64-elf/mips64-elf/lib/libc.a(lib_a-signalr.o)
 .debug_line    0x00000000000084fb      0x680 /opt/toolchains/n64/mips64-elf/mips64-elf/lib/libc.a(lib_a-svfiprintf.o)
 .debug_line    0x0000000000008b7b      0x1fa /opt/toolchains/n64/mips64-elf/mips64-elf/lib/libc.a(lib_a-wbuf.o)
 .debug_line    0x0000000000008d75      0x1a4 /opt/toolchains/n64/mips64-elf/mips64-elf/lib/libc.a(lib_a-wcrtomb.o)
 .debug_line    0x0000000000008f19      0x198 /opt/toolchains/n64/mips64-elf/mips64-elf/lib/libc.a(lib_a-wctomb_r.o)
 .debug_line    0x00000000000090b1      0x159 /opt/toolchains/n64/mips64-elf/mips64-elf/lib/libc.a(lib_a-callocr.o)
 .debug_line    0x000000000000920a       0x63 /opt/toolchains/n64/mips64-elf/mips64-elf/lib/libnosys.a(_exit.o)

.debug_str      0x0000000000000000     0x27b3
 .debug_str     0x0000000000000000      0x139 /opt/toolchains/n64/mips64-elf/mips64-elf/lib/libm.a(lib_a-s_sin.o)
                                        0x17f (size before relaxing)
 .debug_str     0x0000000000000139       0xb1 /opt/toolchains/n64/mips64-elf/mips64-elf/lib/libm.a(lib_a-w_pow.o)
                                        0x1c2 (size before relaxing)
 .debug_str     0x00000000000001ea       0xa5 /opt/toolchains/n64/mips64-elf/mips64-elf/lib/libm.a(lib_a-e_pow.o)
                                        0x1ee (size before relaxing)
 .debug_str     0x000000000000028f       0xad /opt/toolchains/n64/mips64-elf/mips64-elf/lib/libm.a(lib_a-e_rem_pio2.o)
                                        0x200 (size before relaxing)
 .debug_str     0x000000000000033c       0x4b /opt/toolchains/n64/mips64-elf/mips64-elf/lib/libm.a(lib_a-e_sqrt.o)
                                        0x19e (size before relaxing)
 .debug_str     0x0000000000000387       0x43 /opt/toolchains/n64/mips64-elf/mips64-elf/lib/libm.a(lib_a-k_cos.o)
                                        0x191 (size before relaxing)
 .debug_str     0x00000000000003ca       0x77 /opt/toolchains/n64/mips64-elf/mips64-elf/lib/libm.a(lib_a-k_rem_pio2.o)
                                        0x19d (size before relaxing)
 .debug_str     0x0000000000000441       0x43 /opt/toolchains/n64/mips64-elf/mips64-elf/lib/libm.a(lib_a-k_sin.o)
                                        0x191 (size before relaxing)
 .debug_str     0x0000000000000484       0x3c /opt/toolchains/n64/mips64-elf/mips64-elf/lib/libm.a(lib_a-s_fabs.o)
                                        0x185 (size before relaxing)
 .debug_str     0x00000000000004c0       0xa2 /opt/toolchains/n64/mips64-elf/mips64-elf/lib/libm.a(lib_a-s_finite.o)
                                        0x18d (size before relaxing)
 .debug_str     0x0000000000000562       0x3e /opt/toolchains/n64/mips64-elf/mips64-elf/lib/libm.a(lib_a-s_floor.o)
                                        0x191 (size before relaxing)
 .debug_str     0x00000000000005a0       0x4d /opt/toolchains/n64/mips64-elf/mips64-elf/lib/libm.a(lib_a-s_fpclassify.o)
                                        0x18e (size before relaxing)
 .debug_str     0x00000000000005ed       0x3c /opt/toolchains/n64/mips64-elf/mips64-elf/lib/libm.a(lib_a-s_lib_ver.o)
                                        0x1a5 (size before relaxing)
 .debug_str     0x0000000000000629       0x44 /opt/toolchains/n64/mips64-elf/mips64-elf/lib/libm.a(lib_a-s_matherr.o)
                                        0x177 (size before relaxing)
 .debug_str     0x000000000000066d       0x38 /opt/toolchains/n64/mips64-elf/mips64-elf/lib/libm.a(lib_a-s_nan.o)
                                        0x180 (size before relaxing)
 .debug_str     0x00000000000006a5       0x44 /opt/toolchains/n64/mips64-elf/mips64-elf/lib/libm.a(lib_a-s_rint.o)
                                        0x19e (size before relaxing)
 .debug_str     0x00000000000006e9       0x4f /opt/toolchains/n64/mips64-elf/mips64-elf/lib/libm.a(lib_a-s_scalbn.o)
                                        0x1a9 (size before relaxing)
 .debug_str     0x0000000000000738       0x46 /opt/toolchains/n64/mips64-elf/mips64-elf/lib/libm.a(lib_a-s_copysign.o)
                                        0x18c (size before relaxing)
 .debug_str     0x000000000000077e      0x427 /opt/toolchains/n64/mips64-elf/mips64-elf/lib/libc.a(lib_a-assert.o)
                                        0x51a (size before relaxing)
 .debug_str     0x0000000000000ba5       0x9e /opt/toolchains/n64/mips64-elf/mips64-elf/lib/libc.a(lib_a-errno.o)
                                        0x4ee (size before relaxing)
 .debug_str     0x0000000000000c43       0xad /opt/toolchains/n64/mips64-elf/mips64-elf/lib/libc.a(lib_a-fclose.o)
                                        0x502 (size before relaxing)
 .debug_str     0x0000000000000cf0       0x78 /opt/toolchains/n64/mips64-elf/mips64-elf/lib/libc.a(lib_a-fflush.o)
                                        0x533 (size before relaxing)
 .debug_str     0x0000000000000d68      0x100 /opt/toolchains/n64/mips64-elf/mips64-elf/lib/libc.a(lib_a-findfp.o)
                                        0x5e0 (size before relaxing)
 .debug_str     0x0000000000000e68       0x67 /opt/toolchains/n64/mips64-elf/mips64-elf/lib/libc.a(lib_a-fiprintf.o)
                                        0x52c (size before relaxing)
 .debug_str     0x0000000000000ecf       0x4d /opt/toolchains/n64/mips64-elf/mips64-elf/lib/libc.a(lib_a-fopen.o)
                                        0x511 (size before relaxing)
 .debug_str     0x0000000000000f1c       0x68 /opt/toolchains/n64/mips64-elf/mips64-elf/lib/libc.a(lib_a-fread.o)
                                        0x53a (size before relaxing)
 .debug_str     0x0000000000000f84      0x159 /opt/toolchains/n64/mips64-elf/mips64-elf/lib/libc.a(lib_a-freer.o)
                                        0x62f (size before relaxing)
 .debug_str     0x00000000000010dd      0x138 /opt/toolchains/n64/mips64-elf/mips64-elf/lib/libc.a(lib_a-fseek.o)
                                        0x61e (size before relaxing)
 .debug_str     0x0000000000001215       0xa6 /opt/toolchains/n64/mips64-elf/mips64-elf/lib/libc.a(lib_a-fstatr.o)
                                        0x5dd (size before relaxing)
 .debug_str     0x00000000000012bb       0x46 /opt/toolchains/n64/mips64-elf/mips64-elf/lib/libc.a(lib_a-ftell.o)
                                        0x4fa (size before relaxing)
 .debug_str     0x0000000000001301       0x5a /opt/toolchains/n64/mips64-elf/mips64-elf/lib/libc.a(lib_a-fwalk.o)
                                        0x50b (size before relaxing)
 .debug_str     0x000000000000135b       0x85 /opt/toolchains/n64/mips64-elf/mips64-elf/lib/libc.a(lib_a-fwrite.o)
                                        0x54b (size before relaxing)
 .debug_str     0x00000000000013e0       0x44 /opt/toolchains/n64/mips64-elf/mips64-elf/lib/libc.a(lib_a-impure.o)
                                        0x506 (size before relaxing)
 .debug_str     0x0000000000001424       0x51 /opt/toolchains/n64/mips64-elf/mips64-elf/lib/libc.a(lib_a-makebuf.o)
                                        0x5f2 (size before relaxing)
 .debug_str     0x0000000000001475       0x45 /opt/toolchains/n64/mips64-elf/mips64-elf/lib/libc.a(lib_a-malloc.o)
                                        0x508 (size before relaxing)
 .debug_str     0x00000000000014ba       0xe9 /opt/toolchains/n64/mips64-elf/mips64-elf/lib/libc.a(lib_a-mallocr.o)
                                        0x6dd (size before relaxing)
 .debug_str     0x00000000000015a3       0xff /opt/toolchains/n64/mips64-elf/mips64-elf/lib/libc.a(lib_a-memcpy.o)
                                        0x132 (size before relaxing)
 .debug_str     0x00000000000016a2       0x72 /opt/toolchains/n64/mips64-elf/mips64-elf/lib/libc.a(lib_a-memset.o)
                                        0x179 (size before relaxing)
 .debug_str     0x0000000000001714       0x6b /opt/toolchains/n64/mips64-elf/mips64-elf/lib/libc.a(lib_a-mlock.o)
                                        0x50f (size before relaxing)
 .debug_str     0x000000000000177f       0x3f /opt/toolchains/n64/mips64-elf/mips64-elf/lib/libc.a(lib_a-openr.o)
                                        0x4f8 (size before relaxing)
 .debug_str     0x00000000000017be       0x42 /opt/toolchains/n64/mips64-elf/mips64-elf/lib/libc.a(lib_a-realloc.o)
                                        0x500 (size before relaxing)
 .debug_str     0x0000000000001800       0x61 /opt/toolchains/n64/mips64-elf/mips64-elf/lib/libc.a(lib_a-reallocr.o)
                                        0x5af (size before relaxing)
 .debug_str     0x0000000000001861       0x71 /opt/toolchains/n64/mips64-elf/mips64-elf/lib/libc.a(lib_a-reent.o)
                                        0x52b (size before relaxing)
 .debug_str     0x00000000000018d2       0x56 /opt/toolchains/n64/mips64-elf/mips64-elf/lib/libc.a(lib_a-refill.o)
                                        0x511 (size before relaxing)
 .debug_str     0x0000000000001928       0x53 /opt/toolchains/n64/mips64-elf/mips64-elf/lib/libc.a(lib_a-sbrkr.o)
                                        0x4fc (size before relaxing)
 .debug_str     0x000000000000197b       0x4c /opt/toolchains/n64/mips64-elf/mips64-elf/lib/libc.a(lib_a-sprintf.o)
                                        0x529 (size before relaxing)
 .debug_str     0x00000000000019c7       0x64 /opt/toolchains/n64/mips64-elf/mips64-elf/lib/libc.a(lib_a-stdio.o)
                                        0x52d (size before relaxing)
 .debug_str     0x0000000000001a2b       0x4e /opt/toolchains/n64/mips64-elf/mips64-elf/lib/libc.a(lib_a-strcmp.o)
                                        0x149 (size before relaxing)
 .debug_str     0x0000000000001a79       0xa0 /opt/toolchains/n64/mips64-elf/mips64-elf/lib/libc.a(lib_a-strcpy.o)
                                        0x157 (size before relaxing)
 .debug_str     0x0000000000001b19       0x42 /opt/toolchains/n64/mips64-elf/mips64-elf/lib/libc.a(lib_a-strlen.o)
                                        0x13d (size before relaxing)
 .debug_str     0x0000000000001b5b      0x15d /opt/toolchains/n64/mips64-elf/mips64-elf/lib/libc.a(lib_a-svfprintf.o)
                                        0x6d4 (size before relaxing)
 .debug_str     0x0000000000001cb8       0x3a /opt/toolchains/n64/mips64-elf/mips64-elf/lib/libc.a(lib_a-vfiprintf.o)
                                        0x670 (size before relaxing)
 .debug_str     0x0000000000001cf2       0x4a /opt/toolchains/n64/mips64-elf/mips64-elf/lib/libc.a(lib_a-writer.o)
                                        0x4fa (size before relaxing)
 .debug_str     0x0000000000001d3c       0x44 /opt/toolchains/n64/mips64-elf/mips64-elf/lib/libc.a(lib_a-wsetup.o)
                                        0x4f8 (size before relaxing)
 .debug_str     0x0000000000001d80       0x3e /opt/toolchains/n64/mips64-elf/mips64-elf/lib/libc.a(lib_a-abort.o)
                                        0x133 (size before relaxing)
 .debug_str     0x0000000000001dbe       0x41 /opt/toolchains/n64/mips64-elf/mips64-elf/lib/libc.a(lib_a-closer.o)
                                        0x4ea (size before relaxing)
 .debug_str     0x0000000000001dff       0xf5 /opt/toolchains/n64/mips64-elf/mips64-elf/lib/libc.a(lib_a-dtoa.o)
                                        0x5ed (size before relaxing)
 .debug_str     0x0000000000001ef4       0x45 /opt/toolchains/n64/mips64-elf/mips64-elf/lib/libc.a(lib_a-flags.o)
                                        0x4ed (size before relaxing)
 .debug_str     0x0000000000001f39       0x4b /opt/toolchains/n64/mips64-elf/mips64-elf/lib/libc.a(lib_a-fputwc.o)
                                        0x515 (size before relaxing)
 .debug_str     0x0000000000001f84       0x5c /opt/toolchains/n64/mips64-elf/mips64-elf/lib/libc.a(lib_a-fvwrite.o)
                                        0x54f (size before relaxing)
 .debug_str     0x0000000000001fe0       0x43 /opt/toolchains/n64/mips64-elf/mips64-elf/lib/libc.a(lib_a-isattyr.o)
                                        0x4ec (size before relaxing)
 .debug_str     0x0000000000002023      0x274 /opt/toolchains/n64/mips64-elf/mips64-elf/lib/libc.a(lib_a-locale.o)
                                        0x75c (size before relaxing)
 .debug_str     0x0000000000002297       0x41 /opt/toolchains/n64/mips64-elf/mips64-elf/lib/libc.a(lib_a-lseekr.o)
                                        0x4f8 (size before relaxing)
 .debug_str     0x00000000000022d8       0x53 /opt/toolchains/n64/mips64-elf/mips64-elf/lib/libc.a(lib_a-memchr.o)
                                        0x156 (size before relaxing)
 .debug_str     0x000000000000232b       0x4b /opt/toolchains/n64/mips64-elf/mips64-elf/lib/libc.a(lib_a-memmove.o)
                                        0x16f (size before relaxing)
 .debug_str     0x0000000000002376       0xf6 /opt/toolchains/n64/mips64-elf/mips64-elf/lib/libc.a(lib_a-mprec.o)
                                        0x5fa (size before relaxing)
 .debug_str     0x000000000000246c       0x3f /opt/toolchains/n64/mips64-elf/mips64-elf/lib/libc.a(lib_a-readr.o)
                                        0x4f8 (size before relaxing)
 .debug_str     0x00000000000024ab       0xf3 /opt/toolchains/n64/mips64-elf/mips64-elf/lib/libc.a(lib_a-signal.o)
                                        0x559 (size before relaxing)
 .debug_str     0x000000000000259e       0x50 /opt/toolchains/n64/mips64-elf/mips64-elf/lib/libc.a(lib_a-signalr.o)
                                        0x4f9 (size before relaxing)
 .debug_str     0x00000000000025ee       0x1a /opt/toolchains/n64/mips64-elf/mips64-elf/lib/libc.a(lib_a-svfiprintf.o)
                                        0x647 (size before relaxing)
 .debug_str     0x0000000000002608       0x48 /opt/toolchains/n64/mips64-elf/mips64-elf/lib/libc.a(lib_a-wbuf.o)
                                        0x4fc (size before relaxing)
 .debug_str     0x0000000000002650       0x56 /opt/toolchains/n64/mips64-elf/mips64-elf/lib/libc.a(lib_a-wcrtomb.o)
                                        0x526 (size before relaxing)
 .debug_str     0x00000000000026a6       0x5b /opt/toolchains/n64/mips64-elf/mips64-elf/lib/libc.a(lib_a-wctomb_r.o)
                                        0x535 (size before relaxing)
 .debug_str     0x0000000000002701       0x19 /opt/toolchains/n64/mips64-elf/mips64-elf/lib/libc.a(lib_a-callocr.o)
                                        0x52e (size before relaxing)
 .debug_str     0x000000000000271a       0x99 /opt/toolchains/n64/mips64-elf/mips64-elf/lib/libnosys.a(_exit.o)
                                         0xa5 (size before relaxing)

.debug_frame    0x0000000000000000     0x12a4
 .debug_frame   0x0000000000000000       0x28 /opt/toolchains/n64/mips64-elf/mips64-elf/lib/libm.a(lib_a-s_sin.o)
 .debug_frame   0x0000000000000028       0x30 /opt/toolchains/n64/mips64-elf/mips64-elf/lib/libm.a(lib_a-w_pow.o)
 .debug_frame   0x0000000000000058       0x3c /opt/toolchains/n64/mips64-elf/mips64-elf/lib/libm.a(lib_a-e_pow.o)
 .debug_frame   0x0000000000000094       0x30 /opt/toolchains/n64/mips64-elf/mips64-elf/lib/libm.a(lib_a-e_rem_pio2.o)
 .debug_frame   0x00000000000000c4       0x20 /opt/toolchains/n64/mips64-elf/mips64-elf/lib/libm.a(lib_a-e_sqrt.o)
 .debug_frame   0x00000000000000e4       0x20 /opt/toolchains/n64/mips64-elf/mips64-elf/lib/libm.a(lib_a-k_cos.o)
 .debug_frame   0x0000000000000104       0x48 /opt/toolchains/n64/mips64-elf/mips64-elf/lib/libm.a(lib_a-k_rem_pio2.o)
 .debug_frame   0x000000000000014c       0x20 /opt/toolchains/n64/mips64-elf/mips64-elf/lib/libm.a(lib_a-k_sin.o)
 .debug_frame   0x000000000000016c       0x20 /opt/toolchains/n64/mips64-elf/mips64-elf/lib/libm.a(lib_a-s_fabs.o)
 .debug_frame   0x000000000000018c       0x20 /opt/toolchains/n64/mips64-elf/mips64-elf/lib/libm.a(lib_a-s_finite.o)
 .debug_frame   0x00000000000001ac       0x20 /opt/toolchains/n64/mips64-elf/mips64-elf/lib/libm.a(lib_a-s_floor.o)
 .debug_frame   0x00000000000001cc       0x20 /opt/toolchains/n64/mips64-elf/mips64-elf/lib/libm.a(lib_a-s_fpclassify.o)
 .debug_frame   0x00000000000001ec       0x20 /opt/toolchains/n64/mips64-elf/mips64-elf/lib/libm.a(lib_a-s_matherr.o)
 .debug_frame   0x000000000000020c       0x20 /opt/toolchains/n64/mips64-elf/mips64-elf/lib/libm.a(lib_a-s_nan.o)
 .debug_frame   0x000000000000022c       0x24 /opt/toolchains/n64/mips64-elf/mips64-elf/lib/libm.a(lib_a-s_rint.o)
 .debug_frame   0x0000000000000250       0x2c /opt/toolchains/n64/mips64-elf/mips64-elf/lib/libm.a(lib_a-s_scalbn.o)
 .debug_frame   0x000000000000027c       0x20 /opt/toolchains/n64/mips64-elf/mips64-elf/lib/libm.a(lib_a-s_copysign.o)
 .debug_frame   0x000000000000029c       0x40 /opt/toolchains/n64/mips64-elf/mips64-elf/lib/libc.a(lib_a-assert.o)
 .debug_frame   0x00000000000002dc       0x20 /opt/toolchains/n64/mips64-elf/mips64-elf/lib/libc.a(lib_a-errno.o)
 .debug_frame   0x00000000000002fc       0x3c /opt/toolchains/n64/mips64-elf/mips64-elf/lib/libc.a(lib_a-fclose.o)
 .debug_frame   0x0000000000000338       0x58 /opt/toolchains/n64/mips64-elf/mips64-elf/lib/libc.a(lib_a-fflush.o)
 .debug_frame   0x0000000000000390      0x11c /opt/toolchains/n64/mips64-elf/mips64-elf/lib/libc.a(lib_a-findfp.o)
 .debug_frame   0x00000000000004ac       0x40 /opt/toolchains/n64/mips64-elf/mips64-elf/lib/libc.a(lib_a-fiprintf.o)
 .debug_frame   0x00000000000004ec       0x40 /opt/toolchains/n64/mips64-elf/mips64-elf/lib/libc.a(lib_a-fopen.o)
 .debug_frame   0x000000000000052c       0x54 /opt/toolchains/n64/mips64-elf/mips64-elf/lib/libc.a(lib_a-fread.o)
 .debug_frame   0x0000000000000580       0x48 /opt/toolchains/n64/mips64-elf/mips64-elf/lib/libc.a(lib_a-freer.o)
 .debug_frame   0x00000000000005c8       0x48 /opt/toolchains/n64/mips64-elf/mips64-elf/lib/libc.a(lib_a-fseek.o)
 .debug_frame   0x0000000000000610       0x2c /opt/toolchains/n64/mips64-elf/mips64-elf/lib/libc.a(lib_a-fstatr.o)
 .debug_frame   0x000000000000063c       0x3c /opt/toolchains/n64/mips64-elf/mips64-elf/lib/libc.a(lib_a-ftell.o)
 .debug_frame   0x0000000000000678       0x5c /opt/toolchains/n64/mips64-elf/mips64-elf/lib/libc.a(lib_a-fwalk.o)
 .debug_frame   0x00000000000006d4       0x48 /opt/toolchains/n64/mips64-elf/mips64-elf/lib/libc.a(lib_a-fwrite.o)
 .debug_frame   0x000000000000071c       0x30 /opt/toolchains/n64/mips64-elf/mips64-elf/lib/libc.a(lib_a-makebuf.o)
 .debug_frame   0x000000000000074c       0x30 /opt/toolchains/n64/mips64-elf/mips64-elf/lib/libc.a(lib_a-malloc.o)
 .debug_frame   0x000000000000077c       0x38 /opt/toolchains/n64/mips64-elf/mips64-elf/lib/libc.a(lib_a-mallocr.o)
 .debug_frame   0x00000000000007b4       0x20 /opt/toolchains/n64/mips64-elf/mips64-elf/lib/libc.a(lib_a-memcpy.o)
 .debug_frame   0x00000000000007d4       0x20 /opt/toolchains/n64/mips64-elf/mips64-elf/lib/libc.a(lib_a-memset.o)
 .debug_frame   0x00000000000007f4       0x30 /opt/toolchains/n64/mips64-elf/mips64-elf/lib/libc.a(lib_a-mlock.o)
 .debug_frame   0x0000000000000824       0x2c /opt/toolchains/n64/mips64-elf/mips64-elf/lib/libc.a(lib_a-openr.o)
 .debug_frame   0x0000000000000850       0x20 /opt/toolchains/n64/mips64-elf/mips64-elf/lib/libc.a(lib_a-realloc.o)
 .debug_frame   0x0000000000000870       0x38 /opt/toolchains/n64/mips64-elf/mips64-elf/lib/libc.a(lib_a-reallocr.o)
 .debug_frame   0x00000000000008a8       0x6c /opt/toolchains/n64/mips64-elf/mips64-elf/lib/libc.a(lib_a-reent.o)
 .debug_frame   0x0000000000000914       0x40 /opt/toolchains/n64/mips64-elf/mips64-elf/lib/libc.a(lib_a-refill.o)
 .debug_frame   0x0000000000000954       0x2c /opt/toolchains/n64/mips64-elf/mips64-elf/lib/libc.a(lib_a-sbrkr.o)
 .debug_frame   0x0000000000000980       0x40 /opt/toolchains/n64/mips64-elf/mips64-elf/lib/libc.a(lib_a-sprintf.o)
 .debug_frame   0x00000000000009c0       0x88 /opt/toolchains/n64/mips64-elf/mips64-elf/lib/libc.a(lib_a-stdio.o)
 .debug_frame   0x0000000000000a48       0x20 /opt/toolchains/n64/mips64-elf/mips64-elf/lib/libc.a(lib_a-strcmp.o)
 .debug_frame   0x0000000000000a68       0x20 /opt/toolchains/n64/mips64-elf/mips64-elf/lib/libc.a(lib_a-strcpy.o)
 .debug_frame   0x0000000000000a88       0x3c /opt/toolchains/n64/mips64-elf/mips64-elf/lib/libc.a(lib_a-svfprintf.o)
 .debug_frame   0x0000000000000ac4       0x74 /opt/toolchains/n64/mips64-elf/mips64-elf/lib/libc.a(lib_a-vfiprintf.o)
 .debug_frame   0x0000000000000b38       0x2c /opt/toolchains/n64/mips64-elf/mips64-elf/lib/libc.a(lib_a-writer.o)
 .debug_frame   0x0000000000000b64       0x2c /opt/toolchains/n64/mips64-elf/mips64-elf/lib/libc.a(lib_a-wsetup.o)
 .debug_frame   0x0000000000000b90       0x28 /opt/toolchains/n64/mips64-elf/mips64-elf/lib/libc.a(lib_a-abort.o)
 .debug_frame   0x0000000000000bb8       0x2c /opt/toolchains/n64/mips64-elf/mips64-elf/lib/libc.a(lib_a-closer.o)
 .debug_frame   0x0000000000000be4       0x64 /opt/toolchains/n64/mips64-elf/mips64-elf/lib/libc.a(lib_a-dtoa.o)
 .debug_frame   0x0000000000000c48       0x20 /opt/toolchains/n64/mips64-elf/mips64-elf/lib/libc.a(lib_a-flags.o)
 .debug_frame   0x0000000000000c68       0x4c /opt/toolchains/n64/mips64-elf/mips64-elf/lib/libc.a(lib_a-fputwc.o)
 .debug_frame   0x0000000000000cb4       0x3c /opt/toolchains/n64/mips64-elf/mips64-elf/lib/libc.a(lib_a-fvwrite.o)
 .debug_frame   0x0000000000000cf0       0x2c /opt/toolchains/n64/mips64-elf/mips64-elf/lib/libc.a(lib_a-isattyr.o)
 .debug_frame   0x0000000000000d1c       0x98 /opt/toolchains/n64/mips64-elf/mips64-elf/lib/libc.a(lib_a-locale.o)
 .debug_frame   0x0000000000000db4       0x2c /opt/toolchains/n64/mips64-elf/mips64-elf/lib/libc.a(lib_a-lseekr.o)
 .debug_frame   0x0000000000000de0       0x20 /opt/toolchains/n64/mips64-elf/mips64-elf/lib/libc.a(lib_a-memchr.o)
 .debug_frame   0x0000000000000e00       0x20 /opt/toolchains/n64/mips64-elf/mips64-elf/lib/libc.a(lib_a-memmove.o)
 .debug_frame   0x0000000000000e20      0x1f8 /opt/toolchains/n64/mips64-elf/mips64-elf/lib/libc.a(lib_a-mprec.o)
 .debug_frame   0x0000000000001018       0x2c /opt/toolchains/n64/mips64-elf/mips64-elf/lib/libc.a(lib_a-readr.o)
 .debug_frame   0x0000000000001044       0xb4 /opt/toolchains/n64/mips64-elf/mips64-elf/lib/libc.a(lib_a-signal.o)
 .debug_frame   0x00000000000010f8       0x3c /opt/toolchains/n64/mips64-elf/mips64-elf/lib/libc.a(lib_a-signalr.o)
 .debug_frame   0x0000000000001134       0x64 /opt/toolchains/n64/mips64-elf/mips64-elf/lib/libc.a(lib_a-svfiprintf.o)
 .debug_frame   0x0000000000001198       0x3c /opt/toolchains/n64/mips64-elf/mips64-elf/lib/libc.a(lib_a-wbuf.o)
 .debug_frame   0x00000000000011d4       0x4c /opt/toolchains/n64/mips64-elf/mips64-elf/lib/libc.a(lib_a-wcrtomb.o)
 .debug_frame   0x0000000000001220       0x3c /opt/toolchains/n64/mips64-elf/mips64-elf/lib/libc.a(lib_a-wctomb_r.o)
 .debug_frame   0x000000000000125c       0x28 /opt/toolchains/n64/mips64-elf/mips64-elf/lib/libc.a(lib_a-callocr.o)
 .debug_frame   0x0000000000001284       0x20 /opt/toolchains/n64/mips64-elf/mips64-elf/lib/libnosys.a(_exit.o)

.debug_ranges   0x0000000000000000      0x740
 .debug_ranges  0x0000000000000000      0x100 /opt/toolchains/n64/mips64-elf/mips64-elf/lib/libm.a(lib_a-e_pow.o)
 .debug_ranges  0x0000000000000100       0x60 /opt/toolchains/n64/mips64-elf/mips64-elf/lib/libm.a(lib_a-e_rem_pio2.o)
 .debug_ranges  0x0000000000000160       0x18 /opt/toolchains/n64/mips64-elf/mips64-elf/lib/libm.a(lib_a-k_cos.o)
 .debug_ranges  0x0000000000000178       0x70 /opt/toolchains/n64/mips64-elf/mips64-elf/lib/libm.a(lib_a-s_rint.o)
 .debug_ranges  0x00000000000001e8       0x30 /opt/toolchains/n64/mips64-elf/mips64-elf/lib/libm.a(lib_a-s_copysign.o)
 .debug_ranges  0x0000000000000218       0x30 /opt/toolchains/n64/mips64-elf/mips64-elf/lib/libc.a(lib_a-fflush.o)
 .debug_ranges  0x0000000000000248       0x18 /opt/toolchains/n64/mips64-elf/mips64-elf/lib/libc.a(lib_a-fread.o)
 .debug_ranges  0x0000000000000260       0x60 /opt/toolchains/n64/mips64-elf/mips64-elf/lib/libc.a(lib_a-mallocr.o)
 .debug_ranges  0x00000000000002c0       0x18 /opt/toolchains/n64/mips64-elf/mips64-elf/lib/libc.a(lib_a-memcpy.o)
 .debug_ranges  0x00000000000002d8       0x20 /opt/toolchains/n64/mips64-elf/mips64-elf/lib/libc.a(lib_a-memset.o)
 .debug_ranges  0x00000000000002f8      0x148 /opt/toolchains/n64/mips64-elf/mips64-elf/lib/libc.a(lib_a-reallocr.o)
 .debug_ranges  0x0000000000000440      0x138 /opt/toolchains/n64/mips64-elf/mips64-elf/lib/libc.a(lib_a-svfprintf.o)
 .debug_ranges  0x0000000000000578       0x78 /opt/toolchains/n64/mips64-elf/mips64-elf/lib/libc.a(lib_a-vfiprintf.o)
 .debug_ranges  0x00000000000005f0       0x60 /opt/toolchains/n64/mips64-elf/mips64-elf/lib/libc.a(lib_a-fputwc.o)
 .debug_ranges  0x0000000000000650       0x20 /opt/toolchains/n64/mips64-elf/mips64-elf/lib/libc.a(lib_a-fvwrite.o)
 .debug_ranges  0x0000000000000670       0x38 /opt/toolchains/n64/mips64-elf/mips64-elf/lib/libc.a(lib_a-mprec.o)
 .debug_ranges  0x00000000000006a8       0x30 /opt/toolchains/n64/mips64-elf/mips64-elf/lib/libc.a(lib_a-signal.o)
 .debug_ranges  0x00000000000006d8       0x50 /opt/toolchains/n64/mips64-elf/mips64-elf/lib/libc.a(lib_a-svfiprintf.o)
 .debug_ranges  0x0000000000000728       0x18 /opt/toolchains/n64/mips64-elf/mips64-elf/lib/libc.a(lib_a-callocr.o)
